:1000000000000320D101000025EF0100DDEE01001A
:10001000DDEE0100DDEE0100DDEE0100DDEE0100B0
:10002000DDEE0100DDEE0100DDEE010025EF010057
:1000300025EF0100DDEE0100B9190200BD1A020032
:1000400025EF010025EF010025EF010025EF01005C
:1000500025EF010025EF010025EF010025EF01004C
:1000600025EF010025EF010025EF010025EF01003C
:1000700025EF010025EF010025EF010025EF01002C
:1000800025EF010025EF010025EF010025EF01001C
:1000900025EF010025EF010025EF010025EF01000C
:1000A00025EF010025EF010025EF010025EF0100FC
:1000B00025EF010025EF010025EF010035FA0100D1
:1000C00025EF0100A501020025EF0100390702001C
:1000D00025EF01005D28020025EF010025EF01005A
:1000E00025EF010025EF010001E7010025EF0100E8
:1000F00025EF010025EF010025EF010025EF0100AC
:100100002D1F0200411F0200551F0200691F02003F
:1001100025EF0100C509020025EF010025EF0100D0
:1001200025EF010025EF010025EF010025EF01007B
:1001300025EF010025EF010025EF010025EF01006B
:1001400025EF010025EF01005529020025EF0100F0
:1001500025EF010025EF010025EF010025EF01004B
:1001600025EF010025EF010025EF010025EF01003B
:1001700025EF010025EF010025EF010025EF01002B
:1001800025EF010025EF010025EF010025EF01001B
:1001900025EF010025EF01004D2A020025EF0100A7
:1001A00025EF010025EF010025EF010025EF0100FB
:1001B00025EF010025EF010025EF010025EF0100EB
:1001C00025EF010025EF010025EF010025EF0100DB
:1001D0005C4B4CF2205210B51A804DF628121A8052
:1001E00000BF00BF1EF0A2FE574B4FF030621A60F6
:1001F000564A9A60564ADA60564B4FF470021A60BB
:10020000554B564A1A60564B1A78110703D51A787F
:1002100042F008021A70534B5349AA221A70534AEB
:10022000534B8B4204D252F8040F43F8040BF8E707
:10023000504B514900228B4202D243F8042BFAE77B
:100240004E494F4A002352F8230041F8230001335E
:10025000742BF8D14B4B4C4A802103F8011B93427D
:10026000FBD14A4B454A1A60494B8A221A70A3F5C2
:10027000805324225A70A0221A709A799207FCD5D2
:100280009A79D406FCD4434A937903F00C03082BE3
:10029000FAD1414B60221A7002331A78802AFCD1BD
:1002A0003C4B01221A715D225A719A799006FCD555
:1002B0009979384A4906FBD5384B394919600021EC
:1002C000596020231370937903F00C030C2BFAD19F
:1002D000344B354A1A60354A354C136813F4807331
:1002E00003D123604FF4A8531360324B324A1A6093
:1002F00000225A60072243F8042C304AC3F80C2D20
:1003000062B61EF065FF2368DA0705D52C481EF09B
:10031000E1FE2C4B2C4A1A602C4B1B785B0609D54E
:10032000284C294B22689A4204D125481EF0D2FE5F
:100330000023236024F086FD1EF0FEFD21F01EFE4A
:10034000FEE700BF0E20054030800440823F0400DD
:100350000100002B88ED00E0002008E0030000858C
:1003600002D0074000E007408812FF1F0CC70200C0
:100370003007FF1F8812FF1F8420FF1F0002FF1F8E
:100380000000000000E400E064E400E008ED00E0AC
:10039000005006400040064001E007404480044011
:1003A0000000060204800440C010070010D0034083
:1003B00014D0034014E000E01FBF02000000202022
:1003C000334001611CE00340A5C3945A00F007408C
:1003D000FFFFFFFFFFFFFFFFFFFFFFFFFFFFFFFF2D
:1003E000FFFFFFFFFFFFFFFFFFFFFFFFFFFFFFFF1D
:1003F000FFFFFFFFFFFFFFFFFFFFFFFFFFFFFFFF0D
:10040000FFFFFFFFFFFFFFFFFFFFFFFFDEF9FFFF23
:1004100010B5054C237833B9044B13B10448AFF33E
:1004200000800123237010BD8812FF1F0000000010
:1004300008C70200084B10B51BB108490848AFF3C4
:1004400000800848036803B910BD074B002BFBD0A0
:10045000BDE81040184700BF000000008C12FF1FCD
:1004600008C702008812FF1F0000000000690B6926
:100470009842D4BF00200120704700BF80698B697B
:100480000028B8BF4042002BB8BF5B429842D4BF9F
:1004900000200120704700BFF0B586460120DEF83D
:1004A0005870DEF83030BA6A106079683A680A44E9
:1004B0007A600EF1300493B15A69002A08DB9A6A17
:1004C00010605E6819683D695A6931445960521B71
:1004D00019690A445A6154F8043F002BECD1DEF844
:1004E0002430144ADEF81840DEF86C000021116058
:1004F000DB00516803F1804303F5603321440D2490
:1005000019611460DA68502122F08002DA60D96043
:1005100000B1F0BD7A68FB689A4200D0F0BDDEF809
:100520005C3001228EF82820002BF7D0BDE8F04087
:10053000184700BF00800340C36A00F12C0233B1AA
:100540000120D96A52F8043F0860002BF9D17047A6
:100550000C4BD3F8902072B9596A1A6AD3ED0A7A13
:1005600002FB01F207EE102A60EE277AB8EE477A16
:1005700087EE870A7047D3F89810D3F89420D3ED0C
:10058000277AEDE7EC15FF1F836D012280F890209C
:100590005B6872B6DFED0B6AD0ED207A90ED1F7AC2
:1005A00067EEA67AF4EEC77AC0ED1E7AD0ED227A15
:1005B000F1EE10FAD8BFF1EE677AC0ED237A62B699
:1005C000704700BF00000000036A8B4210B523D0C3
:1005D000C369994200D010BD8369002BFBD072B66D
:1005E000194AC369846900211160DB00516803F175
:1005F000804303F5603321440D2419611460DA68E7
:10060000502122F08002DA60D96062B60069036886
:10061000BDE810405B6818470446006903689B68A2
:10062000984794F82430002BD5D004F1080021F02D
:100630005BFC0023E06963601EF04AF8206ABDE8B5
:1006400010401EF045B800BF008003402DE9F04186
:100650008568002D31D0816D836F04464868D4F8D9
:10066000AC101B1A002BB8BF5B428B423ADBD4F8AC
:10067000B0108B422A4608DBE16F8B4265DB936842
:1006800023F002039360BDE8F081D4F888100029BC
:10069000F5D02B683B4A93421ED96A683A48B0FBB2
:1006A000F1F19B1A99420AD3CB1A002401200322AC
:1006B000AC60E8602B60AA602960BDE8F0816069E9
:1006C0000368002601240322AE601B68EC602960E9
:1006D000AA60BDE8F04118472B4BB3FBF1F129604C
:1006E000BDE8F081D4E92401D4F8A82002FB03F38B
:1006F000C61841F100073046394624F08BF907EE61
:10070000900AB1EEE70AB4EE400AF1EE10FA2ED1EB
:10071000FDEEC07A2A4617EE903A17EE901ADBB13A
:10072000002DB6D11949184D0E68B5FBF3F51EB171
:1007300002210120B047A26800200121032390601C
:10074000D16015609360BDE8F081CB1AD4F8A82081
:10075000D4E92601013BC9E7002D90D10B4B1B6862
:10076000002B8CD0022101209847A26887E73946E8
:10077000304624F04FF900EE100A22F081FBA56804
:10078000C6E700BF7FA9030000879303DC1BFF1FA0
:10079000F8B50446D0ED1F7A94ED1E7A806DF4EE24
:1007A000477AF1EE10FA436838D1FDEEC77A17EEBA
:1007B000905A94F890300BB1002D76D08368AB42FC
:1007C0002BD0002D0368B4BF4FF0FF3201229A42B4
:1007D00015D004F12801012608E013685B42012BC3
:1007E00013600BBF126B536B13601E6051F8042F24
:1007F000002AF2D1636FC3EB03139B003FD185EA5C
:10080000E572A2EBE572A368FAB9002B7AD09A6878
:1008100022F002029A608560F8BDF8BDD4ED236A2B
:10082000F5EEC06A77EEA67AF1EE10FAB4EEE77A4A
:100830002FDDF1EE10FAD8BFF0EE477ABDEEE77A81
:10084000C4ED1F7A17EE105AB3E7002B47D0196892
:10085000314EB14223D95E68304FB7FBF2F2891BAB
:100860008A4232D26069002601689E600127032611
:10087000DF6009681A609E608847A06DCBE7013B86
:10088000FDD185EAE572A2EBE572A368002ABCD02F
:10089000DBE7F1EE10FA58BFF0EE477ACEE71F49DA
:1008A000B1FBF2F21A608560F8BD04F10C0021F092
:1008B0001BFB206AA5601DF00BFF606A1DF008FF9E
:1008C000A36D9D6084F89050F8BD511A0027012651
:1008D00003249F60DE6019609C601A609BE71049EA
:1008E0000E4E0F68B6FBF2F627B101200221B84781
:1008F000A368A06D0024012103229C60D9601E60C2
:100900009A6088E7064B1B68002B80D001200221EB
:100910009847A368A06D7AE77FA903000087930337
:10092000DC1BFF1F70B5044608460D4625F008FB8A
:1009300023680246294620465B68BDE87040184798
:1009400038B5044608460D4625F0FAFA23680246F3
:1009500029465B68204698470546204621F056FB0D
:10096000284438BD38B5054621F0A0FB044628468A
:1009700021F04CFB204438BD38B5054621F096FBEC
:100980000446284621F042FB204438BD38B50A22EF
:100990000023054621F04AFB0446284621F036FB99
:1009A000204438BD38B5C9B2054621F089FB04465C
:1009B000284621F02BFB204438BD00BF10B509218B
:1009C0002C4820F093FE2C4821F020FBFE212B48E0
:1009D0001BF04EFC00282FD10A2128481BF048FCB0
:1009E00098B9182125481BF043FC00283AD10F2163
:1009F00022481BF03DFC50BB09212048204C1BF035
:100A000037FC002832D1206009E01D4C1D480A2324
:100A10001946236020F06AFE174821F0F7FA0C21EE
:100A2000194820F063FE2168134821F03FFB12486B
:100A3000BDE8104021F0EABA114C14480123092105
:100A4000236020F053FE0C4821F0E0FAE7E70C4C5D
:100A50000F480F230A21236020F048FE064821F0AA
:100A6000D5FADCE7064C0B481823F3E70A480923BC
:100A7000CEE700BF088602002408FF1F6019FF1F91
:100A80006C17FF1F208602005086020014860200A9
:100A9000388602002C8602004486020070B50D469E
:100AA00084B00A2106464148144620F01FFE29461C
:100AB0003F4821F0FBFA3E4821F0A8FABCB13D4B7B
:100AC000D3F8A420A2F10102B2FA82F252093A4C00
:100AD00023680193019923680093009B5B1A092BFB
:100AE000F9D9032E2FD8DFE806F0241A0F04224686
:100AF000EDE7002D51D12AB92E4B042093F8741044
:100B00001EF0FAFA04B070BD002D3DD1002AF9D1D3
:100B1000284B112093F877101EF0EEFAF2E755BB40
:100B2000002AEFD1234B162093F876101EF0E4FA3A
:100B3000E8E7BDB9002AE5D11E4B0E2093F87510E9
:100B40001EF0DAFADEE7002DDCD022681B4B0392A0
:100B500003991A6823680293029B5B1A9A42F9D898
:100B600004B070BD134B93F875100E2081F0010195
:100B70001EF0C2FAE9E70F4B93F87610162081F0C9
:100B800001011EF0B9FAE0E70A4B93F87710112043
:100B900081F001011EF0B0FAD7E7064B93F874100C
:100BA000042081F001011EF0A7FACEE76086020062
:100BB0002408FF1FEC15FF1F141CFF1F5807FF1F01
:100BC000F0B52DED028B85B0044601AE0DF10F0797
:100BD0000FE0FF2D66D001A8357025F0B1F9014670
:100BE00001A820F083FD334821F010FA0136BE42FF
:100BF00029D0236820465B6998470021C5B22E485A
:100C000020F074FD2B4821F001FA33212B4820F00D
:100C10006DFD284620F0EEFD0221294820F066FDFA
:100C20002946244821F042FA224821F0EFF9042D08
:100C3000CFD11921234820F059FD01361D4821F05C
:100C4000E5F9BE42D5D101A824F0ECF804211E48F4
:100C5000B0EE408AF0EE608A20F048FD01A825F051
:100C60006FF9014601A820F041FD124821F0CEF9AC
:100C70000721164820F03AFDB0EE480AF0EE680A67
:100C800004210C4821F01CFA0A4821F0BFF9B0EE0B
:100C9000480AF0EE680A05B0BDEC028BF0BD23688F
:100CA0005B699847236820461B69984700282046BF
:100CB000F5DC9BE72408FF1F54A002006C860200AD
:100CC000D4B20200A0860200BC860200C4860200E4
:100CD00003280FD8DFE800F00B0805020A48FFF7E9
:100CE0006FBF0A48FFF76CBF0948FFF769BF0948A3
:100CF000FFF766BF9FED020B704700BFAFF30080A8
:100D0000000000000000F0BF0408FF1FF407FF1FF1
:100D1000E407FF1F2408FF1F012828D0022813D052
:100D200010B19FED140A7047134A1169D368D2EDD0
:100D3000056A03FB01F307EE103A60EE267AB8EE7F
:100D4000477A87EE870A70470B4B5A6B012AE8D81F
:100D5000D96B9A6BD3ED116A02FB01F207EE102AF0
:100D600060EE267AB8EE477A87EE870A7047FFF77B
:100D7000EFBB00BF00000000EC15FF1F38B5434D6E
:100D80004348EA6BAB6B95ED107AD5ED127A414C86
:100D900003FB02F32DED048B08EE103AB8EE488AFF
:100DA000DFED3D8A28EE078A0D2167EEA88AF0EE76
:100DB000409A20F09BFC18EE100A23F0BFF941EC9A
:100DC000100B0221204621F07BF9204621F01EF96C
:100DD0001121324820F08AFC286C23F0AFF941EC55
:100DE000100B0221204621F06BF9204621F00EF96C
:100DF0000F212B4820F07AFC89EEA89A18EE900A71
:100E000023F09CF941EC100B0221204621F058F907
:100E1000204621F0FBF81021224820F067FC19EE53
:100E2000900A23F08BF941EC100B0221204621F0AF
:100E300047F9204621F0EAF807211B4820F056FC2C
:100E400019EE100A23F07AF941EC100B022120462A
:100E500021F036F928EE098A204621F0D7F808213A
:100E6000124820F043FC18EE100A23F067F941EC19
:100E7000100B0221204621F023F9204621F0C6F86C
:100E8000B0EE480ABDEC048B38BD00BFEC15FF1F67
:100E9000FC8602002408FF1FDB0FC9400C870200FC
:100EA0002087020030870200448702004C8702003E
:100EB000144A1548D2ED117AD16B936B80EE270A54
:100EC00010B503FB01F31921104C2DED028B08EE38
:100ED000103AB8EE488A28EE008A20F007FC18EE97
:100EE000100A23F02BF941EC100B0221204621F0CF
:100EF000E7F8204621F08AF8B0EE480ABDEC028BF4
:100F000010BD00BFEC15FF1F588702002408FF1F0B
:100F10000128F0EE407A1CD0022813D010B19FEDCA
:100F2000160A7047154AD2ED056A1169D36887EE33
:100F3000A67A03FB01F300EE103AB8EE400A20EE69
:100F4000070A70470D4B5B6B9BB1012BE7D1FFF795
:100F5000AFBF0A4AD2F8903023B9D2ED0A6A516A7B
:100F6000136AE4E7D2ED276AD2F89810D2F89430E9
:100F7000DDE7FFF703BF00BF00000000EC15FF1F17
:100F800038B52F4D2F4C95ED007AD4ED007AB5EEA3
:100F9000C07AF1EE10FA48BFB1EE477AF5EEC07AAA
:100FA00048BF85ED007AF1EE10FA44BFF1EE677AA2
:100FB000C4ED007A67EEA77A2DED048BE7EE077A91
:100FC00008EE100A17EE900A08EE901A23F0B6F811
:100FD00041EC100B21F094FE51EC100B23F0FAFBC6
:100FE00094ED006AD5ED006A07EE900A87EE867AE6
:100FF00087EEA69AF8EEE88AB8EEC88A67EE287AF5
:1010000017EE900A23F09AF841EC100B21F0D8FD6E
:1010100051EC100B23F0DEFB68EE097A206017EE2E
:10102000900A23F08BF841EC100B21F0C9FD51EC34
:10103000100B23F0CFFBBDEC048B286038BD00BF44
:101040007014FF1F6814FF1FBA4AF8B592E80A002F
:1010500003FB01F307EE903A92ED027AB64CF8EEFC
:10106000677A2DED028BB0EE408AF0EE608A67EE73
:10107000877A17EE900A23F061F841EC100B21F00B
:101080009FFD51EC100B23F05DFB09210546AB4899
:1010900020F02CFB2168AA4821F008F8A84820F08D
:1010A000B5FFB0EE480AF0EE680A0221A44821F02C
:1010B00007F8A34820F0AAFF2368013B042B00F2A5
:1010C000D180DFE803F045688BAD03009D4C2368B9
:1010D000022B84ED048B284600F0C78023F01CF817
:1010E00053EC182B23F0A8F923F02CFBA060162159
:1010F000954820F0FBFA2946914820F0D7FF1021AF
:10110000924820F0F3FAB0EE480AF0EE680A0221A5
:101110008B4820F0D5FF03218D4820F0E7FA062107
:101120008C4820F0E3FA06218B4820F0DFFAA16812
:10113000834820F0BBFF824820F068FF874B81483E
:101140001968BDEC028B1822BDE8F8401DF034BED2
:10115000834C2368022B84ED048B284600F0D58055
:1011600022F0DAFF53EC182B23F066F923F0EAFAA9
:10117000A06006217B4820F0B9FA0621764820F0CD
:10118000B5FAA1686E4820F091FF6D4820F03EFF4F
:10119000754B7348D4E7754C2368022B84ED048BA0
:1011A000284600F09E8022F0B7FF53EC182B23F066
:1011B00043F923F0C7FAA06006216D4820F096FAA3
:1011C0000621654820F092FAA1685D4820F06EFF84
:1011D0005B4820F01BFF674B6448B1E7664C23680F
:1011E000022B84ED048B284667D022F095FF53EC48
:1011F000182B23F021F923F0A5FAA06006215F48FF
:1012000020F074FA0621544820F070FAA1684C4886
:1012100020F04CFF4A4820F0F9FE594B56488FE722
:10122000584C2368022B84ED048B284631D022F0E1
:1012300073FF53EC182B23F0FFF823F083FAA06020
:101240000621514820F052FA0621434820F04EFA78
:10125000A1683B4820F02AFF394820F0D7FE4B4BCD
:1012600048486DE7BDEC028BF8BD22F055FF002227
:1012700006460F46464B51EC180B23F0DDF80246AC
:101280000B463046394622F0ADFF23F05BFAA060F2
:101290002DE722F041FF002206460F463C4B51EC61
:1012A000180B23F0C9F802460B463046394622F0A7
:1012B00099FF23F047FAA060C2E722F02DFF002239
:1012C00006460F46324B51EC180B23F0B5F8024698
:1012D0000B463046394622F085FF23F033FAA060F2
:1012E0008CE722F019FF002206460F46284B51ECEE
:1012F000180B23F0A1F802460B463046394622F07F
:1013000071FF23F01FFAA06056E722F005FF0022CC
:1013100006460F461E4B51EC180B23F08DF8024683
:101320000B463046394622F05DFF23F00BFAA060F1
:101330001FE700BFEC15FF1F7415FF1F7487020025
:101340002408FF1F5017FF1FA8870200C087020054
:1013500070B20200D4870200888702005C07FF1F7A
:10136000F016FF1F808702005007FF1F0817FF1F9E
:10137000908702005407FF1F2017FF1F9887020065
:101380006807FF1F3817FF1FA08702007807FF1F9D
:1013900000807640F8B51D212DED028B914D924CC9
:1013A000924E08EE100A924820F0A0F9914820F0E1
:1013B0002DFE95E8090003FB00F307EE903A95ED4A
:1013C000027AD4ED036A8C4A8C49F8EE677AB8EE5B
:1013D000C88A67EE877A002387EEA67A0B601360CF
:1013E000C7EE087A17EE900A22F0A8FE41EC100B27
:1013F00021F0E6FB51EC100B23F0A4F927683060D4
:10140000012F00F0B98065D3022F41D07C4F7D4879
:10141000152120F06BF93168764820F047FE7548B9
:1014200020F0F4FD2421784820F060F9E06822F0F3
:1014300085FE41EC100B02216E4820F041FE6D4804
:1014400020F0E4FD2921714820F050F9A06922F034
:1014500075FE41EC100B0221664820F031FE654814
:1014600020F0D4FD14216A4820F040F93968614821
:1014700020F01CFE5F4820F0C9FD1421654820F0D3
:1014800035F9BDEC028B5B48BDE8F84020F0BEBDED
:101490002B21614894ED068A20F028F9A06922F0FA
:1014A0004DFE41EC100B3946524820F009FE5148E0
:1014B00020F0ACFD6B6B002B00F08980012BA5D1D7
:1014C000B0EE480AFFF7F4FC4D4FBDEEC00A87EDC1
:1014D000000A9CE794ED067AD5ED057A484F87EE31
:1014E000278AD5ED047A95ED037AF8EE677AB8EE9F
:1014F000477A67EE887A67EE877A17EE900A22F0CD
:101500001DFE41EC100B21F05BFB51EC100B23F0A6
:1015100019F918213860414820F0E8F8A06922F054
:101520000DFE41EC100B0221324820F0C9FD31487C
:1015300020F06CFD24213A4820F0D8F8686922F0A8
:10154000FDFD41EC100B02212A4820F0B9FD29488D
:1015500020F05CFD1121334820F0C8F818EE100A85
:1015600022F0ECFD41EC100B0221224820F0A8FDF6
:10157000204820F04BFD4AE7D5F89030D4ED065ACC
:10158000F3B195ED276A95ED267AD5ED257A1C4FB6
:10159000C5EE866AB8EE477AF8EE677A26EE877A65
:1015A00067EE277A17EE900A22F0C8FD41EC100B87
:1015B00021F006FB51EC100B23F0C4F8386026E74D
:1015C00095ED0A6A95ED097AD5ED087ADFE7B0EE78
:1015D000480AFFF7D3FB0A4FBDEEC00A87ED000AA9
:1015E00015E700BFEC15FF1F0814FF1F8415FF1F30
:1015F000DC8702002408FF1FB412FF1F6418FF1FBE
:101600001C13FF1F8088020098880200C088020017
:10161000EC8802000489020054880200FC87020062
:1016200018880200408802000C4B1B68032B13D85B
:10163000DFE803F00E0A06020146094820F0C0BCAC
:101640000146084820F0BCBC0146074820F0B8BC61
:101650000146064820F0B4BC704700BF4807FF1F92
:101660000408FF1FF407FF1FE407FF1F2408FF1FE4
:10167000F0B585B06C496D4C6D4E6E4F684620F0EC
:1016800093FE00216846FFF7CFFF684620F04CFE2E
:101690006949684620F088FE00216846FFF7C4FFCC
:1016A000684620F041FE6549684620F07DFE002135
:1016B0006846FFF7B9FF684620F036FE5E49684687
:1016C00020F072FE00216846FFF7AEFF684620F06A
:1016D0002BFE5B49684620F067FE00216846FFF755
:1016E000A3FF684620F020FE5349684620F05CFEC8
:1016F00000216846FFF798FF684620F015FE514923
:10170000684620F051FE00216846FFF78DFF6846CD
:1017100020F00AFE4849684620F046FE002168464F
:10172000FFF782FF684620F0FFFD4749256891EDED
:10173000027ADFED466A3668454A91E8090003FB04
:1017400000F307EE903A06EE105AF8EE677AB8EE1C
:10175000C66A67EE877A012E86EE277A67EE267ACA
:10176000C2ED007A50D033D3022E0FD1D7ED007ADC
:101770003046B8EEE70AFFF7CFFA364B3046012283
:10178000002183ED000AFFF789F92568324A334BBF
:1017900015600821002532481D601FF0A7FF216851
:1017A000304820F083FC2F4820F030FC05212E48E3
:1017B0001FF09CFF39682B4820F078FC294820F066
:1017C00025FC294601220320FFF768F905B0F0BD8A
:1017D000D7ED007A0A69CB6891ED057A1D4DF8EED8
:1017E000E77A03FB02F327EE877A07EE903AF8EEEA
:1017F000677A0021C7EE276A08460122C5ED006A14
:10180000FFF74CF92568C1E7D7ED007AB8EEE70A93
:10181000FEF79EFE0F4B32463046002183ED000A54
:10182000FFF73CF92568B1E71C8902006418FF1F27
:101830000814FF1FB412FF1F308902003489020010
:10184000488902005C890200EC15FF1F0000B443C8
:101850009416FF1FBC13FF1F6C15FF1FF812FF1F0C
:1018600010A602002408FF1F00A2020010B5F0EE2F
:10187000407A0021F2EE046ABDEEE77AB8EEC77A4C
:10188000B4EE677AF1EE10FA04D00131062967EE62
:10189000A67AF1D11E4B1B68032B37D8DFE803F083
:1018A000291C0F0210EE100ACCB222F047FC41ECCA
:1018B000100B21461748BDE8104020F001BC10EE87
:1018C000100ACCB222F03AFC41EC100B214612482F
:1018D000BDE8104020F0F4BB10EE100ACCB222F0AC
:1018E0002DFC41EC100B21460C48BDE8104020F0C7
:1018F000E7BB10EE100ACCB222F020FC41EC100B3A
:1019000021460748BDE8104020F0DABB10BD00BFFB
:101910004807FF1F0408FF1FF407FF1FE407FF1F0E
:101920002408FF1F084B1B68032B0BD8DFE803F0CC
:10193000080604021EF054BE1EF0D8BA1DF06CBF9B
:101940001FF058BF704700BF4807FF1F2DE9F04147
:10195000DFF85080104F114E114D044601464046AD
:1019600020F02EFB404620F051FB2146384620F067
:1019700027FB384620F04AFB2146304620F020FB6A
:10198000304620F043FB2146284620F019FB28462C
:10199000BDE8F04120F03ABBE407FF1FF407FF1F4A
:1019A0000408FF1F2408FF1F2DE9F04FB24CA3B01D
:1019B00001210D201DF0B4FB23680893089A2368C9
:1019C0000793079BAC4D9B1A0E2BF8D9AB4BAC4938
:1019D0001E681EA820F0E8FC00211EA8FFF724FEC8
:1019E0001EA820F0A1FC0A2231461EA820F00EFD00
:1019F0001EA8FFF7ABFF1EA820F096FC40F2871050
:101A00001DF0EEFC0C219F481DF010FF03219E48A5
:101A10001DF00CFF2B680693069A23680593059B1F
:101A2000954D9B1A312BF8D90C2196481DF0FEFEDE
:101A3000032195481DF0FAFE2B680493049A23684D
:101A40000393039B8C4D9B1A312BF8D907218F48A8
:101A50001DF0ECFE03218C481DF0E8FE2B6802937C
:101A6000029A23680193019B9B1A312BF9D91DF02F
:101A70005FFF0028864D0CDD01230C2185482B607B
:101A80001FF034FE2968844820F010FB824820F0C3
:101A9000BDFA40F287101EF053F80C2179481EF071
:101AA0007DFA032178481EF079FA23680E930E9A86
:101AB00023680D930D9B704E9B1A312BF8D90C2186
:101AC00070481EF06BFA03216F481EF067FA336806
:101AD0000C930C9A23680B930B9B674E9B1A312B2C
:101AE000F8D9072169481EF059FA032166481EF00B
:101AF00055FA33680A930A9A23680993099B9B1A3B
:101B0000312BF9D91EF0CCFA00280CDD02230C2170
:101B100062482B601FF0EAFD29685F4820F0C6FA92
:101B20005D4820F073FA82201EF014FC0C21554809
:101B30001EF060FD032154481EF05CFD23681493E1
:101B4000149A23681393139B4B4E9B1A312BF8D98D
:101B50000C214C481EF04EFD03214B481EF04AFD5F
:101B600033681293129A23681193119B424E9B1A69
:101B7000312BF8D9072145481EF03CFD032142488E
:101B80001EF038FD33681093109A23680F930F9B53
:101B90009B1A312BF9D91EF061FD00280CDD0323BF
:101BA0000C213F482B601FF0A1FD29683A4820F026
:101BB0007DFA394820F02AFA0A213A483A4E1FF0B5
:101BC00095FD2968344820F071FA334820F01EFA58
:101BD000364B1B683746C6EB03083D46A83608EB74
:101BE00005001DF0A1F805F8010BB542F7D1304B07
:101BF000304E1B68B346C6EB03085D46343608EB2F
:101C000005001DF091F805F8010BB542F7D12A4BFC
:101C10002A4E1B683246C6EB03081546403608EBD1
:101C200005001DF081F805F8010BAE42F7D1244BF9
:101C3000244E1B68B246C6EB03085546343608EB03
:101C400005001DF071F805F8010BB542F7D11E4BE8
:101C50001E4D1E68A946761BC846103506EB0800C7
:101C60001DF062F808F8010BA845F7D1184B194D83
:101C70001E68A84630E000BF141CFF1F7420FF1F21
:101C80007089020078890200308902008889020088
:101C90004807FF1F908902002408FF1FA089020047
:101CA000B0890200C0890200EC15FF1F7C14FF1FE1
:101CB0009007FF1F2819FF1F3C07FF1F1418FF1F65
:101CC0008407FF1FC013FF1F8C07FF1F7415FF1F22
:101CD0005007FF1FF016FF1F761B183506EB080094
:101CE0001DF022F808F8010B4545F7D1C54BC64D4C
:101CF0001E68A846761B183506EB08001DF014F880
:101D000008F8010BA845F7D1C04BC14D1E68A84685
:101D1000761B183506EB08001DF006F808F8010BD5
:101D2000A845F7D1BB4BBC4D1E682B46761B984689
:101D3000403506EB08001CF0F7FF08F8010B45459D
:101D4000F7D1B64BB64D1E682B46761B98465C35D0
:101D500006EB08001CF0E8FF08F8010BA845F7D1D6
:101D6000B04BB14D1E682B46761B9846543506EB9A
:101D700008001CF0D9FF08F8010B4545F7D1AB4B23
:101D8000AB4D1E682B46761B9846603506EB080067
:101D90001CF0CAFF08F8010BA845F7D11321A5488C
:101DA0001FF0A4FCDBF83010A34820F07FF9A24814
:101DB00020F02CF91221A1481FF098FCDAF830101D
:101DC0009D4820F073F99C4820F020F91A219C4886
:101DD0001FF08CFCD9F80010974820F067F996485E
:101DE00020F014F9132197481FF080FC8A4B924889
:101DF00019680A22002320F019F98F4820F006F90B
:101E0000132191481FF072FC904B8B4819680A22ED
:101E1000002320F00BF9884820F0F8F812218C48B4
:101E20001FF064FC804B8448996C0A22002320F048
:101E3000FDF8814820F0EAF8172186481FF056FC8B
:101E40007B4B7D4819680A22002320F0EFF87A487E
:101E500020F0DCF8132180481FF048FC704B7648D6
:101E6000996B0A22002320F0E1F8734820F0CEF8A5
:101E7000012104201DF054F901210E201DF050F91C
:101E8000012116201DF04CF9012111201DF048F907
:101E9000012200210320FEF701FE00210846012255
:101EA000FEF7FCFD012210460021FEF7F7FD01229E
:101EB00000210220FEF7F2FD0221387E1DF030F9EC
:101EC0000221387F1DF02CF923681A931A9A23688F
:101ED0001993199B614D9B1A092BF8D90121387E62
:101EE0001DF00AF90121387F1DF006F9022197F84B
:101EF0002C001DF015F9022197F830001DF010F9A3
:101F00002B681893189A23681793179B534D9B1AA5
:101F1000092BF8D9012197F82C001DF0EDF80121CB
:101F200097F830001DF0E8F8022197F84C001DF0FA
:101F3000F7F8022197F850001DF0F2F8012197F808
:101F40004C001DF0D9F897F8500001211DF0D4F88D
:101F50002B681693169A23681593159B9B1A092BC9
:101F6000F9D9012118201DF0DBF8012118201DF0FE
:101F7000C3F801210F201DF0D3F801210F201DF01F
:101F8000BBF801210A201DF0CBF801210A201DF029
:101F9000B3F8012109201DF0C3F8012109201DF02B
:101FA000ABF8FEF70BFD012200210320FEF776FDC2
:101FB0002A4E032501210D201DF09EF823681E9353
:101FC0001E9A23681D931D9B9B1A312BF9D9002162
:101FD0000D201DF091F833681C931C9A23681B9305
:101FE0001B9B9B1AB3F5967FF8D3013DE2D10E21DE
:101FF0001B481FF07BFB104820F008F823B0BDE819
:10200000F08F00BF5407FF1F0817FF1F6807FF1F4F
:102010002017FF1F6C07FF1FAC15FF1F3407FF1FA2
:102020002013FF1F3807FF1F8014FF1F4C07FF1FDF
:102030000814FF1FCC8902002408FF1FE08902005A
:10204000F4890200108A0200248A02001418FF1F7B
:10205000388A02004C8A0200648A0200141CFF1FA6
:10206000788A020003280BD8DFE800F00806040293
:102070001EF004BB1EF024B81DF06ABC1FF0D0BADD
:102080000020704708B51DF053FC002801DD012039
:1020900008BD1EF005F8002801DD022008BD1EF075
:1020A000DDFA0028D4BF0020032008BD38B50D4C50
:1020B0002068FFF7D7FFC5B202E02068FFF7D2FF24
:1020C000FFF7E0FF0028F8DC042107481FF00EFBB3
:1020D000294606481FF0EAFF04481FF097FF2846EC
:1020E00038BD00BF4807FF1F888A02002408FF1F71
:1020F00008B5FFF7C7FF002808DB154B1868FFF786
:10210000B1FF144BC0B25328187001D0002008BD95
:10211000012200210320FEF7C1FC0F4B1B68012B9D
:1021200009D003D3022B0BD0012008BD0122104699
:102130000021FEF7B3FC012210460021FEF7AEFCA1
:10214000012200210220FEF7A9FC012008BD00BFEA
:102150004807FF1FF413FF1F0814FF1FF0B51C21D1
:1021600083B02748274C284D284E294F1FF0BEFA30
:1021700028481FF04BFF0E2127481FF0B7FA2168AF
:1021800024481FF093FF23481FF040FF00230193D2
:1021900009E0019B306818441CF0E0FD019B01330D
:1021A000142B019314DC2868FFF75CFFC0B2FF28F2
:1021B0002368014619D0032BEBD1019B3A680146F5
:1021C000D0181CF0CBFD019B0133142B0193EADDE9
:1021D0002368032B0CBF114B114B042219680DEB24
:1021E00002001CF0E9FD03B0F0BD032B0CBF084A50
:1021F000064A019B1068002118441CF0AFFDE7E778
:10220000908A02008007FF1F4807FF1F7C07FF1FFF
:102210004407FF1F2408FF1FB08A02008807FF1F22
:102220006007FF1F2DE9F04F95B0074604A819F08D
:10223000DBFF88201FF0AAFE0823102280E80C0094
:10224000C61800F18808354634462046002110346F
:1022500020F0AAF8A045F8D11721BF481FF046FA90
:10226000BE481FF0D3FE0CA80123BD4ABD491AF099
:10227000ABF80E9A9DF83C309DF8341006928DF81C
:102280001C308DF814100FAA0DF11D030DF12A005A
:1022900012F8011F03F8011B8342F9D1139B0B9322
:1022A0000CA819F0AFFF04A819F0DAFF002800F01D
:1022B000AF8104A819F0C2FF0A210446AA481FF002
:1022C00015FA214600230A22A4481FF0AFFEA348B6
:1022D0001FF09CFE002F4AD017F1060900F1B780CD
:1022E0000024A24610E0013C0CA819F0B9FF80467A
:1022F000002842D00CA819F0A5FF01340CA819F051
:1023000081FF4C4500F3A380012204A90CA81AF018
:10231000CFF80CA819F078FF804623F011FE014693
:1023200040461FF0E3F98D481FF070FE0CA819F02D
:102330006DFF0028D7D10CA819F066FF01468B4825
:1023400023F032FC0A2100285CD189481FF0CEF925
:102350000CA819F059FF804623F0F2FD01464046D3
:102360001FF0C4F97D48013C1FF050FEC2E7814BCD
:1023700064221A604FF00609B2E70F217E48DFF8A9
:10238000F4B11FF0B3F9214674481FF08FFE03210A
:102390007A481FF0ABF9DBF8001070481FF086FE9A
:1023A00004F1080303217548CBF800301FF09EF9B3
:1023B000DBF8001069481FF079FE68481FF026FE20
:1023C00068466F491FF0F0FF41466846FFF72CF959
:1023D00068461FF0A9FF2220FFF7A4FA631E00EE53
:1023E000103A4046B8EEC00AFFF740FA6846654921
:1023F0001FF0DAFF68464146FFF716F968461FF0FE
:1024000093FF77E760481FF071F9214653481FF0AA
:102410004DFE032159481FF069F90CA819F0F4FE8C
:10242000804623F08DFD014640461FF05FF90321F1
:1024300052481FF05BF9A74240F3F48006EB0A1103
:1024400046481FF0BDFD45481FF0E0FD4CE7012662
:10245000741E03214D481FF049F921463F481FF0E3
:1024600025FE032145481FF041F929463B481FF04E
:10247000A7FDB41E39481FF0C9FD052C04D8DFE8BC
:1024800004F068666462359541490CA81FF08CFF22
:1024900000210CA8FFF7C8F80CA81FF045FF3D4924
:1024A0000CA81FF081FF00210CA8FFF7BDF80CA8B5
:1024B0001FF03AFF29460CA81FF08AFF00210CA844
:1024C000FFF7B2F80CA81FF02FFF2E490CA81FF041
:1024D0006BFF00210CA8FFF7A7F80CA81FF024FF42
:1024E000072E00F08F8010350136B1E72A490CA87D
:1024F0001FF05AFF00210CA8FFF796F80CA81FF058
:1025000013FF24490CA81FF04FFF00210CA8FFF770
:102510008BF80CA81FF008FF29460CA81FF058FFE5
:1025200000210CA8FFF780F80CA81FF0FDFE15494C
:102530000CA81FF039FF0CA80021FFF775F80CA8B4
:102540001FF0F2FECFE71549D1E71549CFE715494E
:10255000CDE71549CBE700BFC08A02002408FF1F62
:10256000D88A02006019FF1FDC8A0200F88A020084
:10257000048B02007007FF1F208B02001C8B0200DF
:10258000308B0200448B0200108B02004C8B020047
:10259000508B0200688B0200CC8B0200B48B0200CF
:1025A0009C8B0200848B02006C8B020023490CA8D8
:1025B0001FF0FAFE00210CA8FFF736F80CA81FF058
:1025C000B3FE1F490CA81FF0EFFE00210CA8FFF777
:1025D0002BF80CA81FF0A8FE29460CA81FF0F8FE47
:1025E00000210CA8FFF720F80CA81FF09DFE15494C
:1025F0000CA81FF0D9FE0CA80021FFF715F80CA8B5
:102600001FF092FE04A819F0FDFD15B0BDE8F08F93
:102610000E210D481FF06AF804A819F0F3FD15B05B
:10262000BDE8F08F0CA819F0EFFD06EB0A18014683
:1026300040461FF041FF0AF1010AFFE6E48B020069
:10264000688B0200448B0200E88A020008B5084B40
:10265000DFED080AD3ED007A27EE800A20F0B0FB08
:1026600020F006FB044BD3ED007A20EE270A08BDCC
:102670006C14FF1FDB0FC9409815FF1F08B52C4ACB
:102680002C4B92ED010A93ED007ADFED2B6A2B4B78
:10269000B8EEC77A9B6BC6EE877A012BB8EEC00AFC
:1026A0002DED028B27EE800A3BD034D3022B2CD0A9
:1026B0009FED238AFFF7CAFF224A234B92ED007A4F
:1026C000002283F8902072B6DFED207A93ED206A25
:1026D000D3ED1F6A30EE480AB8EEC77AC0EE275A2B
:1026E000C5EE877A67EE867AF4EEE67AC3ED1E7A57
:1026F000D3ED227AF1EE10FAD8BFF1EE677AC3ED8E
:10270000237A62B6BDEC028B08BD114B93ED018AB2
:10271000B8EEC88ACEE70F4B93ED018AB8EEC88AAF
:10272000C8E70D4B93ED018AB8EEC88AC2E700BF37
:10273000B812FF1F5C19FF1FDB0FC9402013FF1FDA
:10274000000000006817FF1FD814FF1FCDCCCC3C41
:102750009816FF1FD417FF1F7017FF1F2DE9F04FAA
:102760001621ADB00446B1481EF0C0FFB0481FF0BE
:102770004DFC601E092800F27B84DFE810F0940015
:10278000CD01A9026B0179042603F901D303D30318
:102790000A00A84B1D680DF15008C8EB050544461A
:1027A0002BAE28191CF0C0FA04F8010BA642F8D190
:1027B000A14907A81FF0F8FD002107A8FEF734FF84
:1027C00007A81FF0B1FD2220FFF7ACF8DDED147A69
:1027D0000020B8EEE70AFFF749F8984907A81FF06C
:1027E000E3FD002107A8FEF71FFF07A81FF09CFDCF
:1027F000934907A81FF0D8FD002107A8FEF714FF92
:1028000007A81FF091FD2220FFF78CF8DDED187A64
:102810000020B8EE670AFFF729F8884907A81FF0DB
:10282000C3FD07A80021FEF7FFFE07A81FF07CFDEF
:10283000229B012B00F0EC86C0F0B886022B40F002
:102840009582804907A81FF0AFFD002107A8FEF779
:10285000EBFE07A81FF068FD2220FFF763F8DDED0F
:10286000177A0020B8EE670AFFF700F8734907A847
:102870001FF09AFD002107A8FEF7D6FE07A81FF05B
:1028800053FD714907A81FF08FFD002107A8FEF72F
:10289000CBFE07A81FF048FD2220FFF743F80020D9
:1028A000DDED1B7A1AE3694B1D6807AC2E1B0DF199
:1028B000500830191CF038FA04F8010BA045F8D183
:1028C000C8EB050521AE444628191CF02DFA04F882
:1028D000010BA642F8D1584903A81FF065FD00215D
:1028E00003A8FEF7A1FE03A81FF01EFD584903A888
:1028F0001FF05AFD002103A8FEF796FE03A81FF063
:1029000013FDDDED087A0020B8EEE70AFEF7AEFF12
:102910004A4903A81FF048FD002103A8FEF784FEE2
:1029200003A81FF001FD464903A81FF03DFD00214B
:1029300003A8FEF779FE03A81FF0F6FC444903A89C
:102940001FF032FD002103A8FEF76EFE03A81FF062
:10295000EBFCDDED107A0020B8EEE70AFEF786FF0B
:10296000364903A81FF020FD03A80021FEF75CFEF6
:1029700003A81FF0D9FC139C012C00F03B85022C0E
:1029800000F0D184002C40F0F1812E4903A81FF003
:102990000BFD214603A8FEF747FE03A81FF0C4FC69
:1029A0002B4903A81FF000FD214603A8FEF73CFEBB
:1029B00003A81FF0B9FCDDED097A2046B8EEE70A5E
:1029C000FEF754FF1D4903A81FF0EEFC214603A8A3
:1029D000FEF72AFE03A81FF0A7FC1B4903A81FF05F
:1029E000E3FC214603A8FEF71FFE03A81FF09CFC92
:1029F000174903A81FF0D8FC214603A8FEF714FED0
:102A000003A81FF091FCDDED117A2046B8EEE70A2D
:102A1000FEF72CFF094903A81FF0C6FC03A82146B6
:102A2000FEF702FE03A81FF07FFC9FE1FC8B020073
:102A30002408FF1F3407FF1F148C0200448B020080
:102A4000288C02003C8C0200508C02009007FF1F73
:102A5000688B0200924B1D680DF15008C8EB05050C
:102A6000444624AE28191CF05FF904F8010BA64275
:102A7000F8D1149A052A00F279810123934013F0CA
:102A8000240440F0E98313F0120540F03A8613F075
:102A9000090F00F06B8107A882491FF085FC2946C9
:102AA00007A8FEF7C1FD07A81FF03EFC2220FEF795
:102AB00039FFDDED157A2846B8EEE70AFEF7D6FEB7
:102AC00007A879491FF070FC294607A8FEF7ACFD5E
:102AD00007A81FF029FC07A874491FF065FC2946C8
:102AE00007A8FEF7A1FD07A81FF01EFC2220FEF795
:102AF00019FFDDED167A2846B8EE670AFEF7B6FE36
:102B000007A869491FF050FC07A82946FEF78CFD6D
:102B100007A81FF009FC29E1654B1D680DF150085D
:102B2000C8EB0505444621AE28191CF0FDF804F851
:102B3000010BA642F8D11E9B5E4801930B21DDF8E4
:102B400054B0DDF874A0DDF85890179F1F9E189DB3
:102B5000149C1EF0CBFD58481FF058FA209B032B05
:102B600000F20481DFE813F03003FC02C8028702A0
:102B7000524B1D680DF15008C8EB0505444629AEBF
:102B800028191CF0D1F804F8010BA642F8D14C49E1
:102B900007A81FF009FC002107A8FEF745FD07A8BC
:102BA0001FF0C2FB2220FEF7BDFEDDED147A0020EF
:102BB000B8EEE70AFEF75AFE3B4907A81FF0F4FB00
:102BC000002107A8FEF730FD07A81FF0ADFB3D4927
:102BD00007A81FF0E9FB002107A8FEF725FD07A8BD
:102BE0001FF0A2FB2220FEF79DFEDDED1C7A0020E7
:102BF000B8EE670AFEF73AFE2B4907A81FF0D4FB90
:102C0000002107A8FEF710FD07A81FF08DFB072184
:102C10002D481EF06BFD269C2748214600230A22E2
:102C20001FF004FA24481FF0F1F9012C00F048834A
:102C3000C0F01484022C40F099801A4907A81FF0B4
:102C4000B3FB002107A8FEF7EFFC07A81FF06CFB01
:102C50002220FEF767FE1D4B93ED030A0020B8EE1D
:102C6000C00AFEF703FE104907A81FF09DFB0021D4
:102C700007A8FEF7D9FC07A81FF056FB0B4907A8C9
:102C80001FF092FB002107A8FEF7CEFC07A81FF05B
:102C90004BFB2220FEF746FE0020DDED1F7A1DE1F2
:102CA0006C07FF1F3C8C0200448B0200508C02001A
:102CB0008407FF1FC08C02002408FF1F3807FF1F76
:102CC000148C0200288C0200B88C02008014FF1FB4
:102CD0008A4B1D6807AC2D1B0BAE28191CF024F87D
:102CE00004F8010BA642F8D10DF150088449404682
:102CF0001FF05AFB00214046FEF796FC40461FF0AD
:102D000013FB2220FEF70EFEDDED087A0020B8EE60
:102D1000E70AFEF7ABFD7B4940461FF045FB00216B
:102D20004046FEF781FC40461FF0FEFA76494046D9
:102D30001FF03AFB00214046FEF776FC40461FF0AC
:102D4000F3FA2220FEF7EEFDDDED0A7A0020B8EE60
:102D5000670AFEF78BFD6B4940461FF025FB404696
:102D60000021FEF761FC40461FF0DEFA674940464D
:102D70001FF01AFB00214046FEF756FC40461FF0AC
:102D8000D3FA634940461FF00FFB00214046FEF78F
:102D90004BFC40461FF0C8FA5E4940461FF004FB5A
:102DA00000214046FEF740FC40461FF0BDFA58495E
:102DB00040461FF0F9FA00214046FEF735FC404638
:102DC0001FF0B2FA2DB0BDE8F08F534B1D680DF126
:102DD0005008C8EB0505444624AE28191BF0A4FF93
:102DE00004F8010BA642F8D1454907A81FF0DCFA08
:102DF000002107A8FEF718FC07A81FF095FA22206B
:102E0000FEF790FDDDED157A0020B8EEE70AFEF73B
:102E10002DFD3C4907A81FF0C7FA002107A8FEF7BF
:102E200003FC07A81FF080FA374907A81FF0BCFA77
:102E3000002107A8FEF7F8FB07A81FF075FA22206B
:102E4000FEF770FDDDED167A0020B8EE670AFEF79A
:102E50000DFD2C4907A81FF0A7FA07A80021FEF7CF
:102E6000E3FB07A81FF060FA149B012B00F02883F6
:102E7000C0F06A83022B7FF479AF284907A81FF0BE
:102E800093FA002107A8FEF7CFFB07A81FF04CFA22
:102E90002220FEF747FDDDED1B7A0020B8EEE70AA1
:102EA000FEF7E4FC174907A81FF07EFA002107A8E7
:102EB000FEF7BAFB07A81FF037FA194907A81FF059
:102EC00073FA002107A8FEF7AFFB07A81FF02CFA42
:102ED0002220FEF727FDDDED1C7A0020B8EE670A00
:102EE000FEF7C4FC074907A81FF05EFA07A80021F7
:102EF000FEF79AFB07A81FF017FA37E78C07FF1FAA
:102F0000148C0200448B0200288C0200F48C020016
:102F1000308902000C8D02003C07FF1F3C8C020030
:102F2000508C0200C24B1D680DF15008C8EB05051E
:102F300044462CAE28191BF0F7FE04F8010BA642FC
:102F4000F8D1BC49BC4C07A81FF02EFA002107A8F5
:102F5000FEF76AFB07A81FF0E7F92220FEF7E2FC64
:102F6000DDED207A0020B8EEE70AFEF77FFCB349DA
:102F700007A81FF019FA002107A8FEF755FB07A8BC
:102F80001FF0D2F9AE4907A81FF00EFA002107A8DA
:102F9000FEF74AFB07A81FF0C7F92220FEF7C2FC84
:102FA000289D07EE905A0020B8EE670AFEF75EFCF7
:102FB000A24907A81FF0F8F9002107A8FEF734FB83
:102FC00007A81FF0B1F90F219E481EF08FFB0023C8
:102FD0000A22216D9C481FF029F89B481FF016F823
:102FE00016219A481EF082FB002329460A229648A1
:102FF0001FF01CF894481FF009F82368012B00F01B
:103000004D83C0F01983022B7FF4B0AE904907A81E
:103010001FF0CAF9002107A8FEF706FB07A81FF05A
:1030200083F92220FEF77EFCDDED237A0020B8EE46
:10303000E70AFEF71BFC814907A81FF0B5F900213C
:1030400007A8FEF7F1FA07A81FF06EF9814907A853
:103050001FF0AAF9002107A8FEF7E6FA07A81FF05B
:1030600063F92220FEF75EFC0020DDED2B7A35E7C8
:103070000DF150087AE66F4907A81FF095F9002175
:1030800007A8FEF7D1FA07A81FF04EF92220FEF795
:1030900049FC07EE90BA0020B8EEE70AFEF7E6FB1F
:1030A000664907A81FF080F9002107A8FEF7BCFABF
:1030B00007A81FF039F9624907A81FF075F9002128
:1030C00007A8FEF7B1FA07A81FF02EF92220FEF795
:1030D00029FC07EE90AAB8EEE70A0020FEF7C6FB2F
:1030E00007A856491FF060F907A80021FEF79CFACF
:1030F00007A81FF019F939E6554907A81FF054F938
:10310000002107A8FEF790FA07A81FF00DF922206A
:10311000FEF708FC07EE905A0020B8EEE70AFEF72B
:10312000A5FB464907A81FF03FF9002107A8FEF7B5
:103130007BFA07A81FF0F8F8464907A81FF034F9F2
:10314000002107A8FEF770FA07A81FF0EDF822206B
:10315000FEF7E8FB07EE904A0020B8EEE70ABDE76D
:103160003B4907A81FF020F9002107A8FEF75CFAE9
:1031700007A81FF0D9F82220FEF7D4FB07EE907ABB
:103180000020B8EEE70AFEF771FB2C4907A81FF0F4
:103190000BF9002107A8FEF747FA07A81FF0C4F8AB
:1031A0002C4907A81FF000F9002107A8FEF73CFAF8
:1031B00007A81FF0B9F82220FEF7B4FB07EE906ACB
:1031C0000020B8EEE70A89E7214907A81FF0ECF8CC
:1031D000002107A8FEF728FA07A81FF0A5F822206B
:1031E000FEF7A0FB07EE909A0020B8EEE70AFEF784
:1031F0003DFB124907A81FF0D7F8002107A8FEF7EA
:1032000013FA07A81FF090F8124907A81FF0CCF88E
:10321000002107A8FEF708FA07A81FF085F822206A
:10322000FEF780FBDDED017A0020B8EEE70A55E7F6
:103230004C07FF1F148C02000814FF1F448B020070
:10324000288C0200CC8C02002408FF1FDC8C0200BA
:103250003C8C0200508C0200B24907A81FF0A4F871
:10326000002107A8FEF7E0F907A81FF05DF822206B
:10327000FEF758FBDDED1B7A0020B8EEE70AFEF7FB
:10328000F5FAA94907A81FF08FF8002107A8FEF753
:10329000CBF907A81FF048F8A44907A81FF084F845
:1032A000002107A8FEF7C0F907A81FF03DF822206B
:1032B000FEF738FBDDED1C7A0020B8EE670A0DE75B
:1032C000984907A81FF070F8002107A8FEF7ACF98D
:1032D00007A81FF029F82220FEF724FB944B93ED5A
:1032E000020A0020B8EEC00AFEF7C0FA8E4907A80D
:1032F0001FF05AF8002107A8FEF796F907A81FF05B
:1033000013F88A4907A81FF04FF8002107A8FEF715
:103310008BF907A81FF008F82220FEF703FB002016
:10332000DDED1E7ADAE5182182481EF0DFF9824BC6
:10333000824819681EF0BAFE80481EF067FE192107
:103340007F481EF0D3F914997C481EF0AFFE7B48ED
:103350001EF05CFE18217B481EF0C8F9079C7748D8
:1033600021461EF0A3FE75481EF050FE6D4903A8CD
:103370001FF01AF8002103A8FEF756F903A81EF063
:10338000D3FF2220FEF7CEFADDED0B7A0020B8EE57
:10339000E70AFEF76BFA644903A81FF005F800215D
:1033A00003A8FEF741F903A81EF0BEFF64201BF03E
:1033B000BDFE5E4903A81EF0F7FF002103A8FEF73B
:1033C00033F903A81EF0B0FF2220FEF7ABFA07EE98
:1033D000904AB8EEE70A0020FEF748FA524903A8DF
:1033E0001EF0E2FF03A80021FEF71EF903A81EF05D
:1033F0009BFFBBE44B4903A81EF0D6FF002103A8A6
:10340000FEF712F903A81EF08FFF2220FEF78AFABA
:10341000DDED0A7A0020B8EEE70AFEF727FA424906
:1034200003A81EF0C1FF002103A8FEF7FDF803A8C2
:103430001EF07AFF3D4903A81EF0B6FF002103A845
:10344000FEF7F2F803A81EF06FFF2220FEF76AFADB
:10345000DDED127A0020B8EEE70ABDE7314907A892
:103460001EF0A2FF002107A8FEF7DEF807A81EF055
:103470005BFF2220FEF756FADDED157A0020B8EE4C
:10348000E70AFEF7F3F9284907A81EF08DFF00218F
:1034900007A8FEF7C9F807A81EF046FF234907A8AA
:1034A0001EF082FF002107A8FEF7BEF807A81EF055
:1034B0003BFF2220FEF736FA0020DDED1D7A0DE5F8
:1034C000184907A81EF070FF002107A8FEF7ACF806
:1034D00007A81EF029FF2220FEF724FADDED197A55
:1034E000B8EEE70A0020FEF7C1F90F4907A81EF061
:1034F0005BFF002107A8FEF797F807A81EF014FF4E
:103500000A4907A81EF050FF002107A8FEF78CF813
:1035100007A81EF009FF2220FEF704FA0020DDEDC7
:103520001A7ADBE43C8C0200448B0200508C0200CF
:103530008014FF1F648C02002819FF1F2408FF1F3E
:10354000808C02009C8C02008F4907A81EF02CFF83
:10355000002107A8FEF768F807A81EF0E5FE222064
:10356000FEF7E0F9DDED177A0020B8EEE70AFEF786
:103570007DF9864907A81EF017FF002107A8FEF76E
:1035800053F807A81EF0D0FE814907A81EF00CFFD3
:10359000002107A8FEF748F807A81EF0C5FE222064
:1035A000FEF7C0F90020DDED187A97E4764907A808
:1035B0001EF0FAFE002107A8FEF736F807A81EF055
:1035C000B3FE2220FEF7AEF9DDED157A0020B8EE4D
:1035D000E70AFEF74BF96D4907A81EF0E5FE00214A
:1035E00007A8FEF721F807A81EF09EFE684907A865
:1035F0001EF0DAFE002107A8FEF716F807A81EF055
:1036000093FE2220FEF78EF90020DDED197A65E4A5
:103610005D4907A81EF0C8FE002107A8FEF704F8C0
:1036200007A81EF081FE2220FEF77CF9DDED167A58
:103630000020B8EE670A56E7534907A81EF0B4FE0B
:10364000002107A8FDF7F0FF07A81EF06DFE22205D
:10365000FEF768F9DDED217A0020B8EEE70AFEF703
:1036600005F94A4907A81EF09FFE002107A8FDF7AB
:10367000DBFF07A81EF058FE454907A81EF094FE80
:10368000002107A8FDF7D0FF07A81EF04DFE22205D
:10369000FEF748F90020DDED297A1FE43A4907A832
:1036A0001EF082FE002107A8FDF7BEFF07A81EF04E
:1036B0003BFE2220FEF736F9DDED227A0020B8EE3F
:1036C000E70AFEF7D3F8314907A81EF06DFE002186
:1036D00007A8FDF7A9FF07A81EF026FE2C4907A89A
:1036E0001EF062FE002107A8FDF79EFF07A81EF04E
:1036F0001BFE2220FEF716F90020DDED2A7AFFF7E7
:10370000EDBB07A820491EF04FFE214607A8FDF794
:103710008BFF07A81EF008FE2220FEF703F9DDED5F
:10372000187A2046B8EEE70AFEF7A0F807A817496E
:103730001EF03AFE214607A8FDF776FF07A81EF007
:10374000F3FD07A812491EF02FFE214607A8FDF73A
:103750006BFF07A81EF0E8FD2220FEF7E3F8DDED81
:10376000197A2046B8EE670AFEF780F807A80749DD
:103770001EF01AFE07A82146FDF756FF07A81EF007
:10378000D3FDFFF7F3BA00BF3C8C0200448B02006C
:10379000508C020070B5E84BAEB01D6804AC2D1B18
:1037A0002EAE28191BF0C0FA04F8010BB442F8D170
:1037B000E249E34DE34C68461EF0F6FD0021684601
:1037C000FDF732FF68461EF0AFFD2220FEF7AAF893
:1037D000DDED047A0020B8EE670AFEF747F8DA4913
:1037E00068461EF0E1FD00216846FDF71DFF6846B2
:1037F0001EF09AFDD54968461EF0D6FD00216846A8
:10380000FDF712FF68461EF08FFD2220FEF78AF8B2
:10381000DDED057A0020B8EE670AFEF727F8CA4901
:1038200068461EF0C1FD00216846FDF7FDFE6846B2
:103830001EF07AFDC64968461EF0B6FD00216846B6
:10384000FDF7F2FE68461EF06FFD2220FEF76AF8D3
:103850009DED060A0420FEF709F8BB4968461EF0F4
:10386000A3FD00216846FDF7DFFE68461EF05CFD03
:10387000B84968461EF098FD00216846FDF7D4FE61
:1038800068461EF051FD2220FEF74CF89DF884108A
:103890006846002914BF294621461EF085FD0021F7
:1038A0006846FDF7C1FE68461EF03EFDA649684623
:1038B0001EF07AFD00216846FDF7B6FE68461EF050
:1038C00033FDA54968461EF06FFD00216846FDF7EF
:1038D000ABFE68461EF028FD2220FEF723F8DDED42
:1038E000257A0020B8EE670AFDF7C0FF96496846C2
:1038F0001EF05AFD00216846FDF796FE68461EF050
:1039000013FD964968461EF04FFD00216846FDF7FD
:103910008BFE68461EF008FD2220FEF703F8DDED61
:10392000267A0020B8EE670AFDF7A0FF86496846B0
:103930001EF03AFD00216846FDF776FE68461EF04F
:10394000F3FC874968461EF02FFD00216846FDF70D
:103950006BFE68461EF0E8FC2220FDF7E3FFDDED7C
:10396000077A0020B8EE670AFDF780FF76496846BF
:103970001EF01AFD00216846FDF756FE68461EF04F
:10398000D3FC784968461EF00FFD00216846FDF71C
:103990004BFE68461EF0C8FC2220FDF7C3FFDDED9C
:1039A000087A0020B8EE670AFDF760FF66496846AE
:1039B0001EF0FAFC00216846FDF736FE68461EF050
:1039C000B3FC694968461EF0EFFC00216846FDF72C
:1039D0002BFE68461EF0A8FC2220FDF7A3FF9DEDFC
:1039E000090A0420FDF742FF574968461EF0DCFC37
:1039F00000216846FDF718FE68461EF095FC5B49FD
:103A000068461EF0D1FC00216846FDF70DFE6846B1
:103A10001EF08AFC2220FDF785FF9DF88510684680
:103A2000002914BF294621461EF0BEFC002168462D
:103A3000FDF7FAFD68461EF077FC434968461EF024
:103A4000B3FC00216846FDF7EFFD68461EF06CFCF4
:103A5000474968461EF0A8FC00216846FDF7E4FDD2
:103A600068461EF061FC2220FDF75CFFDDED0C7A5C
:103A70000020B8EE670AFDF7F9FE334968461EF0EC
:103A800093FC00216846FDF7CFFD68461EF04CFC14
:103A9000384968461EF088FC00216846FDF7C4FDE1
:103AA00068461EF041FC2220FDF73CFFDDED0D7A5B
:103AB0000020B8EE670AFDF7D9FE234968461EF0DC
:103AC00073FC00216846FDF7AFFD68461EF02CFC34
:103AD000294968461EF068FC00216846FDF7A4FDF0
:103AE00068461EF021FC2220FDF71CFF9DED0E0A0A
:103AF0000520FDF7BBFE144968461EF055FC002169
:103B00006846FDF791FD68461EF00EFC1B496846AD
:103B10001EF04AFC00216846FDF786FD68461EF04F
:103B200003FC2220FDF7FEFE9DF886106846002962
:103B300014BF2946214623E07C14FF1F308D02006C
:103B4000248D0200288D0200448B0200488D020063
:103B5000608D0200788D0200908D0200A48D02001D
:103B6000BC8D0200CC8D0200DC8D0200EC8D0200C9
:103B7000FC8D02000C8E02001C8E02002C8E0200B6
:103B80001EF012FC00216846FDF74EFD68461EF04F
:103B9000CBFBE84968461EF007FC00216846FDF7AC
:103BA00043FD68461EF0C0FBE34968461EF0FCFB7F
:103BB00000216846FDF738FD68461EF0B5FB22205F
:103BC000FDF7B0FEDDED297A0020B8EE670AFDF7BB
:103BD0004DFED84968461EF0E7FB00216846FDF718
:103BE00023FD68461EF0A0FBD44968461EF0DCFBAE
:103BF00000216846FDF718FD68461EF095FB22205F
:103C0000FDF790FEDDED2A7A0020B8EE670AFDF799
:103C10002DFEC84968461EF0C7FB00216846FDF727
:103C200003FD68461EF080FBC54968461EF0BCFBDC
:103C300000216846FDF7F8FC68461EF075FB22205F
:103C4000FDF770FE9DED2B0A0520FDF70FFEB9492B
:103C500068461EF0A9FB00216846FDF7E5FC6846B2
:103C60001EF062FBB74968461EF09EFB00216846C5
:103C7000FDF7DAFC68461EF057FB2220FDF752FEE6
:103C80009DF8B0106846002914BF294621461EF051
:103C90008BFB00216846FDF7C7FC68461EF044FB1D
:103CA000A44968461EF080FB68460021FDF7BCFC75
:103CB00068461EF039FB289B012B00F0E581A249E4
:103CC00068461EF071FB00216846FDF7ADFC6846B2
:103CD0001EF02AFB9D4968461EF066FB00216846DF
:103CE000FDF7A2FC68461EF01FFB994968461EF0CE
:103CF0005BFB00216846FDF797FC68461EF014FB4D
:103D0000924968461EF050FB00216846FDF78CFC86
:103D100068461EF009FB8F4968461EF045FB0021EE
:103D20006846FDF781FC68461EF0FEFA8749684642
:103D30001EF03AFB00216846FDF776FC68461EF04F
:103D4000F3FA854968461EF02FFB00216846FDF70F
:103D50006BFC68461EF0E8FA7C4968461EF024FBBE
:103D600000216846FDF760FC68461EF0DDFA7B49DD
:103D700068461EF019FB00216846FDF755FC6846B1
:103D80001EF0D2FA2220FDF7CDFDDDED127A0020E3
:103D9000B8EE670AFDF76AFD664968461EF004FB47
:103DA00000216846FDF740FC68461EF0BDFA6C49EC
:103DB00068461EF0F9FA00216846FDF735FC6846B2
:103DC0001EF0B2FA2220FDF7ADFDDDED137A0020E2
:103DD000B8EE670AFDF74AFD564968461EF0E4FA58
:103DE00000216846FDF720FC68461EF09DFA5D49FB
:103DF00068461EF0D9FA00216846FDF715FC6846B2
:103E00001EF092FA2220FDF78DFD9DED140A04208C
:103E1000FDF72CFD474968461EF0C6FA00216846AA
:103E2000FDF702FC68461EF07FFA4F4968461EF017
:103E3000BBFA00216846FDF7F7FB68461EF074FAEE
:103E40002220FDF76FFD494A494B9DF887106846CF
:103E5000002914BF114619461EF0A6FA0021684633
:103E6000FDF7E2FB68461EF05FFA324968461EF035
:103E70009BFA00216846FDF7D7FB68461EF054FA0E
:103E8000119C002C00F0BC803A4968461EF08CFA68
:103E900000216846FDF7C8FB68461EF045FA2B492D
:103EA00068461EF081FA00216846FDF7BDFB6846B2
:103EB0001EF03AFA304968461EF076FA002168464C
:103EC000FDF7B2FB68461EF02FFA204968461EF047
:103ED0006BFA68460021FDF7A7FB68461EF024FA3E
:103EE000264968461EF060FA00216846FDF79CFBF3
:103EF00068461EF019FA2220FDF714FD9DED150A03
:103F00000420FDF7B3FC0B4968461EF04DFA002172
:103F10006846FDF789FB68461EF006FA2D9C002CCA
:103F200000F09B80164968461EF03EFA0021684664
:103F300028E000BF448B02003C8E0200548E020039
:103F40006C8E0200848E0200EC8E0200308902002A
:103F5000FC8E02000C8F0200248F02003C8F0200B6
:103F60004C8F02005C8F02006C8F0200248D0200D7
:103F7000288D02007C8F02008C8F0200BC8F020013
:103F8000E08F0200FDF750FB68461EF0CDF9604956
:103F900068461EF009FA68460021FDF745FB6846B1
:103FA0001EF0C2F95B4968461EF0FEF90021684622
:103FB000FDF73AFB68461EF0B7F9554968461EF012
:103FC000F3F900216846FDF72FFB68461EF0ACF9B7
:103FD000514968461EF0E8F900216846FDF724FBC8
:103FE00068461EF0A1F94A4968461EF0DDF9002135
:103FF0006846FDF719FB68461EF096F92EB070BDB5
:10400000464968461EF0D0F921466846FDF70CFB8C
:1040100068461EF089F93E4968461EF0C5F92146FA
:104020006846FDF701FB68461EF07EF93C4968468C
:104030001EF0BAF921466846FDF7F6FA68461EF00A
:1040400073F9334968461EF0AFF968462146FDF71B
:10405000EBFA68461EF068F942E7324968461EF0FE
:10406000A3F921466846FDF7DFFA68461EF05CF9C1
:10407000274968461EF098F968462146FDF7D4FAAC
:1040800068461EF051F98DE7274968461EF08CF905
:1040900000216846FDF7C8FA68461EF045F91C493C
:1040A00068461EF081F900216846FDF7BDFA6846B2
:1040B0001EF03AF91D4968461EF076F9002168465F
:1040C000FDF7B2FA68461EF02FF9114968461EF056
:1040D0006BF900216846FDF7A7FA68461EF024F93F
:1040E000134968461EF060F900216846FDF79CFA06
:1040F00068461EF019F9064968461EF055F9002178
:104100006846FDF791FA68461EF00EF9094919E66E
:1041100030890200F48F02000C9002009C8F020094
:10412000AC8F0200CC8F02009C8E0200AC8E02008D
:10413000BC8E0200D48E020070B5C84BAEB01D68B4
:1041400004AC2D1B2EAE28191AF0EEFD04F8010B5D
:10415000A642F8D1C249C34C68461EF025F9002199
:104160006846FDF761FA68461EF0DEF82220FDF78A
:10417000D9FBD4ED067A0020B8EE670AFDF776FB8E
:10418000B94968461EF010F900216846FDF74CFA5F
:1041900068461EF0C9F8B54968461EF005F90021C9
:1041A0006846FDF741FA68461EF0BEF82220FDF78A
:1041B000B9FBD4ED077A0020B8EE670AFDF756FB8D
:1041C000A94968461EF0F0F800216846FDF72CFA70
:1041D00068461EF0A9F8A64968461EF0E5F80021D9
:1041E0006846FDF721FA68461EF09EF82220FDF78A
:1041F00099FBD4ED1E7A0020B8EE670AFDF736FB76
:10420000994968461EF0D0F800216846FDF70CFA7F
:1042100068461EF089F8974968461EF0C5F80021E7
:104220006846FDF701FA68461EF07EF82220FDF789
:1042300079FBD4ED0B7A0020B8EE670AFDF716FB88
:10424000894968461EF0B0F800216846FDF7ECF990
:1042500068461EF069F8884968461EF0A5F80021F6
:104260006846FDF7E1F968461EF05EF82220FDF78A
:1042700059FBD4ED0C7A0020B8EE670AFDF7F6FA88
:10428000794968461EF090F800216846FDF7CCF9A0
:1042900068461EF049F8794968461EF085F8002105
:1042A0006846FDF7C1F968461EF03EF82220FDF78A
:1042B00039FBD4ED1F7A0020B8EE670AFDF7D6FA75
:1042C000694968461EF070F800216846FDF7ACF9B0
:1042D00068461EF029F86A4968461EF065F8002114
:1042E0006846FDF7A1F968461EF01EF82220FDF78A
:1042F00019FBD4ED137A0020B8EE670AFDF7B6FA81
:10430000594968461EF050F800216846FDF78CF9BF
:1043100068461EF009F85B4968461EF045F8002122
:104320006846FDF781F968461DF0FEFF2220FDF783
:10433000F9FAD4ED147A0020B8EE670AFDF796FA80
:10434000494968461EF030F800216846FDF76CF9CF
:1043500068461DF0E9FF4C4968461EF025F800212B
:104360006846FDF761F968461DF0DEFF2220FDF783
:10437000D9FAD4ED207A0020B8EE670AFDF776FA74
:10438000394968461EF010F800216846FDF74CF9DF
:1043900068461DF0C9FF0D213C481DF0A7F9D4F86F
:1043A0008C103B4800230A221DF040FE38481DF0C7
:1043B0002DFED4F88C40002C43D1364968461DF0C0
:1043C000F3FF68462146FDF72FF968461DF0ACFF64
:1043D000314968461DF0E8FF00216846FDF724F9E1
:1043E00068461DF0A1FF2D4968461DF0DDFF002144
:1043F0006846FDF719F968461DF096FF264968469C
:104400001DF0D2FF00216846FDF70EF968461DF049
:104410008BFF234968461DF0C7FF00216846FDF762
:1044200003F968461DF080FF1B4968461DF0BCFF7C
:1044300000216846FDF7F8F868461DF075FF2EB0BC
:1044400070BD184968461DF0AFFF68460021FDF7B2
:10445000EBF868461DF068FFBAE700BF7C14FF1F49
:1044600020900200EC15FF1F448B020034900200E4
:10447000489002005C90020070900200849002005C
:1044800098900200AC900200C0900200D49002000C
:104490002408FF1FF8900200308902000C910200EE
:1044A00028910200E490020070B59D4BAEB01D68EB
:1044B00004AC2D1B2EAE28191AF036FC04F8010BA3
:1044C000B442F8D1684697491DF06EFF0021684656
:1044D000FDF7AAF868461DF027FF2220FDF722FA13
:1044E000DDED197A0020B8EEE70AFDF7BFF968465E
:1044F0008D491DF059FF68460021FDF795F8684683
:104500001DF012FF684689491DF04EFF00216846E4
:10451000FDF78AF868461DF007FF2220FDF702FA32
:10452000DDED1A7A0020B8EE670AFDF79FF96846BC
:104530007D491DF039FF68460021FDF775F8684692
:104540001DF0F2FE68467A491DF02EFF00216846F4
:10455000FDF76AF868461DF0E7FE2220FDF7E2F954
:10456000DDED1B7A0020B8EEE70AFDF77FF968461B
:104570006D491DF019FF68460021FDF755F86846A2
:104580001DF0D2FE68466B491DF00EFF0021684603
:10459000FDF74AF868461DF0C7FE2220FDF7C2F974
:1045A000DDED1C7A0020B8EE670AFDF75FF968467A
:1045B0005D491DF0F9FE68460021FDF735F86846B3
:1045C0001DF0B2FE68465C491DF0EEFE0021684613
:1045D000FDF72AF868461DF0A7FE2220FDF7A2F994
:1045E000DDED1D7A0020B8EEE70AFDF73FF96846D9
:1045F0004D491DF0D9FE68460021FDF715F86846C3
:104600001DF092FE68464D491DF0CEFE0021684621
:10461000FDF70AF868461DF087FE2220FDF782F9B3
:10462000DDED1E7A0020B8EE670AFDF71FF9684637
:104630003D491DF0B9FE68460021FCF7F5FF6846CC
:104640001DF072FE68463E491DF0AEFE0021684630
:10465000FCF7EAFF68461DF067FE2220FDF762F9CD
:10466000DDED1F7A0020B8EEE70AFDF7FFF8684697
:104670002D491DF099FE68460021FCF7D5FF6846DC
:104680001DF052FE68462F491DF08EFE002168463F
:10469000FCF7CAFF68461DF047FE2220FDF742F9ED
:1046A000DDED207A0020B8EE670AFDF7DFF86846F6
:1046B0001D491DF079FE68460021FCF7B5FF6846EC
:1046C0001DF032FE684620491DF06EFE684600214E
:1046D000FCF7AAFF68461DF027FE68461B491DF03F
:1046E00063FE68460021FCF79FFF68461DF01CFE34
:1046F000684617491DF058FE68460021FCF794FFF4
:1047000068461DF011FE684610491DF04DFE6846D2
:104710000021FCF789FF68461DF006FE2EB070BD33
:104720007C14FF1F40910200448B02005491020050
:10473000689102007C91020090910200A491020015
:10474000B8910200CC910200E4910200308902008D
:104750000092020070B5DA4B1B68013B84B0092B54
:1047600000F2AC81DFE813F0580348045304C1049D
:10477000AA01E8042A064A070A00D001D149D24D0D
:1047800068461DF011FE00216846FCF74DFF6846A3
:104790001DF0CAFD2220FDF7C5F8D5ED0C7A0020EA
:1047A000B8EEE70AFDF762F8C84968461DF0FCFD5F
:1047B00000216846FCF738FF68461DF0B5FDC44986
:1047C00068461DF0F1FD00216846FCF72DFF6846A4
:1047D0001DF0AAFD2220FDF7A5F8D5ED147A0020E2
:1047E000B8EE670AFDF742F8B84968461DF0DCFDEF
:1047F00000216846FCF718FF68461DF095FDB54995
:1048000068461DF0D1FD00216846FCF70DFF6846A3
:104810001DF08AFD2220FDF785F8D5ED107A0020E5
:10482000B8EEE70AFDF722F8A84968461DF0BCFD7E
:1048300000216846FCF7F8FE68461DF075FDA649A4
:1048400068461DF0B1FD00216846FCF7EDFE6846A4
:104850001DF06AFD2220FDF765F8D5ED077A0020EE
:10486000B8EEE70AFDF702F8984968461DF09CFD8E
:1048700000216846FCF7D8FE68461DF055FD9749B3
:1048800068461DF091FD00216846FCF7CDFE6846A4
:104890001DF04AFD2220FDF745F895ED080A00209D
:1048A000FCF7E4FF894968461DF07EFD002168465B
:1048B000FCF7BAFE68461DF037FD894968461DF0D1
:1048C00073FD00216846FCF7AFFE68461DF02CFD25
:1048D0002220FDF727F895ED0B0A0020FCF7C6FF14
:1048E0007A4968461DF060FD68460021FCF79CFE91
:1048F00068461DF019FDAE6A6C46002E02F0BB80C2
:10490000012E23D1774968461DF04EFD00216846EF
:10491000FCF78AFE68461DF007FD2220FDF702F82D
:10492000714968461DF040FD00216846FCF77CFE99
:1049300068461DF0F9FC654968461DF035FD68467E
:104940000021FCF771FE68461DF0EEFC6B6A022B3D
:1049500002F08080032B23D1644920461DF024FD02
:1049600000212046FCF760FE20461DF0DDFC2220E1
:10497000FCF7D8FF5E4920461DF016FD00212046B9
:10498000FCF752FE20461DF0CFFC504920461DF09A
:104990000BFD20460021FCF747FE20461DF0C4FC1D
:1049A0002B68494D012B00F0B387C0F01C87022B08
:1049B00040F084804F4920461DF0F6FC002120463F
:1049C000FCF732FE20461DF0AFFC2220FCF7AAFFC8
:1049D000494920461DF0E8FC00212046FCF724FE52
:1049E00020461DF0A1FC394920461DF0DDFC0021C8
:1049F0002046FCF719FE20461DF096FC3F49204654
:104A00001DF0D2FC00212046FCF70EFE20461DF0D2
:104A10008BFC2220FCF786FFD5ED0F7A0020B8EE44
:104A2000E70AFCF723FF294920461DF0BDFC0021C1
:104A30002046FCF7F9FD20461DF076FC3049204663
:104A40001DF0B2FC00212046FCF7EEFD20461DF0D3
:104A50006BFC2220FCF766FFD5ED177A0020B8EE3C
:104A6000670AFCF703FF194920461DF09DFC002151
:104A70002046FCF7D9FD20461DF056FC2149204672
:104A80001DF092FC00212046FCF7CEFD20461DF0D3
:104A90004BFC2220FCF746FF95ED130A0020B8EEF0
:104AA000C00AFCF7E3FE094920461DF07DFC2046C4
:104AB0000021FCF7B9FD20461DF036FC04B070BDA6
:104AC0008007FF1F189202000814FF1F448B02008A
:104AD0002C92020040920200A4920200B8920200BE
:104AE0000493020034930200A89502001893020078
:104AF0006C930200549202007499020068920200C2
:104B00007C92020090920200B549B64C68461DF0B6
:104B10004BFC00216846FCF787FD68461DF004FC4D
:104B20002220FCF7FFFED4ED007A0020B8EEE70A61
:104B3000FCF79CFEAC4968461DF036FC0021684637
:104B4000FCF772FD68461DF0EFFBA84968461DF0B2
:104B50002BFC00216846FCF767FD68461DF0E4FB6E
:104B60002220FCF7DFFED4ED047A0020B8EE670ABD
:104B7000FCF77CFE9C4968461DF016FC0021684647
:104B8000FCF752FD68461DF0CFFB994968461DF0C1
:104B90000BFC00216846FCF747FD68461DF0C4FB8E
:104BA0002220FCF7BFFED4ED087A0020B8EEE70A19
:104BB000FCF75CFE8C4968461DF0F6FB0021684658
:104BC000FCF732FD68461DF0AFFB8A4968461DF0D0
:104BD000EBFB00216846FCF727FD68461DF0A4FBAF
:104BE0002220FCF79FFED4ED0C7A0020B8EEE70AF5
:104BF000FCF73CFE7C4968461DF0D6FB0021684668
:104C0000FCF712FD68461DF08FFB7B4968461DF0DE
:104C1000CBFB00216846FCF707FD68461DF084FBCE
:104C20002220FCF77FFED4ED0D7A0020B8EEE70AD3
:104C3000FCF71CFE6C4968461DF0B6FB0021684677
:104C4000FCF7F2FC68461DF06FFB6C4968461DF0EE
:104C5000ABFB00216846FCF7E7FC68461DF064FBEF
:104C60002220FCF75FFE94ED160A0020FCF7FEFD03
:104C70005D4968461DF098FB68460021FCF7D4FCAE
:104C800068461DF051FBA36B012B02F00283C2F0BA
:104C90006982022B7FF412AF594968461DF084FBEC
:104CA00000216846FCF7C0FC68461DF03DFB222051
:104CB000FCF738FE534968461DF076FB0021684634
:104CC000FCF7B2FC68461DF02FFB474968461DF013
:104CD0006BFB00216846FCF7A7FC68461DF024FB2F
:104CE000494968461DF060FB00216846FCF79CFCC2
:104CF00068461DF019FB2220FCF714FED4ED037A60
:104D00000020B8EE670AFCF7B1FD374968461DF090
:104D10004BFB00216846FCF787FC68461DF004FB4E
:104D20003A4968461DF040FB00216846FCF77CFCD0
:104D300068461DF0F9FA2220FCF7F4FDD4ED077A5D
:104D40000020B8EE670AFCF791FD274968461DF080
:104D50002BFB00216846FCF767FC68461DF0E4FA6F
:104D60002B4968461DF020FB00216846FCF75CFCDF
:104D700068461DF0D9FA2220FCF7D4FDD4ED0B7A59
:104D80000020B8EEE70AFCF771FD174968461DF0F0
:104D90000BFB00216846FCF747FC68461DF0C4FA8F
:104DA0001C4968461DF000FB00216846FCF73CFCEE
:104DB00068461DF0B9FA2220FCF7B4FD94ED150AFF
:104DC0000020FCF753FD084968461DF0EDFA00216C
:104DD0006846FCF729FC68461DF0A6FA04B070BDD1
:104DE000189202002013FF1F448B02002C92020035
:104DF00040920200A4920200B892020004930200C2
:104E00005492020074990200689202007C9202009F
:104E10009092020034930200BA49BB4C68461DF0E0
:104E2000C3FA00216846FCF7FFFB68461DF07CFAD8
:104E30002220FCF777FDD4ED017A0020B8EEE70AD6
:104E4000FCF714FDB14968461DF0AEFA0021684632
:104E5000FCF7EAFB68461DF067FAAD4968461DF0AD
:104E6000A3FA00216846FCF7DFFB68461DF05CFAF8
:104E70002220FCF757FDD4ED097A0020B8EEE70AAE
:104E8000FCF7F4FCA14968461DF08EFA0021684643
:104E9000FCF7CAFB68461DF047FA9E4968461DF0BC
:104EA00083FA00216846FCF7BFFB68461DF03CFA18
:104EB0002220FCF737FDD4ED057A0020B8EEE70A92
:104EC000FCF7D4FC914968461DF06EFA6846002153
:104ED000FCF7AAFB68461DF027FA256B012D01F0AF
:104EE0005086022D01F0C686002D7FF4E7AD8A4979
:104EF00068461DF059FA29466846FCF795FB684656
:104F00001DF012FA2220FCF70DFD844968461DF0C1
:104F10004BFA29466846FCF787FB68461DF004FA01
:104F20007A4968461DF040FA29466846FCF77CFB42
:104F300068461DF0F9F97A4968461DF035FA2946A8
:104F40006846FCF771FB68461DF0EEF92220FCF77D
:104F5000E9FCD4ED027A2846B8EEE70AFCF786FCB5
:104F60006A4968461DF020FA29466846FCF75CFB52
:104F700068461DF0D9F96B4968461DF015FA2946B7
:104F80006846FCF751FB68461DF0CEF92220FCF77D
:104F9000C9FCD4ED0A7A2846B8EEE70AFCF766FCAD
:104FA0005A4968461DF000FA29466846FCF73CFB62
:104FB00068461DF0B9F95C4968461DF0F5F92946C7
:104FC0006846FCF731FB68461DF0AEF92220FCF77D
:104FD000A9FC94ED060A2846B8EEC00AFCF746FC88
:104FE0004A4968461DF0E0F968462946FCF71CFB73
:104FF00068461DF099F961E54C4C236B032B3FF695
:105000005DADDFE813F00B07960621067C053D49F0
:10501000474D68461DF0C8F900216846FCF704FBBF
:1050200068461DF081F92220FCF77CFCD5ED017A61
:105030000020B8EEE70AFCF719FC344968461DF079
:10504000B3F900216846FCF7EFFA68461DF06CF9E9
:105050002F4968461DF0A8F900216846FCF7E4FADC
:1050600068461DF061F92220FCF75CFCD5ED037A5F
:105070000020B8EE670AFCF7F9FB244968461DF0EA
:1050800093F900216846FCF7CFFA68461DF04CF909
:10509000204968461DF088F900216846FCF7C4FAEB
:1050A00068461DF041F92220FCF73CFCD5ED027A60
:1050B0000020B8EEE70AFCF7D9FB144968461DF05A
:1050C00073F968460021FCF7AFFA68461DF02CF929
:1050D0002B68013B6C46042B3FF6F0ACDFE813F085
:1050E000CD071307BC07AB079A07124C2368052BA3
:1050F0003FF6E4ACDFE813F08E081E0B740ADD09FE
:105100004609F807189202002819FF1F448B020075
:105110002C9202004092020054920200AC980200CD
:10512000689202007C92020090920200C013FF1F5E
:105130007415FF1FAC15FF1F9449954D68461DF06F
:1051400033F900216846FCF76FFA68461DF0ECF869
:105150002220FCF7E7FBD5ED017A0020B8EEE70A44
:10516000FCF784FB8B4968461DF01EF90021684658
:10517000FCF75AFA68461DF0D7F8874968461DF0D3
:1051800013F900216846FCF74FFA68461DF0CCF889
:105190002220FCF7C7FBD5ED027A0020B8EE670AA3
:1051A000FCF764FB7B4968461DF0FEF80021684669
:1051B000FCF73AFA68461DF0B7F8784968461DF0E2
:1051C000F3F800216846FCF72FFA68461DF0ACF8AA
:1051D0002220FCF7A7FBD5ED097A0020B8EEE70AFC
:1051E000FCF744FB6B4968461DF0DEF86846002179
:1051F000FCF71AFA68461DF097F86B6B012B6C46AA
:1052000000F04C87C1F01584302B01F01284312B53
:1052100000F0448762495E4E20461DF0C5F800212B
:105220002046FCF701FA20461DF07EF82220FCF70C
:1052300079FB95ED0F0A0020FCF718FB5549204635
:105240001DF0B2F800212046FCF7EEF920461DF0D3
:105250006BF8544920461DF0A7F800212046FCF7C2
:10526000E3F920461DF060F82220FCF75BFB95ED8A
:105270000E0A0020FCF7FAFA464920461DF094F881
:1052800000212046FCF7D0F920461DF04DF82B6890
:10529000012B01F0E386C1F06B86022B7FF40EAC8C
:1052A000414920461DF080F800212046FCF7BCF95A
:1052B00020461DF039F82220FCF734FB3B492046FC
:1052C0001DF072F800212046FCF7AEF920461DF0D3
:1052D0002BF8304920461DF067F800212046FCF7E6
:1052E000A3F920461DF020F8314920461DF05CF856
:1052F00000212046FCF798F920461DF015F82220E1
:10530000FCF710FBD6ED077A0020B8EEE70AFCF7B1
:10531000ADFA204920461DF047F800212046FCF751
:1053200083F920461DF000F8224920461DF03CF884
:1053300000212046FCF778F920461CF0F5FF2220DA
:10534000FCF7F0FAD6ED087A0020B8EE670AFCF711
:105350008DFA104920461DF027F800212046FCF761
:1053600063F920461CF0E0FF134920461DF01CF8AD
:1053700000212046FCF758F920461CF0D5FF2220DA
:10538000FCF7D0FA96ED0C0AFFF788BB18920200E2
:105390001418FF1F448B02002C920200409202005E
:1053A000B892020004930200549202007499020021
:1053B000689202007C920200909202008449854D1E
:1053C00068461CF0F1FF00216846FCF72DF968469D
:1053D0001CF0AAFF2220FCF7A5FAD5ED007A0020E8
:1053E000B8EEE70AFCF742FA7B4968461CF0DCFF9E
:1053F00000216846FCF718F968461CF095FF7749CC
:1054000068461CF0D1FF00216846FCF70DF968469C
:105410001CF08AFF2220FCF785FAD5ED087A0020DF
:10542000B8EE670AFCF722FA6B4968461CF0BCFF2D
:1054300000216846FCF7F8F868461CF075FF6849DB
:1054400068461CF0B1FF00216846FCF7EDF868469D
:105450001CF06AFF2220FCF765FAD5ED047A0020E3
:10546000B8EEE70AFCF702FA5B4968461CF09CFFBD
:1054700000216846FCF7D8F868461CF055FF5949EA
:1054800068461CF091FF00216846FCF7CDF868469D
:105490001CF04AFF2220FCF745FAD5ED147A0020D3
:1054A000B8EE670AFCF7E2F94B4968461CF07CFF4E
:1054B00068460021FCF7B8F868461CF035FFEE6C32
:1054C0006C46002E01F03382012E00F09782AB6C07
:1054D000404D012B01F0D684C1F04584022B7FF4AE
:1054E000EDAA414920461CF05FFF00212046FCF751
:1054F0009BF820461CF018FF2220FCF713FA3B49CA
:1055000020461CF051FF00212046FCF78DF8204674
:105510001CF00AFF304920461CF046FF00212046BF
:10552000FCF782F820461CF0FFFE314920461CF0B3
:105530003BFF00212046FCF777F820461CF0F4FEE4
:105540002220FCF7EFF9D5ED037A0020B8EEE70A48
:10555000FCF78CF9204920461CF026FF002120464C
:10556000FCF762F820461CF0DFFE224920461CF0C2
:105570001BFF00212046FCF757F820461CF0D4FE04
:105580002220FCF7CFF9D5ED0B7A0020B8EE670AA0
:10559000FCF76CF9104920461CF006FF002120465C
:1055A000FCF742F820461CF0BFFE134920461CF0D1
:1055B000FBFE00212046FCF737F820461CF0B4FE25
:1055C0002220FCF7AFF995ED070AFFF767BA00BF95
:1055D000189202008014FF1F448B02002C920200DC
:1055E0004092020018930200549202007499020043
:1055F000689202007C92020090920200B549B64D7A
:1056000068461CF0D1FE00216846FCF70DF868469C
:105610001CF08AFE2220FCF785F9D5ED0C7A0020DB
:10562000B8EEE70AFCF722F9AC4968461CF0BCFE6C
:1056300000216846FBF7F8FF68461CF075FEA84994
:1056400068461CF0B1FE00216846FBF7EDFF684696
:105650001CF06AFE2220FCF765F9D5ED147A0020D3
:10566000B8EE670AFCF702F99C4968461CF09CFEFC
:1056700000216846FBF7D8FF68461CF055FE9949A3
:1056800068461CF091FE00216846FBF7CDFF684696
:105690001CF04AFE2220FCF745F9D5ED107A0020D7
:1056A000B8EEE70AFCF7E2F88C4968461CF07CFE8D
:1056B00000216846FBF7B8FF68461CF035FE8A49B2
:1056C00068461CF071FE00216846FBF7ADFF684696
:1056D0001CF02AFE2220FCF725F9D5ED047A0020E3
:1056E000B8EEE70AFCF7C2F87C4968461CF05CFE9D
:1056F00000216846FBF798FF68461CF015FE7B49C1
:1057000068461CF051FE00216846FBF78DFF684695
:105710001CF00AFE2220FCF705F995ED030A002093
:10572000FCF7A4F86D4968461CF03EFE002168466F
:10573000FBF77AFF68461CF0F7FD6D4968461CF0E0
:1057400033FE00216846FBF76FFF68461CF0ECFD56
:105750002220FCF7E7F895ED060A0020FCF786F812
:105760005E4968461CF020FE68460021FBF75CFF9E
:1057700068461CF0D9FD6E696C46002E01F0CA81A6
:10578000012E23D15B4968461CF00EFE00216846BD
:10579000FBF74AFF68461CF0C7FD2220FCF7C2F861
:1057A000554968461CF000FE00216846FBF73CFFA7
:1057B00068461CF0B9FD494968461CF0F5FD68468D
:1057C0000021FBF731FF68461CF0AEFDAB68023BE1
:1057D000052B3FF6E5A8DFE813F0440888087708B2
:1057E000660855089908454920461CF0DDFD002152
:1057F0002046FBF719FF20461CF096FD2220FCF7FF
:1058000091F83F4920461CF0CFFD00212046FBF7D0
:105810000BFF20461CF088FD304920461CF0C4FDDB
:1058200000212046FBF700FF20461CF07DFD354996
:1058300020461CF0B9FD00212046FBF7F5FE20466E
:105840001CF072FD2220FCF76DF8D5ED0D7A0020DA
:10585000B8EEE70AFCF70AF8204920461CF0A4FD40
:1058600000212046FBF7E0FE20461CF05DFD2649A6
:1058700020461CF099FD00212046FBF7D5FE20466E
:105880001CF052FD2220FCF74DF8D5ED157A0020D2
:10589000B8EE670AFBF7EAFF104920461CF084FDCA
:1058A00000212046FBF7C0FE20461CF03DFD1749B5
:1058B00020461CF079FD00212046FBF7B5FE20466E
:1058C0001CF032FD2220FCF72DF895ED110AFFF7B0
:1058D000E5B800BF189202000814FF1F448B0200B5
:1058E0002C92020040920200A4920200B8920200A0
:1058F0000493020034930200A8950200549202001F
:10590000AC980200689202007C9202009092020021
:10591000BE4920461CF048FD00212046FBF784FECE
:1059200020461CF001FD2220FBF7FCFFB849204671
:105930001CF03AFD00212046FBF776FE20461CF0C5
:10594000F3FCB44920461CF02FFD00212046FBF754
:105950006BFE20461CF0E8FCAF4920461CF024FDFD
:1059600000212046FBF760FE20461CF0DDFC2220D3
:10597000FBF7D8FFD5ED0E7A0020B8EEE70AFBF76B
:1059800075FFA44920461CF00FFD00212046FBF7BF
:105990004BFE20461CF0C8FCA04920461CF004FD2C
:1059A00000212046FBF740FE20461CF0BDFC2220D3
:1059B000FBF7B8FFD5ED167A0020B8EE670AFBF7C3
:1059C00055FF944920461CF0EFFC00212046FBF7D0
:1059D0002BFE20461CF0A8FC914920461CF0E4FC5C
:1059E00000212046FBF720FE20461CF09DFC2220D3
:1059F000FBF798FF95ED120AFFF750B88949684602
:105A00001CF0D2FC00216846FBF70EFE68461CF035
:105A10008BFC2220FBF786FF834968461CF0C4FC00
:105A200000216846FBF700FE68461CF07DFC7949C2
:105A300068461CF0B9FC00216846FBF7F5FD684696
:105A40001CF072FC794968461CF0AEFC00216846E7
:105A5000FBF7EAFD68461CF067FC2220FBF762FFBB
:105A6000D5ED0C7A0020B8EEE70AFBF7FFFE694996
:105A700068461CF099FC00216846FBF7D5FD684696
:105A80001CF052FC6A4968461CF08EFC00216846F6
:105A9000FBF7CAFD68461CF047FC2220FBF742FFDB
:105AA00095ED0F0A0020FBF7E1FE5A4968461CF00D
:105AB0007BFC00216846FBF7B7FD68461CF034FC10
:105AC0005C4968461CF070FC00216846FBF7ACFDA1
:105AD00068461CF029FC2220FBF724FF95ED0E0AF6
:105AE0000020FBF7C3FE4B4968461CF05DFC68468E
:105AF0000021FBF799FD68461CF016FCE7E44349DA
:105B000068461CF051FC00216846FBF78DFD684695
:105B10001CF00AFC2220FBF705FF474968461CF0F1
:105B200043FC00216846FBF77FFD68461CF0FCFB48
:105B3000384968461CF038FC00216846FBF774FDC4
:105B400068461CF0F1FB3D4968461CF02DFC002125
:105B50006846FBF769FD68461CF0E6FB2220FBF770
:105B6000E1FED4ED017A0020B8EEE70AFBF77EFEF5
:105B7000284968461CF018FC00216846FBF754FDD4
:105B800068461CF0D1FB2E4968461CF00DFC002134
:105B90006846FBF749FD68461CF0C6FB2220FBF770
:105BA000C1FED4ED097A0020B8EEE70AFBF75EFEED
:105BB000184968461CF0F8FB00216846FBF734FDE5
:105BC00068461CF0B1FB1F4968461CF0EDFB002144
:105BD0006846FBF729FD68461CF0A6FB2220FBF770
:105BE000A1FE94ED050AB8EEC00A0020FBF73EFEC8
:105BF000684608491CF0D8FB68460021FBF714FDF5
:105C000068461CF091FB04B070BD00BF54920200C6
:105C10007CC30200448B0200689202007C92020066
:105C200090920200A4920200A8950200B89202008D
:105C3000049302003493020040980200189202007C
:105C40002C92020040920200E54968461CF0ACFB31
:105C500000216846FBF7E8FC68461CF065FB222043
:105C6000FBF760FEDF4968461CF09EFB002168469A
:105C7000FBF7DAFC68461CF057FBDB4968461CF072
:105C800093FB00216846FBF7CFFC68461CF04CFBF9
:105C9000D64968461CF088FB00216846FBF7C4FC27
:105CA00068461CF041FB2220FBF73CFED4ED047A51
:105CB0000020B8EEE70AFBF7D9FDCB4968461CF097
:105CC00073FB00216846FBF7AFFC68461CF02CFB19
:105CD000C74968461CF068FB00216846FBF7A4FC36
:105CE00068461CF021FB2220FBF71CFED4ED007A55
:105CF0000020B8EEE70AFBF7B9FDBB4968461CF087
:105D000053FB00216846FBF78FFC68461CF00CFB38
:105D1000B84968461CF048FB00216846FBF784FC44
:105D200068461CF001FB2220FBF7FCFD94ED080AFD
:105D300059E7AB4968461CF037FB00216846FBF782
:105D400073FC68461CF0F0FA2220FBF7EBFDAA4931
:105D500068461CF029FB00216846FBF765FC684695
:105D60001CF0E2FAA04968461CF01EFB00216846C0
:105D7000FBF75AFC68461CF0D7FA9C4968461CF0B1
:105D800013FB00216846FBF74FFC68461CF0CCFA79
:105D90002220FBF7C7FDD4ED037A0020B8EEE70A16
:105DA000FBF764FD904968461CF0FEFA0021684646
:105DB000FBF73AFC68461CF0B7FA8D4968461CF0C0
:105DC000F3FA00216846FBF72FFC68461CF0ACFA9A
:105DD0002220FBF7A7FDD4ED0B7A0020B8EEE70AEE
:105DE000FBF744FD804968461CF0DEFA0021684656
:105DF000FBF71AFC68461CF097FA7E4968461CF0CF
:105E0000D3FA00216846FBF70FFC68461CF08CFAB9
:105E10002220FBF787FD94ED070AE4E67049684607
:105E20001CF0C2FA00216846FBF7FEFB68461CF036
:105E30007BFA2220FBF776FD704968461CF0B4FA25
:105E400000216846FBF7F0FB68461CF06DFA6649D6
:105E500068461CF0A9FA00216846FBF7E5FB684696
:105E60001CF062FA614968461CF09EFA00216846FF
:105E7000FBF7DAFB68461CF057FA2220FBF752FDCD
:105E8000D4ED027A0020B8EEE70AFBF7EFFC5649A2
:105E900068461CF089FA00216846FBF7C5FB684696
:105EA0001CF042FA524968461CF07EFA002168460E
:105EB000FBF7BAFB68461CF037FA2220FBF732FDED
:105EC000D4ED0A7A0020B8EEE70AFBF7CFFC46498A
:105ED00068461CF069FA00216846FBF7A5FB684696
:105EE0001CF022FA434968461CF05EFA002168461D
:105EF000FBF79AFB68461CF017FA2220FBF712FD0D
:105F000094ED060A6FE636493D4D68461CF04CFAA2
:105F100000216846FBF788FB68461CF005FA222042
:105F2000FBF700FD374920461CF03EFA00212046D1
:105F3000FBF77AFB20461CF0F7F92B4920461CF0B2
:105F400033FA00212046FBF76FFB20461CF0ECF9EA
:105F50002D4920461CF028FA00212046FBF764FB5F
:105F600020461CF0E1F92220FBF7DCFCD5E9040116
:105F70001EF030FC00EE100A0020FBF777FC1A49F7
:105F800020461CF011FA00212046FBF74DFB20466D
:105F90001CF0CAF96B68012B07D0C0F0E185302BEB
:105FA00000F0DE85312B7EF489AD184920461CF0C7
:105FB000FBF900212046FBF737FB20461CF0B4F923
:105FC0002220FBF7AFFC124920461CF0EDF92046D9
:105FD0000021FBF729FB20461CF0A6F9FEF763BD64
:105FE0005492020074990200448B020068920200ED
:105FF0007C920200909202007CC30200AC980200E6
:106000000817FF1F14970200A4920200B892020022
:10601000D4920200CA49CB4D68461CF0C5F9002154
:106020006846FBF701FB68461CF07EF92220FBF76F
:1060300079FCC54977E7C249C44D68461CF0B4F9FC
:1060400000216846FBF7F0FA68461CF06DF9222043
:10605000FBF768FCBE4966E7B949BE4D68461CF0CF
:10606000A3F900216846FBF7DFFA68461CF05CF9EB
:106070002220FBF757FCB84955E7B149B74D6846B0
:106080001CF092F900216846FBF7CEFA68461CF036
:106090004BF92220FBF746FCB14944E7B1492046C1
:1060A0001CF082F900212046FBF7BEFA20461CF0C6
:1060B0003BF92220FBF736FCAB4920461CF074F973
:1060C00000212046FBF7B0FA20461CF02DF9A74925
:1060D00020461CF069F920460021FBF7A5FA20466E
:1060E0001CF022F9FFF796B8954968461CF05CF958
:1060F00000216846FBF798FA68461CF015F9222043
:10610000FBF710FC9A4968461CF04EF900216846DE
:10611000FBF78AFA68461CF007F9944968461CF0B8
:1061200043F900216846FBF77FFA68461CF0FCF84B
:10613000904968461CF038F900216846FBF774FA6C
:1061400068461CF0F1F82220FBF7ECFBD4ED077A4F
:106150000020B8EEE70AFBF789FB844968461CF08B
:1061600023F900216846FBF75FFA68461CF0DCF86B
:10617000814968461CF018F900216846FBF754FA7B
:1061800068461CF0D1F82220FBF7CCFBD4ED087A4E
:106190000020B8EE670AFBF769FB744968461CF0FB
:1061A00003F900216846FBF73FFA68461CF0BCF88B
:1061B000724968461CF0F8F800216846FBF734FA8B
:1061C00068461CF0B1F82220FBF7ACFBD4ED097A4D
:1061D0000020B8EEE70AFBF749FB644968461CF06B
:1061E000E3F800216846FBF71FFA68461CF09CF8AC
:1061F0005C4968461CF0D8F800216846FBF714FAA1
:1062000068461CF091F82220FBF78CFB002094EDEF
:106210000F0AEBE44A4968461CF0C6F800216846BC
:10622000FBF702FA68461CF07FF82220FBF77AFBA6
:10623000534968461CF0B8F800216846FBF7F4F9AA
:1062400068461CF071F8494968461CF0ADF8002119
:106250006846FBF7E9F968461CF066F84549684668
:106260001CF0A2F800216846FBF7DEF968461CF036
:106270005BF82220FBF756FBD4ED017A0020B8EE44
:10628000E70AFBF7F3FA394968461CF08DF800215C
:106290006846FBF7C9F968461CF046F83649684677
:1062A0001CF082F800216846FBF7BEF968461CF036
:1062B0003BF82220FBF736FBD4ED027A0020B8EE43
:1062C000670AFBF7D3FA294968461CF06DF80021EC
:1062D0006846FBF7A9F968461CF026F82749684686
:1062E0001CF062F800216846FBF79EF968461CF036
:1062F0001BF82220FBF716FBD4ED037A0020B8EE42
:10630000E70AFBF7B3FA194968461CF04DF800217B
:106310006846FBF789F968461CF006F8114968469B
:106320001CF042F800216846FBF77EF968461BF036
:10633000FBFF2220FBF7F6FA002094ED0A0A55E451
:10634000549202005017FF1FEC9702003817FF1FEE
:10635000FC9102002017FF1F8C970200F016FF1F10
:10636000E4B90200A4920200FC920200448B0200F5
:10637000F0920200689202007C9202009092020069
:10638000DC920200E24968461CF00EF800216846E3
:10639000FBF74AF968461BF0C7FF2220FBF7C2FA59
:1063A000DC4968461CF000F800216846FBF73CF920
:1063B00068461BF0B9FFD84968461BF0F5FF00217D
:1063C0006846FBF731F968461BF0AEFFD3496846D3
:1063D0001BF0EAFF00216846FBF726F968461BF030
:1063E000A3FF2220FBF79EFAD4ED047A0020B8EE3A
:1063F000E70AFBF73BFAC84968461BF0D5FF0021C6
:106400006846FBF711F968461BF08EFFC4496846E1
:106410001BF0CAFF00216846FBF706F968461BF02F
:1064200083FF2220FBF77EFAD4ED057A0020B8EE38
:10643000670AFBF71BFAB84968461BF0B5FF002155
:106440006846FBF7F1F868461BF06EFFB5496846F1
:106450001BF0AAFF00216846FBF7E6F868461BF030
:1064600063FF2220FBF75EFAD4ED067A0020B8EE37
:10647000E70AFBF7FBF9A84968461BF095FF0021E6
:106480006846FBF7D1F868461BF04EFFA649684600
:106490001BF08AFF00216846FBF7C6F868461BF030
:1064A00043FF2220FBF73EFA002094ED0E0AFFF78F
:1064B0009DBB974968461BF077FF00216846FBF7B4
:1064C000B3F868461BF030FF2220FBF72BFA974900
:1064D00068461BF069FF00216846FBF7A5F868468F
:1064E0001BF022FF8C4968461BF05EFF00216846C6
:1064F000FBF79AF868461BF017FF884968461BF0BF
:1065000053FF00216846FBF78FF868461BF00CFF2D
:106510002220FBF707FAD4ED017A0020B8EEE70A53
:10652000FBF7A4F97C4968461BF03EFF0021684652
:10653000FBF77AF868461BF0F7FE794968461BF0CE
:1065400033FF00216846FBF76FF868461BF0ECFE4E
:106550002220FBF7E7F9D4ED027A0020B8EE670AB3
:10656000FBF784F96C4968461BF01EFF0021684662
:10657000FBF75AF868461BF0D7FE6A4968461BF0DD
:1065800013FF00216846FBF74FF868461BF0CCFE6E
:106590002220FBF7C7F9D4ED037A0020B8EEE70A12
:1065A000FBF764F95C4968461BF0FEFE0021684673
:1065B000FBF73AF868461BF0B7FE5B4968461BF0EC
:1065C000F3FE00216846FBF72FF868461BF0ACFE8F
:1065D0002220FBF7A7F9002094ED0D0AFFF706BB78
:1065E0004B4968461BF0E0FE00216846FBF71CF8AB
:1065F00068461BF099FE2220FBF794F94C49684647
:106600001BF0D2FE00216846FBF70EF868461BF02F
:106610008BFE414968461BF0C7FE00216846FBF728
:1066200003F868461BF080FE3C4968461BF0BCFE40
:1066300000216846FAF7F8FF68461BF075FE222035
:10664000FBF770F9D4ED077A0020B8EEE70AFBF704
:106650000DF9314968461BF0A7FE00216846FAF79C
:10666000E3FF68461BF060FE2D4968461BF09CFE68
:1066700000216846FAF7D8FF68461BF055FE222035
:10668000FBF750F9D4ED087A0020B8EE670AFBF763
:10669000EDF8214968461BF087FE00216846FAF7AD
:1066A000C3FF68461BF040FE1E4968461BF07CFE97
:1066B00000216846FAF7B8FF68461BF035FE222035
:1066C000FBF730F9D4ED097A0020B8EEE70AFBF7C2
:1066D000CDF8114968461BF067FE00216846FAF7BD
:1066E000A3FF68461BF020FE0F4968461BF05CFEC6
:1066F00000216846FAF798FF68461BF015FE222035
:10670000FBF710F9002094ED0C0AFFF76FBA00BFF9
:1067100054920200E8920200448B02006892020048
:106720007C92020090920200A4920200E092020089
:10673000EC920200E34968461BF036FE00216846F1
:10674000FAF772FF68461BF0EFFD2220FBF7EAF82C
:10675000DD4968461BF028FE00216846FAF764FF11
:1067600068461BF0E1FDD94968461BF01DFE00217B
:106770006846FAF759FF68461BF0D6FDD4496846CB
:106780001BF012FE00216846FAF74EFF68461BF028
:10679000CBFD2220FBF7C6F8D4ED047A0020B8EE3A
:1067A000E70AFBF763F8C94968461BF0FDFD0021C5
:1067B0006846FAF739FF68461BF0B6FDC5496846DA
:1067C0001BF0F2FD00216846FAF72EFF68461BF029
:1067D000ABFD2220FBF7A6F8D4ED057A0020B8EE39
:1067E000670AFBF743F8B94968461BF0DDFD002155
:1067F0006846FAF719FF68461BF096FDB6496846E9
:106800001BF0D2FD00216846FAF70EFF68461BF028
:106810008BFD2220FBF786F8D4ED067A0020B8EE37
:10682000E70AFBF723F8A94968461BF0BDFD0021E4
:106830006846FAF7F9FE68461BF076FDA7496846F8
:106840001BF0B2FD00216846FAF7EEFE68461BF029
:106850006BFD2220FBF766F8002094ED0B0AFFF792
:10686000C5B99F4920461BF09FFD00212046FAF73D
:10687000DBFE20461BF058FD2220FBF753F8994918
:10688000FEF779B8964920461BF08EFD0021204680
:10689000FAF7CAFE20461BF047FD2220FBF742F81C
:1068A0009149FEF768B88E4920461BF07DFD002116
:1068B0002046FAF7B9FE20461BF036FD2220FBF7F2
:1068C00031F88A49FEF757B8854920461BF06CFD20
:1068D00000212046FAF7A8FE20461BF025FD2220C5
:1068E000FBF720F88249FEF746B87D4920461BF0A9
:1068F0005BFD00212046FAF797FE20461BF014FDB1
:106900002220FBF70FF87B49FEF735B87449204683
:106910001BF04AFD00212046FAF786FE20461BF0B8
:1069200003FD2220FAF7FEFF7349FEF724B86B49F6
:1069300068461BF039FD31466846FAF775FE684631
:106940001BF0F2FC2220FAF7EDFF6C4968461BF0C1
:106950002BFD31466846FAF767FE68461BF0E4FCFB
:106960005A4968461BF020FD31466846FAF75CFE3E
:1069700068461BF0D9FC624968461BF015FD31469C
:106980006846FAF751FE68461BF0CEFC2220FAF763
:10699000C9FFD5ED0D7A3046B8EEE70AFAF766FF83
:1069A0004A4968461BF000FD31466846FAF73CFE4E
:1069B00068461BF0B9FC534968461BF0F5FC3146AC
:1069C0006846FAF731FE68461BF0AEFC2220FAF763
:1069D000A9FF95ED110A3046FAF748FF3B49684692
:1069E0001BF0E2FC31466846FAF71EFE68461BF0D3
:1069F0009BFC454968461BF0D7FC31466846FAF7D0
:106A000013FE68461BF090FC2220FAF78BFF95EDF1
:106A1000100A3046FAF72AFF2C4968461BF0C4FCDE
:106A200068463146FAF700FE68461BF07DFCFEF72B
:106A30004EBD2A4920461BF0B7FC00212046FAF73C
:106A4000F3FD20461BF070FC2220FAF76BFF2F4964
:106A5000FFF733BB224920461BF0A6FC002120464D
:106A6000FAF7E2FD20461BF05FFC2220FAF75AFFFE
:106A70002749FDF780BF244968461BF095FC314645
:106A80006846FAF7D1FD68461BF04EFC2220FAF763
:106A900049FF1A4968461BF087FC31466846FAF7F9
:106AA000C3FD68461BF040FC084968461BF07CFCAF
:106AB00068463146FAF7B8FD68461BF035FCFDF72D
:106AC00045BF00BF54920200E4920200448B0200D2
:106AD000689202007C92020090920200A49202004E
:106AE0001893020048930200589302005493020046
:106AF000509302004C9302005C9302002C9302001E
:106B0000B89202000493020034930200F49202004F
:106B100060930200CF4968461BF046FC3146684648
:106B2000FAF782FD68461BF0FFFB2220FAF7FAFE17
:106B3000C94968461BF038FC31466846FAF774FDCF
:106B400068461BF0F1FBC54968461BF02DFC684602
:106B50003146FAF769FD68461BF0E6FBFEF736BEE4
:106B6000BF4920461BF020FC00212046FAF75CFDBF
:106B700020461BF0D9FB2220FAF7D4FEB949FFF7D3
:106B800023BAB94968461BF00FFC00216846FAF7A2
:106B90004BFD68461BF0C8FB2220FAF7C3FEB34941
:106BA00068461BF001FC00216846FAF73DFD684687
:106BB0001BF0BAFBA94968461BF0F6FB00216846AA
:106BC000FAF732FD68461BF0AFFBA94968461BF097
:106BD000EBFB00216846FAF727FD68461BF0A4FB93
:106BE0002220FAF79FFED4ED037A0020B8EEE70AE0
:106BF000FAF73CFE994968461BF0D6FB002168462F
:106C0000FAF712FD68461BF08FFB9A4968461BF0A5
:106C1000CBFB00216846FAF707FD68461BF084FBB2
:106C20002220FAF77FFED4ED0B7A0020B8EEE70AB7
:106C3000FAF71CFE894968461BF0B6FB002168463E
:106C4000FAF7F2FC68461BF06FFB8B4968461BF0B5
:106C5000ABFB00216846FAF7E7FC68461BF064FBD3
:106C60002220FAF75FFE94ED070A0020B8EEC00A72
:106C7000FEF7A7B87C4968461BF096FB00216846E2
:106C8000FAF7D2FC68461BF04FFB2220FAF74AFEC7
:106C90007A4968461BF088FB00216846FAF7C4FC75
:106CA00068461BF041FB6D4968461BF07DFB0021E7
:106CB0006846FAF7B9FC68461BF036FB6C49684633
:106CC0001BF072FB00216846FAF7AEFC68461BF029
:106CD0002BFB2220FAF726FED4ED047A0020B8EE32
:106CE000E70AFAF7C3FD5D4968461BF05DFB00212A
:106CF0006846FAF799FC68461BF016FB5D49684642
:106D00001BF052FB00216846FAF78EFC68461BF028
:106D10000BFB2220FAF706FED4ED007A0020B8EE35
:106D2000E70AFAF7A3FD4D4968461BF03DFB002139
:106D30006846FAF779FC68461BF0F6FA4E49684651
:106D40001BF032FB00216846FAF76EFC68461BF028
:106D5000EBFA2220FAF7E6FD94ED080A0020B8EEDF
:106D6000C00AFEF72EB8404920461BF01DFB00214B
:106D70002046FAF759FC20461BF0D6FA2220FAF7F3
:106D8000D1FD3F4920461BF00FFB00212046FAF7BA
:106D90004BFC20461BF0C8FA304920461BF004FB90
:106DA00000212046FAF740FC20461BF0BDFA30498E
:106DB00020461BF0F9FA00212046FAF735FC204660
:106DC0001BF0B2FA2220FAF7ADFDD5ED017A0020D2
:106DD000B8EEE70AFAF74AFD204920461BF0E4FA2C
:106DE00000212046FAF720FC20461BF09DFA21499D
:106DF00020461BF0D9FA00212046FAF715FC204660
:106E00001BF092FA2220FAF78DFDD5ED097A0020C9
:106E1000B8EE670AFAF72AFD104920461BF0C4FABB
:106E200000212046FAF700FC20461BF07DFA1249AB
:106E300020461BF0B9FA00212046FAF7F5FB204660
:106E40001BF072FA2220FAF76DFD95ED050AFDF7A9
:106E500025BE00BF349302002C930200448B020035
:106E6000B8920200CC920200549202007CC302004D
:106E7000689202007C9202009092020074990200D3
:106E8000AC980200B04920461BF08EFA0021204643
:106E9000FAF7CAFB20461BF047FA2220FAF742FD18
:106EA000AA4920461BF080FA00212046FAF7BCFBD5
:106EB00020461BF039FAA64920461BF075FA00213E
:106EC0002046FAF7B1FB20461BF02EFAA1492046D6
:106ED0001BF06AFA00212046FAF7A6FB20461BF0B9
:106EE00023FA2220FAF71EFDD5ED027A0020B8EE33
:106EF000E70AFAF7BBFC964920461BF055FA002139
:106F00002046FAF791FB20461BF00EFA92492046E4
:106F10001BF04AFA00212046FAF786FB20461BF0B8
:106F200003FA2220FAF7FEFCD5ED0A7A0020B8EE2B
:106F3000670AFAF79BFC864920461BF035FA0021C8
:106F40002046FAF771FB20461BF0EEF983492046F4
:106F50001BF02AFA00212046FAF766FB20461BF0B8
:106F6000E3F92220FAF7DEFC95ED060AFDF796BD5F
:106F7000754920461BF018FA00212046FAF754FB09
:106F800020461BF0D1F92220FAF7CCFC74492046A8
:106F90001BF00AFA00212046FAF746FB20461BF0B8
:106FA000C3F96B4920461BF0FFF900212046FAF790
:106FB0003BFB20461BF0B8F9664920461BF0F4F96C
:106FC00000212046FAF730FB20461BF0ADF92220C5
:106FD000FAF7A8FCD6ED037A0020B8EEE70AFAF734
:106FE00045FC5B4920461BF0DFF900212046FAF7FB
:106FF0001BFB20461BF098F9574920461BF0D4F99B
:1070000000212046FAF710FB20461BF08DF92220C4
:10701000FAF788FCD6ED047A0020B8EE670AFAF792
:1070200025FC4B4920461BF0BFF900212046FAF70A
:10703000FBFA20461BF078F9484920461BF0B4F9CA
:1070400000212046FAF7F0FA20461BF06DF92220C5
:10705000FAF768FC96ED0A0AFDF720BD3A4920468A
:107060001BF0A2F900212046FAF7DEFA20461BF0B9
:107070005BF92220FAF756FC344920461BF094F9BC
:1070800000212046FAF7D0FA20461BF04DF930498E
:1070900020461BF089F900212046FAF7C5FA204660
:1070A0001BF042F92B4920461BF07EF900212046B7
:1070B000FAF7BAFA20461BF037F92220FAF732FC29
:1070C000D6ED057A0020B8EEE70AFAF7CFFB2049A3
:1070D00020461BF069F900212046FAF7A5FA204660
:1070E0001BF022F91C4920461BF05EF900212046C6
:1070F000FAF79AFA20461BF017F92220FAF712FC49
:10710000D6ED067A0020B8EE670AFAF7AFFB104911
:1071100020461BF049F900212046FAF785FA20465F
:107120001BF002F90D4920461BF03EF900212046D4
:10713000FAF77AFA20461BF0F7F82220FAF7F2FB6A
:1071400096ED0B0AFDF7AABC549202007CC3020024
:10715000448B0200689202007C920200909202002E
:10716000AC980200964968461BF01EF9002168465B
:10717000FAF75AFA68461BF0D7F82220FAF7D2FB42
:10718000904968461BF010F900216846FAF74CFA5E
:1071900068461BF0C9F88C4968461BF005F90021C8
:1071A0006846FAF741FA68461BF0BEF88749684618
:1071B0001BF0FAF800216846FAF736FA68461BF029
:1071C000B3F82220FAF7AEFBD4ED017A0020B8EE36
:1071D000E70AFAF74BFB7C4968461BF0E5F800210B
:1071E0006846FAF721FA68461BF09EF87849684627
:1071F0001BF0DAF800216846FAF716FA68461BF029
:1072000093F82220FAF78EFBD4ED057A0020B8EE31
:10721000670AFAF72BFB6C4968461BF0C5F800219A
:107220006846FAF701FA68461BF07EF86949684635
:107230001BF0BAF800216846FAF7F6F968461BF029
:1072400073F82220FAF76EFBD4ED097A0020B8EE2D
:10725000E70AFAF70BFB5C4968461BF0A5F800212A
:107260006846FAF7E1F968461BF05EF85A49684645
:107270001BF09AF800216846FAF7D6F968461BF029
:1072800053F82220FAF74EFB002094ED130AFDF785
:1072900098BD4B4968461BF087F800216846FAF70D
:1072A000C3F968461BF040F82220FAF73BFB4B4934
:1072B00068461BF079F800216846FAF7B5F9684688
:1072C0001BF032F8404968461BF06EF80021684612
:1072D000FAF7AAF968461BF027F83C4968461BF004
:1072E00063F800216846FAF79FF968461BF01CF81E
:1072F0002220FAF717FBD4ED027A0020B8EE670AD5
:10730000FAF7B4FA304968461BF04EF80021684697
:10731000FAF78AF968461BF007F82D4968461BF012
:1073200043F800216846FAF77FF968461AF0FCFF37
:107330002220FAF7F7FAD4ED067A0020B8EE670AB1
:10734000FAF794FA204968461BF02EF800216846A7
:10735000FAF76AF968461AF0E7FF1E4968461BF01B
:1073600023F800216846FAF75FF968461AF0DCFF57
:107370002220FAF7D7FAD4ED0A7A0020B8EEE70A0D
:10738000FAF774FA104968461BF00EF800216846B7
:10739000FAF74AF968461AF0C7FF0F4968461BF02A
:1073A00003F800216846FAF73FF968461AF0BCFF77
:1073B0002220FAF7B7FA002094ED140AFDF701BD78
:1073C00054920200AC980200448B020068920200C2
:1073D0007C92020090920200349302007CC302006F
:1073E0002DE9F043B34DB44CD5F800E02468BEF16C
:1073F000010F2DED028B1F4604BFB04B1C68ADB0D2
:1074000006460D46904608A800230122214617F0A3
:1074100099F90FA814F024FF002840F0FF8018A865
:107420009DF83A30A64908AA14F0CEFF1A9A9DF8A2
:107430006C309DF8641011928DF848308DF8401032
:107440001BAA0DF149030DF1560012F8011F03F8B4
:10745000011B8342F9D11F9B169318A814F0D2FE8A
:107460000FA814F0FDFE8146002836D10123092122
:1074700094488DF83B301AF039F920461EF060FD33
:10748000014620461AF032F90F218F489FED8F8A6E
:107490001AF02CF98E481AF0B9FD8E4918A81AF086
:1074A00083FF494618A8FAF7BFF818A81AF03CFF5E
:1074B000894918A81AF078FF18A84946FAF7B4F8CD
:1074C00018A81AF031FF08A817F05AF9B0EE480AC8
:1074D0002DB0BDEC028BBDE8F0830024502218A92A
:1074E00008A88DF83B4017F0A9F9002800F0848027
:1074F000502300932A4618AB314608A817F00EFB1C
:10750000002800F08F8018A81EF01AFD014618A868
:107510001AF0ECF86E481AF079FD704904A81AF0D8
:1075200043FF04A82146FAF77FF804A81AF0FCFEEE
:10753000002F00F0AB802220FAF7F4F918A904A874
:107540001AF032FF214604A8FAF76EF804A81AF0E0
:10755000EBFE2220FAF7E6F9614904A81AF024FFAD
:10756000002104A8FAF760F804A81AF0DDFE07EE7F
:10757000908A0020B8EEE70AFAF778F9564904A88D
:107580001AF012FF002104A8FAF74EF804A81AF026
:10759000CBFE30461EF0D4FC014630461AF0A6F869
:1075A0004B481AF033FD28461EF0CAFC0146284617
:1075B0001AF09CF846481AF029FD052147481AF0B0
:1075C00095F8002F6ED022201AF014F918A81EF09A
:1075D000B7FC014618A81AF089F822201AF00AF917
:1075E00001213F481AF082F8414639481AF05EFD01
:1075F00037481AF00BFD35E009213A489FED338AF0
:107600001AF074F808A81EF09BFC014608A81AF0AE
:107610006DF80C2134481AF069F854E70FA814F0FB
:1076200011FEFCE6102131481AF060F828481AF0E3
:10763000EDFC04212E481AF059F830461EF080FC6B
:10764000014630461AF052F803212A481AF04EF843
:1076500028461EF075FC014628461AF047F81C48DB
:107660001AF0D4FC244A1368049304991368039312
:10767000039B5B1A632BF9D918A81DF0D3FB51ECBF
:10768000100B1DF0A7F808EE100A1CE718A904A8B3
:107690001AF08AFE04A83946F9F7C6FF04A81AF0C2
:1076A00043FE59E718A81EF04BFC014618A81AF033
:1076B0001DF895E7B017FF1F6407FF1F7407FF1F32
:1076C0006019FF1F74930200809302000000000005
:1076D0002408FF1F9093020030890200B893020033
:1076E000C09302009C930200A89302000889020044
:1076F000C4930200CC930200141CFF1F38B5854DC3
:107700008549864C284600234FF43C72FFF768FEFB
:10771000BDEEC00A28460023C822814984ED000A34
:10772000FFF75EFEBDEEC00A284600234FF4497203
:107730007C4984ED010AFFF753FEBDEEC00A2846DE
:1077400000234FF44A72784984ED0C0AFFF748FE93
:10775000BDEEC00A284600233C22744984ED140A79
:10776000FFF73EFEBDEEC00A284600234FF45872D4
:107770006F4984ED100AFFF733FEBDEEC00A2846BC
:1077800000234FF457726B4984ED0D0AFFF728FE72
:10779000BDEEC00A284600234022674984ED150A41
:1077A000FFF71EFEBDEEC00A284600234FF45572B7
:1077B000624984ED110AFFF713FEBDEEC00A2846A8
:1077C00000234FF456725E4984ED0E0AFFF708FE5F
:1077D000BDEEC00A2846002344225A4984ED160A09
:1077E000FFF7FEFDBDEEC00A284600234FF44C72A1
:1077F000554984ED120AFFF7F3FDBDEEC00A284695
:1078000000234FF44B72514984ED0F0AFFF7E8FD56
:10781000BDEEC00A284600231C224D4984ED170AFC
:10782000FFF7DEFDBDEEC00A284600234FF4D872F4
:10783000484984ED130AFFF7D3FDBDEEC00A284680
:1078400000234FF42E72444984ED050AFFF7C8FD6A
:10785000BDEEC00A284601234FF4BA723F4984EDB9
:10786000020AFFF7BDFDBDEEC00A2846B8EEC00A09
:1078700000234FF4F8723A4984ED030AFFF7B0FD94
:10788000BDEEC00A284601234FF41B72354984ED32
:10789000040AFFF7A5FDBDEEC00A2846B8EEC00AEF
:1078A00000234FF4DA72304984ED060AFFF798FDA1
:1078B000BDEEC00A284601234FF41F722B4984ED08
:1078C0000A0AFFF78DFDBDEEC00A2846B8EEC00AD1
:1078D00000234FF43D72264984ED080AFFF780FD2E
:1078E000BDEEC00A284601234FF49672214984ED6B
:1078F000070AFFF775FDBDEEC00A1F4BB8EEC00AC0
:107900002046196884ED0B0A6022BDE8384017F064
:1079100053BA00BFD8930200D09302000814FF1F8F
:10792000DC930200EC930200009402001094020029
:1079300028940200349402003C9402005094020007
:107940005C94020064940200789402008494020023
:107950008C940200A0940200B8940200C494020027
:10796000DC940200F49402000C95020020950200C1
:1079700034950200489502004C07FF1F38B54A4D68
:107980004A494B4C284600234FF4EC72FFF728FD80
:10799000BDEEC00A284600234FF46172454984EDCC
:1079A0000C0AFFF71DFDBDEEC00A284600234FF468
:1079B0006B72414984ED010AFFF712FDBDEEC00A6A
:1079C0002846002314223D4984ED090AFFF708FDEB
:1079D000BDEEC00A284600234FF45372384984EDA7
:1079E000050AFFF7FDFCBDEEC00A284600234FF450
:1079F0005472344984ED020AFFF7F2FCBDEEC00A6E
:107A0000284600233822304984ED0A0AFFF7E8FCB3
:107A1000BDEEC00A284600234FF476722B4984ED50
:107A2000060AFFF7DDFCBDEEC00A284600234FF42E
:107A30005172274984ED030AFFF7D2FCBDEEC00A5C
:107A4000284600235422234984ED0B0AFFF7C8FC83
:107A5000BDEEC00A284600234FF452721E4984ED41
:107A6000070AFFF7BDFCBDEEC00A284600234FF40D
:107A700046721A4984ED040AFFF7B2FCBDEEC00A53
:107A8000284600236C22164984ED000AFFF7A8FC63
:107A9000144BBDEEC00A2046196884ED080A342252
:107AA000BDE8384017F088B95C950200D093020019
:107AB000C013FF1FEC930200009402001094020018
:107AC00028940200349402003C9402005094020076
:107AD0005C94020064940200789402008494020092
:107AE0008C9402008407FF1F38B54A4D4A494B4C1D
:107AF000284600234FF40E72FFF772FCBDEEC00A59
:107B0000284600234FF45A72454984ED0C0AFFF7CA
:107B100067FCBDEEC00A284600234FF46472414959
:107B200084ED010AFFF75CFC0023BDEEC00A284685
:107B30001A463D4984ED090AFFF752FCBDEEC00A22
:107B4000284600234FF46E72384984ED050AFFF78A
:107B500047FCBDEEC00A284600234FF47372344937
:107B600084ED020AFFF73CFCBDEEC00A2846002364
:107B70001022304984ED0A0AFFF732FCBDEEC00A3C
:107B8000284600234FF478722B4984ED060AFFF74C
:107B900027FCBDEEC00A284600234FF47B7227491C
:107BA00084ED030AFFF71CFCBDEEC00A2846002343
:107BB0000822234984ED0B0AFFF712FCBDEEC00A30
:107BC000284600234FF47E721E4984ED070AFFF712
:107BD00007FCBDEEC00A284600234FF47F721A4905
:107BE00084ED040AFFF7FCFBBDEEC00A2846002323
:107BF0000C22164984ED000AFFF7F2FB144BBDEE90
:107C0000C00A2046196884ED080A3422BDE83840CD
:107C100017F0D2B860950200D09302002819FF1F18
:107C2000EC930200009402001094020028940200D9
:107C3000349402003C940200509402005C940200D0
:107C40006494020078940200849402008C940200F0
:107C50009007FF1F38B5594D59495A4C2846002303
:107C60004FF41872FFF7BCFBBDEEC00A2846002394
:107C70004FF4D272544984ED000AFFF7B1FBBDEE18
:107C8000C00A284601234FF41972504984ED0D0AA9
:107C9000FFF7A6FB284601234FF41D724C4984EDE3
:107CA0000F0AFFF79DFB284600234FF45D724949F8
:107CB00084ED0E0AFFF794FBBDEEC00A28460023B0
:107CC0004FF46772444984ED010AFFF789FBBDEE6A
:107CD000C00A284600234C22404984ED020AFFF7DF
:107CE0007FFBBDEEC00A284600234FF46F723C496B
:107CF00084ED090AFFF774FBBDEEC00A2846002395
:107D00004FF47472374984ED030AFFF769FBBDEE47
:107D1000C00A284600234822334984ED040AFFF7AD
:107D20005FFBBDEEC00A284600234FF479722F494D
:107D300084ED0A0AFFF754FBBDEEC00A2846002373
:107D40004FF47C722A4984ED050AFFF749FBBDEE2A
:107D5000C00A284600231822264984ED060AFFF7A8
:107D60003FFBBDEEC00A284600234FF4687222494B
:107D700084ED0B0AFFF734FBBDEEC00A2846002352
:107D80004FF463721D4984ED070AFFF729FBBDEE2E
:107D9000C00A284600235022194984ED080AFFF73B
:107DA0001FFB184BBDEEC00A2046196884ED0C0A73
:107DB0004022BDE8384016F0FFBF00BF68950200C2
:107DC000D09302001418FF1F709502007C950200EA
:107DD00088950200EC9302000094020010940200C7
:107DE00028940200349402003C9402005094020053
:107DF0005C9402006494020078940200849402006F
:107E00008C9402003C07FF1F38B5724D7249734CC9
:107E1000284600234FF4E872FFF7E2FABDEEC00AED
:107E2000284600234FF40D726D4984ED120AFFF7C6
:107E3000D7FABDEEC00A284600234FF40C726949F8
:107E400084ED140AFFF7CCFABDEEC00A28460023E1
:107E50004FF46072644984ED130AFFF7C1FABDEE76
:107E6000C00A284600234FF46A72604984ED000A74
:107E7000FFF7B6FABDEEC00A2846002304225C498B
:107E800084ED080AFFF7ACFABDEEC00A28460023CD
:107E90004FF47172574984ED040AFFF7A1FABDEE61
:107EA000C00A284600234FF46972534984ED010A41
:107EB000FFF796FABDEEC00A2846002358224F4924
:107EC00084ED090AFFF78CFABDEEC00A28460023AC
:107ED0004FF470724A4984ED050AFFF781FABDEE4E
:107EE000C00A284600234FF47572464984ED020A01
:107EF000FFF776FABDEEC00A284600236022424909
:107F000084ED0A0AFFF76CFABDEEC00A284600238A
:107F10004FF447723D4984ED060AFFF761FABDEE62
:107F2000C00A284600234FF44872394984ED030AF9
:107F3000FFF756FABDEEC00A284600233022354925
:107F400084ED0B0AFFF74CFABDEEC00A2846002369
:107F50004FF40B72304984ED070AFFF741FABDEE8A
:107F6000C00A284601234FF49A722C4984ED0D0A69
:107F7000FFF736FA28460123E822294984ED110A41
:107F8000FFF72EFA284600234FF43972254984ED75
:107F9000100AFFF725FABDEEC00A284601234FF468
:107FA0003A72214984ED0C0AFFF71AFA2846012398
:107FB0004FF4A2721D4984ED0F0AFFF711FA1C4B12
:107FC00084ED0E0A204619685422BDE8384016F0A8
:107FD000F3BE00BF94950200D09302008014FF1FEF
:107FE00098950200A0950200EC9302000094020014
:107FF0001094020028940200349402003C94020081
:10800000509402005C940200649402007894020090
:10801000849402008C940200B0950200C095020086
:10802000D8950200F0950200FC950200149602001B
:108030003807FF1F38B5844D8449854C28460023F6
:10804000A422FFF7CDF9BDEEC00A28460023D022B6
:10805000804984ED0E0AFFF7C3F9BDEEC00A284639
:108060000023F0227C4984ED0C0AFFF7B9F9BDEE3C
:10807000C00A284600234FF4E272784984ED0F0AC3
:10808000FFF7AEF9BDEEC00A284601234FF42E7269
:10809000734984ED0D0AFFF7A3F9284600234FF436
:1080A0004F72704984ED160AFFF79AF9BDEEC00AC7
:1080B000284600234FF450726B4984ED000AFFF705
:1080C0008FF9BDEEC00A284601236422674984ED7A
:1080D000040AFFF785F9BDEEC00A284600234FF4D5
:1080E0005C72634984ED080AFFF77AF9BDEEC00AB5
:1080F000284600234FF46D725E4984ED010AFFF7B4
:108100006FF9BDEEC00A2846002334225A4984ED97
:10811000050AFFF765F9BDEEC00A284601234FF4B2
:108120008A72564984ED090AFFF75AF9BDEEC00A72
:108130002846B8EEC00A01234FF49272504984EDEC
:10814000130AFFF74DF9BDEEC00A2846B8EEC00A83
:1081500000234FF45B724B4984ED100AFFF740F99E
:10816000BDEEC00A284600234FF45972464984EDFB
:10817000020AFFF735F9BDEEC00A284600232C227B
:10818000424984ED060AFFF72BF9BDEEC00A2846E6
:1081900001234FF48E723E4984ED0A0AFFF720F95D
:1081A000BDEEC00A2846B8EEC00A0123E0223949D4
:1081B00084ED140AFFF714F9BDEEC00A2846B8EEA4
:1081C000C00A00234FF44E72334984ED110AFFF7C1
:1081D00007F9BDEEC00A284600234FF44D722F491F
:1081E00084ED030AFFF7FCF8BDEEC00A2846002321
:1081F00020222B4984ED070AFFF7F2F8BDEEC00AF2
:10820000284601234FF40272264984ED0B0AFFF73A
:10821000E7F8BDEEC00A2846B8EEC00A01234FF4C5
:108220000472214984ED150AFFF7DAF8BDEEC00AA1
:108230001E4BB8EEC00A2046196884ED120A5C2273
:10824000BDE8384016F0B8BD28960200D093020071
:108250002013FF1F30960200A095020038960200FE
:1082600040960200EC930200009402001094020079
:1082700028940200349402003C94020054960200B8
:1082800068960200509402005C940200649402001C
:108290007C9602009096020078940200849402007A
:1082A0008C940200A4960200B89602003407FF1FC7
:1082B0002DE9F84FA54CA649A64FDFF80883DFF853
:1082C00008B3A54DA54EDFF804A3DFF804932DED08
:1082D000028B204600234FF4B872FFF781F8BDEE01
:1082E000C00A204600234FF462729D4987ED000AC0
:1082F000FFF776F8BDEEC00A204600234FF46C72FB
:10830000984987ED010AFFF76BF8BDEEC00A2046D9
:1083100000236822944987ED030AFFF761F8BDEE58
:10832000C00A204641460023C02287ED020AFFF71B
:1083300057F8BDEEC00A204600234FF40F728B4958
:108340008BED000AFFF74CF8BDEEC00A01234FF495
:10835000B072204686498BED010AFFF741F810EE16
:10836000100A1BF0EBFE41EC100BCBE90401F8F70F
:108370006BFE414620460023A022FFF731F8BDEEF8
:10838000C00A204600234FF431727A4985ED000A75
:10839000FFF726F8BDEEC00A01234FF4B472204661
:1083A000754985ED010AFFF71BF810EE100A1BF066
:1083B000C5FE41EC180B41EC100BC5E90401F8F7C0
:1083C00043FE0C216D48DFF80C8219F08FF9B0EEF6
:1083D000480AF0EE680A0221304619F071FE304674
:1083E00019F014FE1B21664819F080F9A96830467F
:1083F00019F05CFE304619F009FE1B21614819F0A6
:1084000075F995ED040B0221304619F059FE3046FE
:1084100019F0FCFD2046002398225B49FEF7E0FF9F
:10842000BDEEC00A204600234FF4147257498AED6E
:10843000000AFEF7D5FFBDEEC00A01234FF411720A
:10844000204653498AED010AFEF7CAFF10EE100AD2
:108450001BF074FE41EC100BCAE90401F8F7F4FDBF
:10846000204600234FF4D6724A49FEF7B9FFBDEE0D
:10847000C00A204600234FF41372474989ED000AD1
:10848000FEF7AEFFBDEEC00A01234FF4287220466E
:10849000424989ED010AFEF7A3FF10EE100A1BF016
:1084A0004DFE41EC100BC9E90401F8F7CDFD204663
:1084B00000234FF4DC723A49FEF792FFBDEEC00A8A
:1084C000204600234FF40672364988ED000AFEF775
:1084D00087FFBDEEC00A01234FF42A7220463249BD
:1084E00088ED010AFEF77CFF10EE100A1BF026FE55
:1084F00041EC100BC8E90401F8F7A6FD2B4B3846F8
:108500001968102216F058FC294B58461968182291
:1085100016F052FC274B28461968182216F04CFC1E
:10852000254B50461968182216F046FC234B484646
:108530001968182216F040FCBDEC028B204B404617
:1085400019681822BDE8F84F16F036BCD496020020
:10855000CC9602007415FF1F0817FF1F2408FF1F89
:10856000EC9302000094020010940200F0960200C6
:108570000097020008970200189702002097020057
:10858000309702004C970200689702008097020023
:108590009097020098970200B0970200C0970200DF
:1085A000C8970200E0970200F09702008C07FF1FB7
:1085B0005007FF1F5407FF1F6807FF1F7807FF1FA3
:1085C0005C07FF1FD8960200F016FF1F2017FF1F41
:1085D0003817FF1F5017FF1F38B5B42200239A49E0
:1085E0009A489B4C9A4DFEF7FBFE0023C8229949FE
:1085F0009648FEF7F5FE0023D42297499348FEF7EC
:10860000EFFEBDEEC00A0023F42294498F4884EDAA
:10861000000AFEF7E5FEBDEEC00A01234FF48672A4
:108620008F498A4884ED010AFEF7DAFE0023F8221A
:108630008C49864884ED020AFEF7D2FEF7EE007AF6
:10864000B4EEE70AF1EE10FAACBF0123002384F880
:108650007430D822012384497C48FEF7C1FEBCEE69
:10866000C00A0123DC228149784884ED210AFEF703
:10867000B7FEBCEEC00A00234FF4EA727C4973488F
:1086800084ED220AFEF7ACFEBDEEC00A00234FF4D3
:10869000E67278496D4884ED040AFEF7A1FEBDEE4E
:1086A000C00A01234FF400727349684884ED030A3D
:1086B000FEF796FE0023FC227049644884ED050A0B
:1086C000FEF78EFEF7EE007AB4EEE70AF1EE10FA4E
:1086D000ACBF0123002385F875304FF4F2720023FC
:1086E00067495A485A4DFEF77BFEBDEEC00A00238B
:1086F0004FF4F0726349554884ED090AFEF770FEA5
:10870000BDEEC00A01234FF4F4725F494F4884ED77
:10871000080AFEF765FE00234FF480725B494B4860
:1087200084ED0A0AFEF75CFEF7EE007AB4EEE70A83
:10873000F1EE10FAACBF0123002385F87630CC228D
:10874000002353494148424DFEF74AFEBDEEC00AA0
:108750000023C4224F493D4884ED260AFEF740FE1F
:10876000BDEEC00A0123D8224B49384884ED250AC2
:10877000FEF736FE00234FF465724849334884ED16
:10878000270AFEF72DFEF7EE007AB4EEE70AF1EEC7
:1087900010FAACBF0123002385F8A0304FF4087213
:1087A00000233F4929482A4DFEF71AFEBDEEC00AB4
:1087B00000234FF407723B49244884ED0F0AFEF76B
:1087C0000FFEBDEEC00A01234FF4097236491F485F
:1087D00084ED0E0AFEF704FE00234FF48272334943
:1087E0001A4884ED100AFEF7FBFDF7EE007AB4EEAE
:1087F000E70AF1EE10FAACBF0123002385F87730C9
:108800004FF4CC7201232A491048FEF7E9FD0023FA
:10881000942228490D4884ED110AFEF7E1FDBCEED3
:10882000C00A01234FF42C722349084884ED0D0A35
:10883000FEF7D6FD214B84ED120A19680448A822E0
:10884000BDE8384016F0B8BAF89702000498020064
:10885000EC15FF1F0C9802002098020034980200CB
:10886000489802005C980200709802008498020008
:10887000A0980200B0980200C0980200D4980200AC
:10888000E0980200F098020000990200149902009A
:10889000209902003499020044990200589902007C
:1088A0006899020078990200889902009499020060
:1088B000A0990200B4990200C49902007C14FF1F21
:1088C00038B53A4D3A493B4C284600234FF4EE72F6
:1088D000FEF786FDBDEEC00A284600234FF4C472A1
:1088E000354984ED130AFEF77BFDBDEEC00A28462C
:1088F0000023B022314984ED140AFEF771FDBDEE6C
:10890000C00A284600234FF4D4722D4984ED200A72
:10891000FEF766FDBDEEC00A284600234FF4307214
:10892000284984ED060AFEF75BFDBDEEC00A284625
:1089300000238C22244984ED070AFEF751FDBDEE89
:10894000C00A284600234FF41572204984ED1E0A00
:10895000FEF746FDBDEEC00A284600234FF4107214
:108960001B4984ED0B0AFEF73BFDBDEEC00A28460D
:108970000023B022174984ED0C0AFEF731FDBDEE4D
:10898000C00A28460023B822134984ED1F0AFEF7C7
:1089900027FD124BBDEEC00A2046196884ED1F0A60
:1089A000A822BDE8384016F007BA00BFD4990200EB
:1089B000CC990200EC15FF1FDC990200E49902003B
:1089C000EC990200F4990200FC990200049A02005A
:1089D0000C9A0200149A02001C9A02007C14FF1FD9
:1089E00038B5314D3149324C284600234FF43E72A0
:1089F000FEF7F6FCBDEEC00A284600234FF43F7296
:108A00002C4984ED150AFEF7EBFCBDEEC00A2846A2
:108A100000234FF44072284984ED160AFEF7E0FC6B
:108A2000BDEEC00A284600234FF44172234984ED6D
:108A3000170AFEF7D5FCBDEEC00A284600234FF406
:108A400044721F4984ED180AFEF7CAFCBDEEC00A45
:108A5000284600234FF445721A4984ED190AFEF79F
:108A6000BFFCBDEEC00A284600234FF442721649EF
:108A700084ED1A0AFEF7B4FCBDEEC00A28460023B6
:108A80004FF44372114984ED1B0AFEF7A9FC104B09
:108A9000BDEEC00A2046196884ED1C0AA822BDE874
:108AA000384016F089B900BF289A0200EC93020002
:108AB000EC15FF1F00940200309A0200409A020059
:108AC000509A0200609A0200709A0200809A020096
:108AD0007C14FF1F70B5574D5749584C584E2846C7
:108AE00000234FF4E472FEF77BFCBDEEC00A28467B
:108AF00000234FF47272534984ED000AFEF770FCB4
:108B0000BDEEC00A284600234FF477724E4984ED2B
:108B1000010AFEF765FCBDEEC00A284600232822A4
:108B20004A4984ED020AFEF75BFCBDEEC00A284606
:108B30000123A822464984ED030AFEF751FC28468A
:108B400001234FF4C672434984ED0A0AFEF748FC3C
:108B5000284600234FF47A723F4984ED0D0AFEF750
:108B60003FFCBDEEC00A284600234FF47D723B490E
:108B700084ED040AFEF734FCBDEEC00A284600234B
:108B80002422374984ED050AFEF72AFCBDEEC00A0F
:108B9000284601234FF4AA72324984ED060AFEF7F3
:108BA0001FFC284601234FF49E722F4984ED0B0AC7
:108BB000FEF716FC284600234FF45E722B4984ED25
:108BC0000E0AFEF70DFCBDEEC00A284600234FF446
:108BD0005F72274984ED070AFEF702FCBDEEC00A6A
:108BE000284600235C22234984ED080AFEF7F8FB9F
:108BF000BDEEC00A284601234FF4A6721E4984ED3B
:108C0000090AFEF7EDFB2046316884ED0C0A40228C
:108C100016F0D2F828464FF4FA7218490123FEF7ED
:108C2000DFFB316884ED0F0A20464022BDE870402A
:108C300016F0C2B8909A0200D0930200AC15FF1F44
:108C40006C07FF1F28940200349402003C94020039
:108C5000949A0200A09A0200509402005C940200D0
:108C600064940200AC9A0200B89A02007894020060
:108C7000849402008C940200C49A0200D09A0200EC
:108C8000464B474A1B68116810B5012B08BF454B7E
:108C90009AB008BF19680AA80023012215F052FDF6
:108CA00011A813F0DDFA002840F0818102A89DF898
:108CB00042303D490AAA13F087FB049A9DF814300C
:108CC0009DF80C1013928DF850308DF8481005AABD
:108CD0000DF151030DF15E0012F8011F03F8011BA5
:108CE0008342F9D1099B189302A813F08BFA11A8BB
:108CF00013F0B6FA0446002864D1012318212B484A
:108D00008DF8433018F0F2FC294819F07FF9294911
:108D100002A819F049FB214602A8F8F785FC02A831
:108D200019F002FB244902A819F03EFB214602A8D3
:108D3000F8F77AFC02A819F0F7FA204902A819F00E
:108D400033FB214602A8F8F76FFC02A819F0ECFAF1
:108D5000194902A819F028FB214602A8F8F764FC7B
:108D600002A819F0E1FA164902A819F01DFB2146E4
:108D700002A8F8F759FC02A819F0D6FA0E4902A881
:108D800019F012FB214602A8F8F74EFC02A819F0D0
:108D9000CBFA0AA815F0F4FC1AB010BDB017FF1FEB
:108DA0006407FF1F7407FF1F6019FF1FF49A02007A
:108DB0002408FF1F109B02003089020044AB020010
:108DC00090930200002314217B488DF8433018F063
:108DD0008DFC7A4819F01AF911A813F041FA00280D
:108DE00040F0E180FFF7F8FBFFF7FAFDFFF768FDC1
:108DF000FEF77AFEFEF7C2FDFFF75AFAFFF76AFEAA
:108E0000FEF728FFFFF700F8FEF778FCFFF712F9EE
:108E10006B4902A819F0C8FA002102A8F8F704FC6F
:108E200002A819F081FA674902A819F0BDFA0021D9
:108E300002A8F8F7F9FB02A819F076FA624A13685B
:108E40000193019913680093009B5B1A0E2BF9D9CB
:108E50005E4902A819F0A8FA002102A8F8F7E4FB7D
:108E600002A819F061FA574902A819F09DFA0021E9
:108E700002A8F8F7D9FB02A819F056FA544902A83B
:108E800019F092FA002102A8F8F7CEFB02A819F017
:108E90004BFA4C4902A819F087FA002102A8F8F70A
:108EA000C3FB02A819F040FA4A4902A819F07CFA5B
:108EB000002102A8F8F7B8FB02A819F035FA4149D9
:108EC00002A819F071FA002102A8F8F7ADFB02A878
:108ED00019F02AFA404902A819F066FA002102A8FE
:108EE000F8F7A2FB02A819F01FFA364902A819F0F8
:108EF0005BFA002102A8F8F797FB02A819F014FA10
:108F0000364902A819F050FA002102A8F8F78CFBA4
:108F100002A819F009FA2B4902A819F045FA002114
:108F200002A8F8F781FB02A819F0FEF92C4902A863
:108F300019F03AFA002102A8F8F776FB02A819F016
:108F4000F3F9204902A819F02FFA002102A8F8F736
:108F50006BFB02A819F0E8F9224902A819F024FADB
:108F6000002102A8F8F760FB02A819F0DDF9154905
:108F700002A819F019FA002102A8F8F755FB02A877
:108F800019F0D2F9184902A819F00EFA002102A826
:108F9000F8F74AFB02A819F0C7F90A4902A819F024
:108FA00003FA0021EFE611A813F04CF91AE711A813
:108FB00013F048F97AE600BFDC9A02002408FF1F8C
:108FC000109B020030890200141CFF1F44AB0200FA
:108FD000209B02002C9B0200389B0200449B020055
:108FE000509B02005C9B0200689B020090F890304E
:108FF00010B504461BB906E0012016F097F8A368E7
:10900000002BF9D110BDF7F7BFFAF8E78368E3B199
:10901000816D826F4B68D21A30B482EAE273D0F865
:10902000AC40A3EBE273A34210DBD0F8B020934234
:1090300014DA1A190025C2672346C0F8B05030BCB4
:109040004A68086800FB0323CB60704700225C007D
:10905000C0F8B020C0F8AC20C467F0E7C26FD31AE4
:10906000EDE700BF10B50446FFF7D0FFA3682BB1B2
:10907000012016F05BF8A368002BF9D110BD00BFEA
:1090800007EE901AF8EE676A07EE902A9FED1C7AB9
:10909000DFED1C5A9FED1C6A4167F8EE677A66EEB9
:1090A000876A67EE877A66EEA56A27EEA57AF6EEFE
:1090B000007AF0EE675AE6EE865AF0B4E7EE067AEA
:1090C0000346124F5861FDEEE56AFDEEE77A104E59
:1090D0000267802500220124076046600574C4668B
:1090E000C0ED066AC0ED077A8260C26080F8282071
:1090F000C265026680F864208266F0BC704700BFDB
:10910000BD378635C0E1644C0000003D0C8502008F
:109110000085020038B590F86430114A02600446B8
:1091200000F10C0553B1284618F0DEFE0023206A3A
:10913000A36015F0CDFA606A15F0CAFA094B6360B6
:10914000284618F0D1FE0023A360206A15F0C0FA6B
:10915000606A15F0BDFA284618F0C6FE204638BDF4
:109160000C8502000085020010B5034B0360044625
:10917000FFF7D0FF204610BD4485020010B5054B17
:1091800003600446FFF7C6FF2046B82118F000FF31
:10919000204610BD4485020010B5034B0360044611
:1091A000FFF7B8FF204610BD2885020010B5054B1B
:1091B00003600446FFF7AEFF2046942118F0E8FE56
:1091C000204610BD2885020010B50446FFF7A2FF17
:1091D0002046782118F0DCFE204610BD884231D0B0
:1091E0002DE9F04700F10408414516468A468146BC
:1091F00017D0D9F80010D8F80000B04798B9D8F8BF
:109200000050444601E0236863602746284654F82E
:10921000041DB0470028F6D13D6008F10408C2459E
:10922000E7D1BDE8F087C9EB08029308D8F8004001
:1092300005D0C2F10400404449461CF05BF9C9F86E
:109240000040EAE7704700BF2DE9F8430B1A432BB3
:109250001CDD00F14008894641461746FFF7BEFF76
:10926000C14515D0D8F80050444601E0236863603A
:109270002646284654F8041DB8470028F6D108F1C0
:109280000408C1453560EDD1BDE8F883FFF7A6FFBE
:10929000BDE8F8832DE9F04F561E06EBD67683B075
:1092A0007610B14201928846054699460C9F5CDAD9
:1092B0008A4600E0DA460AF101034FEA430B0BF15C
:1092C0008041013955F8330055F8211005EBC304EE
:1092D000B84718B10BF1FF3B05EB8B04236845F849
:1092E0002A30B345E6DB019BDA0707D4019BA3F1E3
:1092F000020A0AEBDA7ABBEB6A0F06D0C34514DC2C
:10930000C4F8009003B0BDE8F08F0BF1010B4FEAF9
:109310004B0B0BF18043013B0BF1FF3B55F8233026
:109320002360C34505EB8B04EADD0BF1FF3606EB4A
:10933000D6767610494655F82600B847731E03EBDB
:10934000D37305EB86045B1030B905EB8B04C4F8CE
:10935000009003B0BDE8F08F55F8262045F82B208B
:10936000B045CDDAB3461E46E4E7019BDB0700EBD0
:109370008104C5D48B46B9E72DE9F04F0C1A432C74
:1093800085B040F389800546894692461E46002AEC
:1093900061D0031D0393E410686855F82410B047AA
:1093A0000AF1FF3A59F8041C002834D055F824007B
:1093B000B047002837D02B6855F824202A6045F89C
:1093C000243068682968039FCB46B846B04780B907
:1093D000ABF1040421682868A346043CB047002888
:1093E000F8D15F4509D23A68DBF800103960CBF854
:1093F000002057F8040F2968E7E7494633465246EC
:1094000038467C1BFFF7B8FF432C45DDBAF1000F4F
:1094100022D0B946BFE76868B04798B195E8030025
:1094200029606860CFE759F8041C6868B0470028D5
:10943000F4D02B6859F8042C2A6049F8043C686879
:109440002968C0E759F8041C55F82400B0472B6878
:109450000028B1D0EEE78846A410A71E7F1005EBC8
:10946000870900E0013F59F8043900962246394641
:109470002846FFF70FFF002FF4D158F8043D2A6863
:109480000096C5EB0804C8F800200021A210284669
:10949000FFF700FF072CF0DC05B0BDE8F08F00BF40
:1094A000836833B1614B1B6813B101210220184757
:1094B00070472DE9F04700F12C064FEA810906EBD1
:1094C0000905AE422DED028B10EE107A8846044657
:1094D00010D04FEAA902B2FA82F2C2F11F02520082
:1094E00029463046524BFFF747FF514A294630463E
:1094F000FFF7AAFEE16AA1658A69002A00F08E8062
:1095000082EAE273A3EBE273B8F1010F4FF00002BD
:109510000B618A6012DD09F1280EA644304650F82E
:10952000042F936983EAE37CACEBE37CC2F810C0C0
:109530000B697045C3EB4C035361F0D1AE4271D05F
:109540004A6A04F1300306E01968496A8A4203F165
:10955000040328BF0A469D42F6D108EE102A0023D4
:10956000251D84F8903084F82830284615F09CF8A2
:109570002062284615F098F8606215F069F804F149
:109580000800616915F01AF8A36DD4ED1C6A93ED1B
:10959000067A9FED286A5B68F8EE487AF8EE666A0C
:1095A000B8EEC77A67EEA67A84ED207A87EE867ADF
:1095B0000022E26784ED217A72B6D4F88430C4F8D0
:1095C000883062B672B694ED200AD4ED1F7A07EEA9
:1095D000107A27EE000AB4EEE70AD4ED227A84ED81
:1095E0001E0AF1EE10FAD8BFF1EE677AC4ED237AC5
:1095F00062B6114A236AE06900211160DB005168FC
:1096000003F1804303F5603301440D2019611060BC
:10961000DA68502122F08002DA60D960BDEC028B5A
:10962000BDE8F087E36A93ED098A98E7DC1BFF1F2A
:109630007D04000000247449008003402DE9F04FB0
:109640002DED028BD3B041F28832052181462DA841
:10965000FFF716FDA748A84B2D9300230360A74DE5
:10966000A748DFF8B48203602A6BA648D8F81C60CC
:109670008DF8443101210360D8F818704891032A0D
:1096800000F20484DFE812F0DE00C500AC00040044
:10969000D5ED057A9FED9C8A6B68D5F824B00193CF
:1096A000F8EEE77A07EE109A67EE887AB8EEC78A86
:1096B000022227EE888A0324F6B230460121FFB247
:1096C00000920DF1740A15F017FD3846012115F0CE
:1096D00013FD2146009A8D4C504614F079FE00236C
:1096E0001E9323680693069923680593059A874B72
:1096F000521A042AF8D901990093504614F0AAFE90
:10970000594614F09BFE824914F0C8FE012211460E
:10971000286BF7F7C3F9479A52AB02F10B0E03EB34
:109720008E0E03EB82024FF0000C42F868ACB7EEED
:10973000000A01212DA84EF890CCCDF81CC1FFF7EE
:10974000AFFE009B1B680493049A23680393039B5A
:109750009B1A042BF9D900238DF8443172B6DDED44
:109760004D7A9DED4C7A68EE277AB4EEE77ACDED2E
:109770004B7ADDED4F7AF1EE10FA58BFF1EE677AD1
:10978000CDED507A62B6DFF894A1DFF894B1DFED49
:109790005E8A2F9B002B00F0EC80F8F773FC00280A
:1097A00040F39080DAF80000F8F75CFCC0B2532870
:1097B0008BF8000000F05082662840F08380DAF8D1
:1097C0000000F7F785FA51EC100B1AF0BBFF2B6B7A
:1097D000032B59D8DFE813F0360328031A034B0094
:1097E000D5ED087A9FED488A2B690193F8EEE77A68
:1097F00007EE109A67EE887AB8EEC78AD8F85060FC
:10980000D8F84C70D5F800B0172227EE888A1024BB
:1098100052E7D5ED077A9FED3C8AEB680193F8EEAD
:10982000E77A07EE109A67EE887AB8EEC78AD8F81A
:109830003060D8F82C70D5F82CB0142227EE888A26
:10984000152439E7D5ED067A9FED2F8AAB68019391
:10985000F8EEE77A07EE109A67EE887AB8EEC78AD4
:10986000D5F828B0052227EE888A062424E707EEDB
:10987000900AB8EEE78A07EE909A28EE288AF8EE6A
:10988000E77A686128EE278A224B1C48196834223F
:1098900015F092FA00238DF8443172B6DDED4D7A61
:1098A0009DED4C7A68EE277AF4EEC77ACDED4B7ACF
:1098B000DDED4F7AF1EE10FAD8BFF1EE677ACDED1B
:1098C000507A62B6304615F01DFC10B9B9F1010F9F
:1098D0002AD0384615F016FC10B9B9F1FF3F23D055
:1098E00023680C930C9A23680B930B9B9B1A092BF0
:1098F000F9D94EE7F812FF1F28850200C013FF1F99
:109900006418FF1FB412FF1F0AD7233C141CFF1F4B
:10991000C09EF87F8407FF1FEC15FF1F4807FF1F3D
:10992000F413FF1F000000008DF8440172B65FEDD4
:10993000036ADDED4D7A9DED4C7A67EEA67AF4EE82
:10994000C77AF1EE10FACDED4B7A00F38982DDEDA6
:109950004F7AF1EE677ACDED507A62B630A818F002
:10996000C3FA002335982F9314F0B2FE369814F002
:10997000AFFE286B032800F0A3811E9BA24AA34FD1
:10998000136007EE903A4FF0000AB8EEE70AC7F806
:1099900000A0F7F7C1F919AEDFF8B4929C4989ED40
:1099A000000A304618F000FD51463046F7F73CFEFD
:1099B000304618F0B9FC2220F7F7B4FF99ED000A01
:1099C0005046F7F753FF2220F7F7ACFFFF20F7F7D9
:1099D000A9FFFF20F7F7A6FFFF20F7F7A3FF2368F3
:1099E0001893189923681793179B8A4A5B1A042BBC
:1099F000F8D987490092304618F0D6FC002130464D
:109A0000F7F712FE304618F08FFC2220F7F78AFF96
:109A100099ED000A0020F7F729FF2220F7F782FFCF
:109A2000FF20F7F77FFFFF20F7F77CFFFF20F7F716
:109A300079FF009A13681693169923681593159B5E
:109A4000744A5B1A042BF8D973490092304618F017
:109A5000ABFC00213046F7F7E7FD304618F064FC18
:109A60002220F7F75FFF97ED000A0020B8EEC00A4A
:109A7000F7F7FCFE2220F7F755FFFF20F7F752FF1C
:109A8000FF20F7F74FFFFF20F7F74CFF009A13680E
:109A90001493149A23681393139B9B1A042BF9D9DC
:109AA00001220021286BF6F7F9FF2B6B032B4AD814
:109AB000DFE803F08D705302D8F8A430012B00F0DA
:109AC000E3815649304618F06FFC00213046F7F725
:109AD000ABFD304618F028FC5149304618F064FCC4
:109AE00000213046F7F7A0FD304618F01DFC4D4927
:109AF000304618F059FC00213046F7F795FD304606
:109B000018F012FC4849304618F04EFC002130464F
:109B1000F7F78AFD304618F007FC4449304618F044
:109B200043FC00213046F7F77FFD304618F0FCFB80
:109B30003F49304618F038FC30460021F7F774FDF5
:109B4000304618F0F1FB3B4B2D932DA8FFF7E2FABE
:109B500053B0BDEC028BBDE8F08FD8F8A430012BD8
:109B600000F08E813449304618F01EFC002130464A
:109B7000F7F75AFD304618F0D7FB2949304618F060
:109B800013FC00213046F7F74FFD304618F0CCFBB0
:109B90002A49ADE7D8F8A430012B00F064812849A8
:109BA000304618F001FC00213046F7F73DFD304605
:109BB00018F0BAFB1A49304618F0F6FB002130467F
:109BC000F7F732FD304618F0AFFB1E4990E7D8F8A2
:109BD000A430012B00F056811B49304618F0E4FBFD
:109BE00000213046F7F720FD304618F09DFB0C4968
:109BF000304618F0D9FB00213046F7F715FD304606
:109C000018F092FB114973E7B412FF1F6C15FF1F88
:109C1000849B0200141CFF1F749B0200689C0200BE
:109C2000308902007C9C0200688B0200D09B0200FD
:109C3000448B0200288502002C9C0200409C0200FC
:109C4000F09B0200049C0200A89B0200BC9B020047
:109C5000BC13FF1F0000000000238DF8443172B6D2
:109C60005FED046ADDED4D7A9DED4C7A67EEA67AE4
:109C7000F4EEC77ACDED4B7ADDED4F7AF1EE10FAC6
:109C8000D8BFF1EE677ACDED507A62B623680A93B9
:109C90000A9A23680993099B814E9B1A042BF8D9D1
:109CA0002DA8FFF7A3F933680893089A2368079350
:109CB000079B9B1A632BF9D9286B03287FF45DAEB1
:109CC000D8F80410D8F800301E9A98ED027ADFED2B
:109CD000756A7548754F026003FB01F307EE903A11
:109CE00006EE102AF8EE677AB8EEC66A67EE877A53
:109CF0006F4B70491A6086EE277A6F4B19AE4FF0A2
:109D000000093046C3F8009067EE267AC7ED007A66
:109D100018F04AFB49463046F7F786FC304618F003
:109D200003FB2220F7F7FEFD97ED000A4846F7F700
:109D30009DFD2220F7F7F6FDFF20F7F7F3FDFF204A
:109D4000F7F7F0FDFF20F7F7EDFD23681293129966
:109D500023681193119B524A5B1A042BF8D9554979
:109D60000092304618F020FB00213046F7F75CFCEB
:109D7000304618F0D9FA2220F7F7D4FD97ED000A03
:109D80000020F7F773FD2220F7F7CCFDFF20F7F74F
:109D9000C9FDFF20F7F7C6FDFF20F7F7C3FD009AC6
:109DA00013681093109A23680F930F9B3C4F9B1AD4
:109DB000042BF8D94149304618F0F6FA0021304614
:109DC000F7F732FC304618F0AFFA2220F7F7AAFD79
:109DD000394B93ED000A0020B8EEC00AF7F746FDB4
:109DE0002220F7F79FFDFF20F7F79CFDFF20F7F7F4
:109DF00099FDFF20F7F796FD3B680E930E9A2368B6
:109E00000D930D9B9B1A042BF9D949E607EE900A96
:109E1000B8EEE78A07EE909A28EE288AF8EEE77AFD
:109E2000286228EE278A2FE507EE900AB8EEE78A27
:109E300007EE909A28EE288AF8EEE77AE86128EE95
:109E4000278A21E507EE900AB8EEE78A07EE909A96
:109E500028EE288AF8EEE77AA86128EE278A13E52B
:109E6000DDED4F7A77E51649304618F09DFA00216E
:109E70003046F7F7D9FB304618F056FA114958E644
:109E80001149F1E71149EFE71149EDE74FF0000BF8
:109E90009FED108ACDF804B0052206240CE400BF23
:109EA000141CFF1F0000B4436418FF1F9416FF1F0B
:109EB0006C15FF1F749B0200B412FF1F849B0200ED
:109EC000DC9B020030890200189C0200949B020077
:109ED000549C0200000000002DE9F04F2DED048B92
:109EE000ADF54B7D14460090029141F28832052178
:109EF00080A8FFF7C5F84FF0000B754B8093012544
:109F000041F288320521A5A89B95724E8DF890B23A
:109F1000FFF7B6F86E4BA5930222032140A8C09527
:109F20008DF824B314F054FA10216B48D6F81C8035
:109F3000D6F81890694F17F0D9FB2146684818F0F9
:109F4000B5F8674818F062F8032C4FF005024FF09F
:109F5000060150A8BABF5D4601245C4614F038FAE9
:109F60001422152160A814F033FA172270A81021CA
:109F700014F02EFA3A6B012A01F01E82022A01F037
:109F8000EE81002A00F0B8859FED568ADFF87CA1AB
:109F90005FFA88F8404601215FFA89F915F0ACF8BC
:109FA0000121484615F0A8F800224192DAF8002075
:109FB0007B690C9203930C997B68D7F824B00193CA
:109FC000DAF800300B930B9B5B1A042BF8D9019A3B
:109FD000029B03FB02F3194640A814F03BFA5946D2
:109FE00014F02CFA404914F059FA08213F4817F0B0
:109FF0007DFB0A213E4817F079FB0199384818F09B
:10A0000055F8374818F002F80821384817F06EFB69
:10A010000721384817F06AFB5946314818F046F8CE
:10A020002F4817F0F3FF0821304817F05FFB11218C
:10A03000314817F05BFB2C49294818F037F82848BD
:10A0400017F0E4FFE4B1D7F830B0BBF1010F01F035
:10A05000D182BBF1020F01F07482BBF1000F01F05D
:10A0600014820521254817F041FB0421244817F0EC
:10A070003DFB01211A4818F019F8194817F0C6FFDE
:10A08000002D41F0CF80DFED178A9FED1E9A14B9A5
:10A09000002D00F06D87DAF800301893189ADAF87E
:10A0A00000301793179B9B1A042BF8D9F7F7EAFF98
:10A0B0000028C0F2AF80DFF858B0DBF80000F7F7F7
:10A0C000D1FF1149C0B2A0F15303087022E000BFD4
:10A0D00028850200EC15FF1F909C02002819FF1F25
:10A0E0002408FF1F00000000C09EF87FA49C02000F
:10A0F000B09C0200D48C0200BC9C0200D09C0200E8
:10A10000D89C02000AD7233CF413FF1F141CFF1F26
:10A110004807FF1F722B7DD8DFE813F0FE037C0099
:10A120007C007C007C007C007C008604B1037C0009
:10A130007C007C007C007C007C007C002A037C008E
:10A140007C007C007C007C007C007C00D7027202DA
:10A150007C0042020B027C007C007C007C007C00C6
:10A160007C007C007C007C007C007C007C007C000F
:10A170007C007C007C007C007C007C007C007C00FF
:10A180007C007C007C007C007C007C007C007C00EF
:10A190007C007C007C007C007C007C007C007C00DF
:10A1A0007C007C007C007C007C007C007C007C00CF
:10A1B0007C007C007C007C007C007C007C007C00BF
:10A1C000BE016A017C007C007C007C0002018A00E8
:10A1D0007C007C007C007C007C007C007C007C009F
:10A1E0007C007C007C007C007C007C007C007C008F
:10A1F0007C007C007C007C007C007C007C007C007F
:10A200007300F7F753FFA04B386319689F48342257
:10A2100014F0D2FD002C6FD1DAF800303493349A68
:10A22000DAF800303393339B9B1A042BF8D92EE7CE
:10A23000A79B002BEED1D7ED087A3969009370A85F
:10A24000B8EEE78A14F006F9914914F027F90122D3
:10A2500011460220F6F722FCBF9A009BBF93CAA9C1
:10A2600001EB820470AA44F8643CB7EE000A0121B5
:10A27000A5A844F8682CFFF713F9009B8DF8243348
:10A2800028EE098A72B6DDEDC57A9DEDC47A67EED7
:10A29000A87AF4EEC77ACDEDC37ADDEDC77AF1EE98
:10A2A00010FAD8BFF1EE677ACDEDC87A62B6DAF867
:10A2B00000302E932E9ADAF800302D932D9B9B1AA6
:10A2C000042BF8D900238DF8243372B6DDEDC57A5E
:10A2D0009DEDC47A68EE277AF4EEC77ACDEDC37AA5
:10A2E000DDEDC77AF1EE10FAD8BFF1EE677ACDED69
:10A2F000C87A62B601230093404614F003FF044677
:10A3000018B9009B012B00F02484484614F0FAFE93
:10A31000044618B9009B013300F0268501247BE731
:10A32000A79B002B7FF476AF3969D7ED087A0093AD
:10A33000494270A8B8EEE78A14F08CF8554914F039
:10A34000ADF8012211460220F6F7A8FBBF9A009B48
:10A35000BF93CAA901EB820470AA44F8643CB7EE2B
:10A36000000A0121A5A844F8682CFFF799F8009B82
:10A370008DF8243328EE098A72B6DDEDC57A9DED9D
:10A38000C47A67EEA87AF4EEC77ACDEDC37ADDED34
:10A39000C77AF1EE10FAD8BFF1EE677ACDEDC87A40
:10A3A00062B6DAF800302C932C9ADAF800302B934E
:10A3B0002B9B9B1A042BF8D900238DF8243372B6FB
:10A3C000DDEDC57A9DEDC47A68EE277AF4EEC77AA2
:10A3D000CDEDC37ADDEDC77AF1EE10FAD8BFF1EE1C
:10A3E000677ACDEDC87A62B64FF0FF33009383E70A
:10A3F000A79B002B7FF40EAFD7ED077AF968009387
:10A4000060A8B8EEE78A14F025F8214914F046F860
:10A41000012211461046F6F741FBBF9A009BBF93FD
:10A42000CAA901EB820460AA44F8643CB7EE000AB2
:10A430000121A5A844F8682CFFF732F8009B8DF89D
:10A44000243328EE098A72B6DDEDC57A9DEDC47A13
:10A4500067EEA87AF4EEC77ACDEDC37ADDEDC77A60
:10A46000F1EE10FAD8BFF1EE677ACDEDC87A62B698
:10A47000DAF800302A932A9ADAF800302993299BD7
:10A480009B1A042BF8D91DE79007FF1F2819FF1FFF
:10A49000C09EF87F40610780A79B002B7FF4BAAE77
:10A4A000F968D7ED077A0093494260A8B8EEE78AC9
:10A4B00013F0D0FFAA4913F0F1FF01221146104614
:10A4C000F6F7ECFABF9A009BBF93CAA901EB82048E
:10A4D00060AA44F8643CB7EE000A0121A5A844F83C
:10A4E000682CFEF7DDFF009B8DF8243328EE098AE7
:10A4F00072B6DDEDC57A9DEDC47A67EEA87AF4EE0A
:10A50000C77ACDEDC37ADDEDC77AF1EE10FAD8BF88
:10A51000F1EE677ACDEDC87A62B6DAF800302893AA
:10A52000289ADAF800302793279B9B1A042BF8D936
:10A5300042E7DBF80000F6F7CBFB51EC100B1AF00A
:10A5400001F93B6B874A012B00F07F87022B00F05B
:10A55000858733B907EE900AB8EEE78A906128EE56
:10A56000098A814B7F481968342214F025FC0023A6
:10A570008DF8243372B6DDEDC57A9DEDC47A68EEB0
:10A58000277AF4EEC77ACDEDC37ADDEDC77AF1EE26
:10A5900010FAD8BFF1EE677ACDEDC87A62B639E627
:10A5A000DBF80000F6F794FB51EC100B1AF0CAF838
:10A5B0006D4B834619686B48C7F814B0342214F009
:10A5C000FBFB00238DF8903272B607EE90BAB8EE1E
:10A5D000E77ADDEDA07ADDED9F6A27EE097A67EE76
:10A5E000277AF4EEE67ACDED9E7ADDEDA27AF1EEF1
:10A5F00010FAD8BFF1EE677ACDEDA37A62B609E61C
:10A60000DDF808B2BBF1000F7FF404AED7ED057A98
:10A61000019BF8EEE77A594240A867EE899A13F059
:10A6200019FF524913F03AFF012211460320F6F7B1
:10A6300035FA9A9ACDF868B280AB03EB82051846DA
:10A6400040ABB7EE000A0121EB62C5F830B0FEF76F
:10A6500027FF8DF890B272B6DDEDA07A9DED9F7A5E
:10A6600067EEA87AF4EEC77ACDED9E7ADDEDA27A98
:10A67000F1EE10FAD8BFF1EE677ACDEDA37A62B6AB
:10A68000DAF800302693269ADAF800302593259BD5
:10A690009B1A042BF8D900238DF8903272B6DDEDA9
:10A6A000A07A9DED9F7A69EEA77AF4EEC77ACDED98
:10A6B0009E7ADDEDA27AF1EE10FAD8BFF1EE677A5C
:10A6C000CDEDA37A62B60125A4E5DDF808B2BBF1B1
:10A6D000000F7FF49FADD7ED057A0199F8EEE77A88
:10A6E00040A867EE899A13F0B5FE204913F0D6FE14
:10A6F000012211460320F6F7D1F99A9ACDF868B2F3
:10A7000080AB03EB8205184640ABB7EE000A01218F
:10A71000EB62C5F830B0FEF7C3FE8DF890B272B6AA
:10A72000DDEDA07A9DED9F7A67EEA87AF4EEC77A08
:10A73000CDED9E7ADDEDA27AF1EE10FAD8BFF1EE02
:10A74000677ACDEDA37A62B6DAF800302493249AC2
:10A75000DAF800302393239B9B1A042BF8D99AE74D
:10A76000406107802819FF1F9007FF1FC09EF87FD8
:10A7700000238DF8243372B6DDEDC57A9DEDC47AE1
:10A7800067EEA87AF4EEC77ACDEDC37ADDEDC77A2D
:10A79000F1EE10FAD8BFF1EE677ACDEDC87A62B665
:10A7A000DAF800302093209ADAF800301F931F9BCC
:10A7B0009B1A042BF8D9A5A8FEF718FC396B0129C0
:10A7C00000F05C86022900F0528619B90122084681
:10A7D000F6F764F9D6F8A430012B00F02886B849C2
:10A7E0003CA817F0E1FD00213CA8F6F71DFF3CA8AE
:10A7F00017F09AFDB3493CA817F0D6FD00213CA8FC
:10A80000F6F712FF3CA817F08FFDAF493CA817F0F0
:10A81000CBFD00213CA8F6F707FF3CA817F084FD0C
:10A82000AA493CA817F0C0FD00213CA8F6F7FCFEA1
:10A830003CA817F079FDA6493CA817F0B5FD00210A
:10A840003CA8F6F7F1FE3CA817F06EFDA1493CA824
:10A8500017F0AAFD00213CA8F6F7E6FE3CA817F089
:10A8600063FDDAF800302293229ADAF8003021935F
:10A87000219B9B1AB3F57A7FF7D30024CCE4DDF853
:10A880009CB2BBF1000F7FF4C5ACB968D7ED067A76
:10A89000494250A8B8EEE78A13F0DCFD8E4913F068
:10A8A000FDFD012211465846F6F7F8F8BF9ACDF89B
:10A8B000FCB2CAAB03EB820450ABB7EE000A012135
:10A8C000A5A844F8683C44F864BCFEF7E9FD28EE0E
:10A8D000098A8DF824B372B6DDEDC57A9DEDC47A90
:10A8E00067EEA87AF4EEC77ACDEDC37ADDEDC77ACC
:10A8F000F1EE10FAD8BFF1EE677ACDEDC87A62B604
:10A90000DAF800301E931E9ADAF800301D931D9B72
:10A910009B1A042BF8D94FE50821704816F0E6FE83
:10A9200006216F4816F0E2FE00238DF8903272B6D1
:10A93000DDEDA07A9DED9F7A67EEA87AF4EEC77AF6
:10A94000CDED9E7ADDEDA27AF1EE10FAD8BFF1EEF0
:10A95000677ACDEDA37A62B6DAF800301A931A9AC4
:10A96000DAF800301993199B9B1A042BF8D980A8A8
:10A97000FEF73CFB0821594816F0B8FE072159485C
:10A9800016F0B4FE584817F041FB012200210320C5
:10A99000F6F784F8D6F8A430012B00F03A85534935
:10A9A0003CA817F001FD00213CA8F6F73DFE3CA8AD
:10A9B00017F0BAFC43493CA817F0F6FC00213CA86C
:10A9C000F6F732FE3CA817F0AFFC49493CA817F057
:10A9D000EBFC00213CA8F6F727FE3CA817F0A4FCEE
:10A9E0003A493CA817F0E0FC00213CA8F6F71CFE11
:10A9F0003CA817F099FC36493CA817F0D5FC00217B
:10AA00003CA8F6F711FE3CA817F08EFC31493CA893
:10AA100017F0CAFC00213CA8F6F706FE3CA817F088
:10AA200083FC0025FFF7F6BBDDF89CB2BBF1000FFD
:10AA30007FF4F0ABD7ED067AB96850A8B8EEE78A94
:10AA400013F008FD2B4913F029FD01221146584649
:10AA5000F6F724F8BF9ACDF8FCB2CAAB03EB820438
:10AA600050ABB7EE000A0121A5A844F8683C44F8B1
:10AA700064BCFEF715FD28EE098A8DF824B372B682
:10AA8000DDEDC57A9DEDC47A67EEA87AF4EEC77A5B
:10AA9000CDEDC37ADDEDC77AF1EE10FAD8BFF1EE55
:10AAA000677ACDEDC87A62B6DAF800301C931C9A4A
:10AAB000DAF800301B931B9B9B1A042BF8D901E496
:10AAC000409D020030890200549D0200688B020004
:10AAD000D09B0200448B020040610780A49C0200CE
:10AAE000E09C0200E89C02002408FF1F049D020075
:10AAF000189D0200C09EF87F009BB968D7ED067ACA
:10AB0000D7F828B0519201FB03F150A80192B8EE9A
:10AB1000E78AD6F81C80D6F81890DFF848A213F020
:10AB200099FC594613F08AFC019A114613F0D0FCA7
:10AB3000DAF8002006920699DAF800300593059BB2
:10AB40005B1A042BF8D97C4950A813F0C1FCFFF71D
:10AB50001FBA1821794816F0C9FD794817F056FA3E
:10AB60008DF8244372B6DDEDC57A9DEDC47A67EEAB
:10AB7000A87AF4EEC77AF1EE10FACDEDC37A40F37D
:10AB80000D83DDEDC77ACDEDC87A62B6A8A817F0BF
:10AB9000ABF90024AD98A79413F09AFDAE9813F08A
:10ABA00097FDD6F88C30002B78D08DF8904272B695
:10ABB000DDEDA07A9DED9F7A67EEA87AF4EEC77A74
:10ABC000CDED9E7ADDEDA27AF1EE10FAD8BFF1EE6E
:10ABD000677ACDEDA37A62B6DAF800303093309A16
:10ABE000DAF800302F932F9B9B1A042BF8D983A8F7
:10ABF00017F07AF900258898829513F069FD8998F5
:10AC000013F066FD294601220320F5F747FFD6F829
:10AC1000A430012B00F085834A493CA817F0C4FBFF
:10AC200029463CA8F6F700FD3CA817F07DFB4649F5
:10AC30003CA817F0B9FB29463CA8F6F7F5FC3CA860
:10AC400017F072FB41493CA817F0AEFB29463CA81F
:10AC5000F6F7EAFC3CA817F067FB3D493CA817F063
:10AC6000A3FB29463CA8F6F7DFFC3CA817F05CFBE9
:10AC700038493CA817F098FB29463CA8F6F7D4FCC5
:10AC80003CA817F051FB34493CA817F08DFB3CA8B9
:10AC90002946F6F7C9FC3CA817F046FBD6F8A430C5
:10ACA000012B00F080822D493CA817F07DFB00218C
:10ACB0003CA8F6F7B9FC3CA817F036FB22493CA8A3
:10ACC00017F072FB00213CA8F6F7AEFC3CA817F089
:10ACD0002BFB23493CA817F067FB00213CA8F6F7A3
:10ACE000A3FC3CA817F020FB19493CA817F05CFB1B
:10ACF00000213CA8F6F798FC3CA817F015FB154975
:10AD00003CA817F051FB00213CA8F6F78DFC3CA8AD
:10AD100017F00AFB10493CA817F046FB00213CA89D
:10AD2000F6F782FC3CA817F0FFFA484614F0EAF95F
:10AD30000024FFF771BA00BFC09EF87F689D020033
:10AD40002408FF1F049D020030890200189D0200A4
:10AD5000688B0200D09B0200448B0200409D0200E1
:10AD6000549D0200141CFF1F1821774816F0BEFCEA
:10AD7000764817F04BF98DF8244372B6DDEDC57AAD
:10AD80009DEDC47A67EEA87AF4EEC77AF1EE10FA78
:10AD9000CDEDC37A40F3FD81DDEDC77ACDEDC87A04
:10ADA00062B6A8A817F0A0F80024AD98A79413F0F5
:10ADB0008FFCAE9813F08CFCD6F88C30002B78D03A
:10ADC0008DF8904272B6DDEDA07A9DED9F7A67EE28
:10ADD000A87AF4EEC77ACDED9E7ADDEDA27AF1EE97
:10ADE00010FAD8BFF1EE677ACDEDA37A62B6DAF841
:10ADF00000303293329ADAF800303193319B9B1A4B
:10AE0000042BF8D983A817F06FF80025889882954D
:10AE100013F05EFC899813F05BFC294601220320A5
:10AE2000F5F73CFED6F8A430012B00F08B824849A0
:10AE30003CA817F0B9FA29463CA8F6F7F5FB3CA860
:10AE400017F072FA43493CA817F0AEFA29463CA81D
:10AE5000F6F7EAFB3CA817F067FA3F493CA817F061
:10AE6000A3FA29463CA8F6F7DFFB3CA817F05CFAEA
:10AE70003A493CA817F098FA29463CA8F6F7D4FBC3
:10AE80003CA817F051FA36493CA817F08DFA29462C
:10AE90003CA8F6F7C9FB3CA817F046FA31493CA894
:10AEA00017F082FA3CA82946F6F7BEFB3CA817F03B
:10AEB0003BFAD6F8A430012B00F082812A493CA845
:10AEC00017F072FA00213CA8F6F7AEFB3CA817F089
:10AED0002BFA20493CA817F067FA00213CA8F6F7A6
:10AEE000A3FB3CA817F020FA20493CA817F05CFA15
:10AEF00000213CA8F6F798FB3CA817F015FA174973
:10AF00003CA817F051FA00213CA8F6F78DFB3CA8AD
:10AF100017F00AFA12493CA817F046FA00213CA89B
:10AF2000F6F782FB3CA817F0FFF90E493CA817F092
:10AF30003BFA00213CA8F6F777FB3CA817F0F4F9A0
:10AF40000024FFF769B900BF849D02002408FF1F99
:10AF5000049D020030890200189D0200688B0200E7
:10AF6000D09B0200448B0200409D0200549D0200D1
:10AF700008219A489A4C16F0B9FB0521994816F019
:10AF8000B5FB0721984816F0B1FB984817F03EF83A
:10AF90003A6B012A00F0D281022A00F0BE8112B978
:10AFA000519A2260519571683268419896ED027A03
:10AFB000DFED8F6A8F4D02FB01F307EE903A06EE4C
:10AFC000100AF8EE677AB8EEC66A67EE877A8A4AA0
:10AFD0008A49106086EE277A3CA867EE267AC5ED8E
:10AFE000007A17F0E1F900213CA8F6F71DFB3CA818
:10AFF00017F09AF92220F6F795FC95ED000A00204B
:10B00000F6F734FC2220F6F78DFCFF20F6F78AFCD9
:10B01000FF20F6F787FCFF20F6F784FCDAF8002023
:10B020003B923B99DAF800303A933A9B744E5B1AA4
:10B03000042BF7D971493CA817F0B6F900213CA8B8
:10B04000F6F7F2FA3CA817F06FF92220F6F76AFC3F
:10B0500095ED000A0020F6F709FC2220F6F762FCC5
:10B06000FF20F6F75FFCFF20F6F75CFCFF20F6F709
:10B0700059FC326839923999DAF800303893389BA4
:10B080005F4E5B1A042BF7D994ED000A386B5D4DC7
:10B09000B8EEC00AF5F740FE5B4985ED000A3CA812
:10B0A00017F082F900213CA8F6F7BEFA3CA817F089
:10B0B0003BF92220F6F736FC95ED000A0020F6F762
:10B0C000D5FB2220F6F72EFCFF20F6F72BFCFF2005
:10B0D000F6F728FCFF20F6F725FC326837923799FF
:10B0E000DAF800303693369B454C5B1A042BF7D9BF
:10B0F00045493CA817F058F900213CA8F6F794FA06
:10B100003CA817F011F92220F6F70CFC95ED000A87
:10B110000020F6F7ABFB2220F6F704FCFF20F6F741
:10B1200001FCFF20F6F7FEFBFF20F6F7FBFB226891
:10B130003C923C99DAF800303593359B5B1A042B2E
:10B14000F8D90024314B41942146012203201C6090
:10B15000F5F7A4FC214620460122F5F79FFC0122C9
:10B1600021461046F5F79AFC214601220220F5F708
:10B1700095FC274BA593A5A8FDF7CCFF244B809306
:10B1800080A8FDF7C7FF0DF54B7DBDEC048BBDE836
:10B19000F08FDDEDC77AF1EE677AFFE5DDEDC77A76
:10B1A000F1EE677AEFE41B493CA817F0FDF80021A7
:10B1B0003CA8F6F739FA3CA817F0B6F81649AAE504
:10B1C00014493CA817F0F0F800213CA8F6F72CFA37
:10B1D0003CA817F0A9F81049A8E600BFA49C0200FB
:10B1E000B412FF1FD09C0200E89C02002408FF1F3D
:10B1F0000000B4439416FF1F6C15FF1F749B0200E0
:10B20000141CFF1FBC13FF1F849B0200F812FF1FBA
:10B21000288502002C9D02003089020000000000F9
:10B220000AD7233C012211460320F5F737FCDAF850
:10B23000002016921699DAF800301593159B5B1AC8
:10B24000042BF8D99A9A80AB02F10B0E03EB8E0E09
:10B2500003EB82024FF0000B40ABD362B7EE000A63
:10B26000012180A8CEF804B0CDF868B2FEF718F935
:10B270008DF890B272B65FED176ADDEDA07A9DEDA4
:10B280009F7A67EEA67AF4EEC77ACDED9E7ADDED71
:10B29000A27AF1EE10FAD8BFF1EE677ACDEDA37A7B
:10B2A00062B6DAF8002014921499DAF80030139399
:10B2B000139B5B1A092BF8D900228DF8902272B6E5
:10B2C0009DED037A5FED2A7A9DEDA06ADDED9F6A20
:10B2D000B8EEC77A67EE277A67EE867AF4EEE67AFA
:10B2E000CDED9E7ADDEDA27AF1EE10FAD8BFF1EE47
:10B2F000677ACDEDA37A62B60821B44816F0F6F964
:10B300000421B34816F0F2F90121B24816F0CEFE3E
:10B31000B04816F07BFEFEF7B6BE719A22607195BA
:10B3200041E6AD493CA817F03FF829463CA8F6F79E
:10B330007BF93CA816F0F8FFA849A5E4619A2260C1
:10B34000619530E6A4493CA817F02EF829463CA8A0
:10B35000F6F76AF93CA816F0E7FFA0499FE5009BC5
:10B360003969D7ED087A3A68019201FB03F170A8B8
:10B37000B8EEE78ACDF8C4B1D6F85080D6F84C9034
:10B38000DFF864A213F066F8019A114613F056F83C
:10B39000594613F09DF8DAF800200A920A99DAF873
:10B3A00000300993099B5B1A042BF8D98C4970A8CB
:10B3B00013F08EF8FEF7ECBD009BF968D7ED077A25
:10B3C000FA6A019201FB03F160A8B8EEE78ACDF8B2
:10B3D00084B1D6F83080D6F82C90DFF80CA213F0A8
:10B3E00039F8019A114613F029F8594613F070F80C
:10B3F000DAF8002008920899DAF800300793079BE2
:10B400005B1A042BF8D9764960A813F061F8FEF7AF
:10B41000BFBD71493CA816F0C7FF00213CA8F6F754
:10B4200003F93CA816F080FF6C49FFF7F0BA6D49AC
:10B430003CA816F0B9FF00213CA8F6F7F5F83CA8A7
:10B4400016F072FF6549FFF702BA07EE900AB8EEF0
:10B45000E78AD06128EE098AFFF783B807EE900AE1
:10B46000B8EEE78A106228EE098AFFF77AB8084634
:10B4700001220021F5F712FBFFF7ACB90A46084696
:10B480000021F5F70BFBFFF7A5B90122114658463D
:10B49000F5F704FBBF9ACDF8FCB2CAAB03EB820E02
:10B4A00050ABB7EE000A0121A5A84EF8683C4EF853
:10B4B00064BCFDF7F5FF8DF824B372B6DFED4B6A7F
:10B4C000DDEDC57A9DEDC47A67EEA67AF4EEC77A13
:10B4D000CDEDC37ADDEDC77AF1EE10FAD8BFF1EE0B
:10B4E000677ACDEDC87A62B6DAF800200E920E992E
:10B4F000DAF800300D930D9B5B1A092BF8D99FEDFC
:10B500003C7AD7ED067AF8EEE77A002267EE877A82
:10B510008DF8242372B6DDEDC56A9DEDC47A67EE21
:10B52000A67AF4EEC77ACDEDC37ADDEDC77AF1EEF7
:10B5300010FAD8BFF1EE677ACDEDC87A62B6FEF7A1
:10B5400090BD012258461146F5F7A8FABF9ACAAB3A
:10B5500002F10B0E03EB8E0E03EB82024FF0000B99
:10B5600070AB42F8683CB7EE000A0121A5A84EF87E
:10B5700090BCCDF8FCB2FDF793FF8DF824B372B602
:10B58000DFED1A6ADDEDC57A9DEDC47A67EEA67A25
:10B59000F4EEC77ACDEDC37ADDEDC77AF1EE10FA9D
:10B5A000D8BFF1EE677ACDEDC87A62B6DAF800203E
:10B5B00012921299DAF800301193119B5B1A092B41
:10B5C000F8D99FED0B7AD7ED087A9CE7A49C02008E
:10B5D000D89C02002408FF1FF09C02003089020062
:10B5E000C09EF87F2C9D0200141CFF1F000000006D
:10B5F0000AD7233C5A4659465846F5F74FFA0022D7
:10B600008DF8242372B65FED076ADDEDC57A9DEDF6
:10B61000C47A67EEA67AF4EEC77ACDEDC37ADDED93
:10B62000C77AF1EE10FAD8BFF1EE677ACDEDC87A9D
:10B6300062B6BF9ACAAB02F10B0103EB810103EBC7
:10B64000820260A8002342F8680CB7EE000A41F8B5
:10B65000903CA5A80121BF93FDF722FFDAF8002056
:10B6600010921099DAF800300F930F9B5B1A092B98
:10B67000F8D91FED217AD7ED077A44E72DE9F04F8D
:10B680008B002DED028B00F12C0808EB0305A8457B
:10B6900085B004460F46B0EE408A00F006819A104D
:10B6A000B2FA82F2C2F11F025200B64B294640465E
:10B6B000FDF762FEB34A29464046FDF7C5FDE66A3E
:10B6C000A665012F40F30B813069C64601225EF862
:10B6D000041F0B690132C0EB430397424B61F6DC58
:10B6E000A84500F02681D4F82C8004F13002D8F867
:10B6F000183011460DE00F68BF6983EAE37E87EAE0
:10B70000E77CAEEBE37EACEBE77C0431F445B8BFFD
:10B710003B468D42EFD1002BB8BF5B4207EE903A1B
:10B72000F8EEE77AD8F82430D6F81C80366A67EE4F
:10B73000887AFCEEE77A17EE907A06E01168496A9B
:10B740008B4202F1040228BF0B469542F6D11D46FA
:10B7500000B127B905B0BDEC028BBDE8F08F4FF00A
:10B76000000304F1040984F82830484612F09CFFD5
:10B770002062484612F098FF606212F069FF61692A
:10B7800004F1080012F01AFFA36D5A68DB68A26783
:10B79000C2EB0309B9F1000FB8BFC9F1000908FBFA
:10B7A00008F306FB06F09B4607FB07F2CDF8049072
:10B7B0004FF0000C00219146019BE367B0EB0B02B8
:10B7C00061EB0C03C4E926016D00104619465A4688
:10B7D00063464FF0000AC4E92423C4F88870C4F813
:10B7E00084602A460023C4F8A850C4F88080C4E9C5
:10B7F000289ACDE902BC19F04BF9019A801841EB67
:10B80000E271CB0FC01841F100014F104FEA300632
:10B81000002E43DBB24241DBDDE902BCB9EB0B0990
:10B820006AEB0C0A2A4600234846514619F030F9C3
:10B83000864240F38780C0EB4606C4F8B060C4F887
:10B84000AC00A368B8F1000F76D0002B7FD01A6847
:10B850004D498A4245D84D4AB2FBF8F21A60226A35
:10B860004B49E469002003250126DE60AA40986068
:10B870009D60086002F180434A6803F5603322440A
:10B880000D201A610860DA68502122F08002DA6027
:10B89000D96005B0BDEC028BBDE8F08F192013F024
:10B8A00045FC192013F042FCF8E7C66A86650129B9
:10B8B0003FF70AAF30693246B369756AD2F81C8027
:10B8C000166A002BB8BF5B4207EE903AB8EEE77AF3
:10B8D00067EE087AFCEEE77A17EE907A38E730697F
:10B8E00001E758682949B1FBF8F1121A914209D3CE
:10B8F0008A1A0026012503209E60DD601A60986088
:10B900001960ACE7606902680027012503269F6083
:10B910001268DD6019609E609047A368002B9ED17D
:10B920001C4A1268002A9AD0284602219047A36830
:10B9300095E73246E66ABFE7DBB19A6822F0020279
:10B940009A608CE7C4F8B060C4F8AC6079E7114A3B
:10B950000E4D1268B5FBF8F51AB10221012090478F
:10B96000A3680020012103229860D9601D609A60BD
:10B9700075E7084B1B687BB1022101209847A3683B
:10B98000DBE700BF6D0400007FA90300008793037D
:10B9900000800340DC1BFF1F4346CEE72DE9F04F3C
:10B9A0002DED028BEDB0804641F288320E463EA866
:10B9B0000521FDF765FB184B3E9305220023062168
:10B9C0000EA8599312F004FD142215211EA812F09E
:10B9D000FFFC124F172210212EA812F0F9FC35217E
:10B9E0000F48FC69BD6915F081FE0E4816F00EFB8C
:10B9F00041460C4816F05AFB0A4816F007FBB8F10E
:10BA0000050F00F23C87DFE818F003023D039F05B5
:10BA1000B70429060F0000BF44850200EC15FF1F84
:10BA2000B09D02002408FF1F0122114602203C6D38
:10BA3000D7F84CB0C54DF5F731F87B6B95ED0F0A93
:10BA4000002B41F04280F5F799F910EE100A18F03A
:10BA500075FBCDE900016A6AEB699FEDBD7A03FBD6
:10BA600002F308EE103AF8EEC87A4FF0000927EE1C
:10BA7000878A2EA8FDEEC87ACDF8BC9017EE901AF2
:10BA800012F0E8FC296A12F0D9FC8246304618F020
:10BA900043FBDDE9002318F0A5FB18F053FE014637
:10BAA000504612F015FD0D21AA4815F01FFE786CC6
:10BAB00018F044FB41EC100B0221A74816F000FBE4
:10BAC000A54816F0A3FA0A21A44815F00FFE4B462C
:10BAD0000A22F96BA04816F0A9FA9F4816F096FAC8
:10BAE0000B219F4815F002FE4B460A22B96B9A487B
:10BAF00016F09CFA984816F089FA0921994815F031
:10BB0000F5FDE86B18F01AFB41EC100B042192488C
:10BB100016F0D6FA904816F079FA0621924815F0F8
:10BB2000E5FD9DED000B02218B4816F0C9FA8A480D
:10BB300016F06CFA0A218D4815F0D8FDE96986489F
:10BB400016F0B4FA844816F061FA0E21884815F010
:10BB5000CDFD696A804816F0A9FA7F4816F056FABA
:10BB60000B21844815F0C2FD18EE100A18F0E6FA11
:10BB700041EC100B0221784816F0A2FA764816F034
:10BB800045FA06217C4815F0B1FD296A72484B46FA
:10BB90000A2216F04BFA704816F038FA589BCDF886
:10BBA00060916CA903F10B0201EB820201EB8303AC
:10BBB0002EAD43F88C5CB7EE000A01213EA842F896
:10BBC000B49CFFF75BFDE4B25FFA8BF520460121E0
:10BBD00013F092FA2846012113F08EFA409BDFF809
:10BBE000B8A1DFF8B891DFF8B8B143B3204613F03D
:10BBF00089FA10B9002E00F31886284613F082FA4D
:10BC000010B9002EC0F22986F6F73CFA002809DBAD
:10BC1000DAF80000F6F726FAC0B2532889F80000D7
:10BC200000F0FB85554A1368059305991368049342
:10BC3000049B5B1A012BF9D9409B002BD6D15049AC
:10BC40000AA816F0B1FB00210AA8F5F7EDFC0AA836
:10BC500016F06AFB4B490AA816F0A6FB00210AA8B9
:10BC6000F5F7E2FC0AA816F05FFB47490AA816F0B0
:10BC70009BFB00210AA8F5F7D7FC0AA816F054FB95
:10BC800040490AA816F090FB00210AA8F5F7CCFC61
:10BC90000AA816F049FB3D490AA816F085FB0021C9
:10BCA0000AA8F5F7C1FC0AA816F03EFB35490AA818
:10BCB00016F07AFB00210AA8F5F7B6FC0AA816F0E0
:10BCC00033FB33490AA816F06FFB00210AA8F5F7E9
:10BCD000ABFC0AA816F028FB2A490AA816F064FB58
:10BCE0000AA80021F5F7A0FC0AA816F01DFBB8F180
:10BCF000050F0ED8012404FA08F818F0240540F0C6
:10BD0000C18518F0120940F0D48518F0090F40F0F1
:10BD10003F86D7F8A430012B00F0A3851D490AA85F
:10BD200016F042FB00210AA8F5F77EFC0AA816F0DF
:10BD3000FBFA14490AA816F037FB00210AA8F5F708
:10BD400073FC0AA816F0F0FA2CE000BFAC15FF1F38
:10BD50000AD7233C289E02002408FF1F389E0200B9
:10BD6000449E0200509E02000CA202005C9E020053
:10BD7000E0B70200689E0200A0A10200141CFF1F91
:10BD8000989E020030890200AC9E0200C09E020014
:10BD9000D49E02001C9F02004807FF1FF413FF1FE0
:10BDA000EC16FF1FA1490AA816F0FEFA00210AA806
:10BDB000F5F73AFC0AA816F0B7FA9D490AA816F05A
:10BDC000F3FA00210AA8F5F72FFC0AA816F0ACFA3E
:10BDD00098490AA816F0E8FA00210AA8F5F724FC09
:10BDE0000AA816F0A1FA94490AA816F0DDFA002173
:10BDF0000AA8F5F719FC0AA816F096FA8F4B3E939D
:10BE00003EA8FDF787F96DB0BDEC028BBDE8F08F61
:10BE100012218B48FC69D7F818B08A4D15F066FCE2
:10BE20000F99894816F042F9874816F0EFF8012279
:10BE300011460020F4F732FE1121844815F056FC1B
:10BE40000F99814816F032F97F4816F0DFF82B6819
:10BE50000393039A2B680293029B9B1A052BF9D933
:10BE60007B4DD7ED057AD5ED0A6A3A69FB6886EE17
:10BE7000A77A03FB02F307EE903AF8EE677A67EED3
:10BE8000877A17EE900A18F059F9EA686B689FED07
:10BE9000717A03FB02F308EE103AF8EEC87A814695
:10BEA00027EE878A8A46FDEEC87A0EA817EE901A0A
:10BEB00012F0D0FAA9680EA812F0C0FA304618F0B5
:10BEC0002BF94A46534618F08DF918F03BFC014611
:10BED0000EA812F0FDFA17215F4815F007FC0F9924
:10BEE000594816F0E3F8584816F090F835215B48A9
:10BEF00015F0FCFB544816F089F80021524816F062
:10BF0000D5F8514816F082F80D21554815F0EEFB92
:10BF1000786918F013F941EC100B02214A4816F029
:10BF2000CFF8494816F072F80A214E4815F0DEFBAA
:10BF300000230A223969444816F078F8424816F07E
:10BF400065F80B21484815F0D1FB00230A22F96857
:10BF50003D4816F06BF83C4816F058F80921434864
:10BF600015F0C4FBA86A18F0E9F841EC100B0221A7
:10BF7000354816F0A5F8344816F048F806213C4834
:10BF800015F0B4FB4AEC109B02212F4816F098F8EC
:10BF90002D4816F03BF80A21364815F0A7FB6968D2
:10BFA000294816F083F8284816F030F80E21324858
:10BFB00015F09CFBE968244816F078F8224816F042
:10BFC00025F80B212D4815F091FB18EE100A18F0FA
:10BFD000B5F841EC100B02211B4816F071F81A4815
:10BFE00016F014F80621264815F080FBA9681648BB
:10BFF00000230A2216F01AF8134816F007F8589B87
:10C000006CA903F10B0201EB820E01EB8303002507
:10C010000EAA43F88C2CB7EE000A01213EA84EF878
:10C02000B45C5895FFF72AFBCDE500BF309F0200B6
:10C03000688B0200D09B0200448B02004485020002
:10C04000E89D0200141CFF1F2408FF1FFC9D020036
:10C05000AC15FF1F0AD7233C109E0200B09D0200C2
:10C06000289E0200389E0200449E0200509E02005C
:10C070000CA202005C9E0200E0B70200689E020073
:10C08000A0A102000122114610463C6BD7F82CB04B
:10C09000DFF8E092AA4DF4F701FD0721A94815F059
:10C0A00025FB00230A22D7F89010A74815F0BEFF01
:10C0B000A54815F0ABFFD7F890A0BAF1000F40F0FB
:10C0C0000E85D5ED0B6AD9ED0A7AD9F82420D9F876
:10C0D000203086EEA77A03FB02F307EE903AF8EEE3
:10C0E000677A67EE877A17EE900A18F027F8CDE99D
:10C0F00000010D21954815F0F9FAD9F8280018F03B
:10C100001DF841EC100B02218F4815F0D9FF8E4825
:10C1100015F07CFF0A218E4815F0E8FA53460A22F2
:10C12000D9F82410884815F081FF874815F06EFF74
:10C130000B21884815F0DAFA53460A22D9F8201064
:10C14000814815F073FF804815F060FF092182488F
:10C1500015F0CCFAE86A17F0F1FF41EC100B022160
:10C16000794815F0ADFF784815F050FF06217B485F
:10C1700015F0BCFA9DED000B0221734815F0A0FFED
:10C18000714815F043FF0A21754815F0AFFA296987
:10C190006D4815F08BFF6C4815F038FF0E21714883
:10C1A00015F0A4FAA969684815F080FF664815F0F3
:10C1B0002DFF06216C4815F099FA534669696248CB
:10C1C0000A2215F033FF604815F020FFAA692B6999
:10C1D0009FED667A03FB02F308EE103AF8EEC87A98
:10C1E0004FF0000927EE878A1EA8FDEEC87ACDF829
:10C1F0007C9017EE901A12F02DF9696912F01EF971
:10C200008246304617F088FFDDE9002317F0EAFF89
:10C2100018F098FA0146504612F05AF90D214B4891
:10C2200015F064FAB86A17F089FF41EC100B02218F
:10C23000454815F045FF444815F0E8FE0A214448FA
:10C2400015F054FA4B460A22796A3F4815F0EEFE83
:10C250003D4815F0DBFE0B213E4815F047FA4B46F2
:10C260000A22396A384815F0E1FE374815F0CEFE4B
:10C270000921394815F03AFAE86A17F05FFF41ECF6
:10C28000100B0221304815F01BFF2F4815F0BEFEA1
:10C290000621324815F02AFA9DED000B02212A48AA
:10C2A00015F00EFF284815F0B1FE0A212C4815F0B4
:10C2B0001DFA2969244815F0F9FE234815F0A6FE59
:10C2C0000E21284815F012FAA9691F4815F0EEFE54
:10C2D0001D4815F09BFE0B21254815F007FA18EEB6
:10C2E000100A17F02BFF41EC100B0221164815F035
:10C2F000E7FE154815F08AFE06211B4815F0F6F9F1
:10C300004B46696910480A2215F090FE0E4815F058
:10C310007DFE589BCDF860916CA903F10B0201EBF7
:10C32000820201EB83031EAD43F88C5CB7EE000A7A
:10C3300001213EA842F8B49CFFF7A0F943E400BFF6
:10C34000AC15FF1F749E02002408FF1F289E0200E8
:10C35000389E0200449E0200509E02000CA2020081
:10C360005C9E0200E0B70200A0A102000AD7233CB5
:10C37000689E0200EC15FF1FAB4DFC69D7F818B0A2
:10C38000012211460020F4F789FBD5ED0D6AD7EDA7
:10C39000057A3A69FB6886EEA77A03FB02F34FF051
:10C3A0000009CDF83C9007EE903AF8EE677A67EE18
:10C3B000877A17EE900A17F0C1FEEA686B689FED66
:10C3C0009B7A03FB02F308EE103AF8EEC87A0EAB44
:10C3D00027EE878ACDE90001FDEEC87A184617EEF0
:10C3E000901A12F037F8A96812F028F88246304601
:10C3F00017F092FEDDE9002317F0F4FE18F0A2F921
:10C400000146504612F064F83521894815F06EF95E
:10C41000884815F0FBFD0321864815F047FE854846
:10C4200015F0F4FD0D21844815F060F9786917F0D6
:10C4300085FE41EC100B02217E4815F041FE7D483F
:10C4400015F0E4FD0A217D4815F050F94B460A220B
:10C450003969784815F0EAFD764815F0D7FD0B21CB
:10C46000774815F043F94B460A22F968714815F0F0
:10C47000DDFD704815F0CAFD0921724815F036F946
:10C48000686B17F05BFE41EC100B0221694815F058
:10C4900017FE684815F0BAFD06216B4815F026F91D
:10C4A0009DED000B0221634815F00AFE614815F06E
:10C4B000ADFD0A21654815F019F969685D4815F068
:10C4C000F5FD5C4815F0A2FD0E21614815F00EF94E
:10C4D000E968584815F0EAFD564815F097FD0B211C
:10C4E0005C4815F003F918EE100A17F027FE41EC2E
:10C4F000100B02214F4815F0E3FD4E4815F086FD64
:10C500000621554815F0F2F84B46A96849480A2219
:10C5100015F08CFD474815F079FD589BCDF86091DA
:10C520006CA903F10B0201EB820201EB83030EAD58
:10C5300043F88C5CB7EE000A01213EA842F8B49C97
:10C54000FFF79CF8FFF73FBB0122114602203C6D2C
:10C55000D7F84CB0344DF4F7A1FA7B6B95ED0C0A8B
:10C56000002B40F01A83F4F709FC10EE100A17F0C4
:10C57000E5FDCDE900016A6AEB699FED2C7A03FBCA
:10C5800002F308EE103AF8EEC87A4FF0000927EEF1
:10C59000878A2EA8FDEEC87ACDF8BC9017EE901AC7
:10C5A00011F058FF296A11F049FF8246304617F012
:10C5B000B3FDDDE9002317F015FE18F0C3F80146BE
:10C5C000504611F085FF0D211B4815F08FF8786C4F
:10C5D00017F0B4FD41EC100B0221164815F070FD68
:10C5E000144815F013FD0A21144815F07FF84B4646
:10C5F0000A22F96B0F4815F019FD0E4815F006FDDB
:10C600000B210F4815F072F84B460A22B96B094806
:10C6100015F00CFD074815F0F9FC0921094815F043
:10C6200065F8286BFFF76EBAAC15FF1F0AD7233CDD
:10C63000B09D02002408FF1F289E0200389E0200C1
:10C64000449E0200509E02000CA202005C9E02006A
:10C65000E0B70200689E0200A0A10200012211467C
:10C6600010463C6BD7F82CB0DFF82093B04DF4F7B0
:10C6700015FA0721AF4815F039F800230A22D7F838
:10C680009010AD4815F0D2FCAB4815F0BFFCD7F8C0
:10C690009030002B40F04381D9ED0A7AD5ED0E6A37
:10C6A000D9F82420D9F8203086EEA77A03FB02F3CC
:10C6B0004FF0000907EE903AF8EE677A67EE877A56
:10C6C00017EE900A17F03AFDAA692B699FED9B7A45
:10C6D000CDF87C9003FB02F308EE103AF8EEC87A2E
:10C6E000CDE9000127EE878A1EA8FDEEC87A17EE75
:10C6F000901A11F0AFFE696911F0A0FE8246304633
:10C7000017F00AFDDDE9002317F06CFD18F01AF8A8
:10C710000146504611F0DCFE0D21894814F0E6FF79
:10C72000B86A17F00BFD41EC100B0221824815F09E
:10C73000C7FC814815F06AFC0A21824814F0D6FF34
:10C740004B460A22796A7C4815F070FC7A4815F04D
:10C750005DFC0B217C4814F0C9FF4B460A22396A64
:10C76000754815F063FC744815F050FC09217748B2
:10C7700014F0BCFFA86B17F0E1FC41EC100B022198
:10C780006D4815F09DFC6C4815F040FC0621704882
:10C7900014F0ACFF9DED000B0221674815F090FCF2
:10C7A000654815F033FC0A216A4814F09FFF296997
:10C7B000614815F07BFC604815F028FC0E216648A6
:10C7C00014F094FFA9695C4815F070FC5A4815F004
:10C7D0001DFC0B21614814F089FF18EE100A17F0B8
:10C7E000ADFC41EC100B0221534815F069FC524896
:10C7F00015F00CFC06215A4814F078FF69694E4880
:10C800004B460A2215F012FC4B4815F0FFFB0122A3
:10C8100011461046F4F742F97BE53EA8FCF722FCEE
:10C8200001238BF80030FFF7FDB900904D482E2111
:10C8300014F05CFF404815F0E9FB41A815F054FBEB
:10C84000009B4698409311F043FF479811F040FF3A
:10C85000454B01221A70FFF7F2B900902E21434890
:10C86000E6E743490AA815F09FFD00210AA8F4F75E
:10C87000DBFE0AA815F058FD3E49FFF7B5BAAB46F6
:10C88000FFF7A1B93C4D2F9B2A683C48134409216E
:10C890002B6014F02BFF2968274815F007FC264869
:10C8A00015F0B4FB224600210220F4F7F7F8FFF759
:10C8B00030BA3349304E0AA815F076FD29460AA849
:10C8C000F4F7B2FE0AA815F02FFD2220F5F72AF89A
:10C8D0002C4B284693ED000AF4F7C8FF2A490AA812
:10C8E00015F062FD29460AA8F4F79EFE0AA815F085
:10C8F0001BFD32681F9B214813440921336014F04B
:10C90000F5FE31680C4815F0D1FB0B4815F07EFBA5
:10C91000224629462046F4F7C1F8FFF7FAB9D9EDC7
:10C92000277AD5ED0E6AD9F89820D9F89430BBE66D
:10C93000AC15FF1F749E02002408FF1F0AD7233C7A
:10C94000289E0200389E0200449E0200509E020073
:10C950000CA202005C9E0200E0B70200689E02008A
:10C96000A0A10200449F0200EC16FF1F749F02006A
:10C97000089F020030890200B412FF1FFC9E0200D3
:10C98000E89E02002019FF1F448B0200EC15FF1FD8
:10C990008649874C874E884D0AA815F005FD494603
:10C9A0000AA8F4F741FE0AA815F0BEFC2220F4F70D
:10C9B000B9FF824B484693ED000AF4F757FF8049D0
:10C9C0000AA815F0F1FC49460AA8F4F72DFE0AA8BA
:10C9D00015F0AAFC22680F9B7A48134409212360B2
:10C9E00014F084FE2168784815F060FB764815F055
:10C9F0000DFB94ED007A3A69FB68D7ED056A73493F
:10CA0000F8EEC77A03FB02F327EEA67A07EE903A18
:10CA1000F8EE677A0AA8C7EE276AC6ED006A15F035
:10CA2000C3FC49460AA8F4F7FFFD0AA815F07CFCF0
:10CA30002220F4F777FF96ED000A4846F4F716FF38
:10CA40002220F4F76FFFFF20F4F76CFFFF20F4F7CC
:10CA500069FFFF20F4F766FF2B680993099A2B689A
:10CA60000893089B544C9B1A042BF8D957490AA8E1
:10CA700015F09AFC00210AA8F4F7D6FD0AA815F0D3
:10CA800053FC2220F4F74EFF96ED000A0020F4F745
:10CA9000EDFE2220F4F746FFFF20F4F743FFFF20CE
:10CAA000F4F740FFFF20F4F73DFF23680793079A50
:10CAB0002B680693069B9B1A042BF9D90021084684
:10CAC0000122F3F7EBFFFFF724B9F4F7F1F910EEC9
:10CAD000100A17F033FBCDE90001FEF7BCBFD5ED1E
:10CAE0000B6AD9ED277AD9F89820D9F8943086EED8
:10CAF000A77A03FB02F307EE903AF8EE677A67EE47
:10CB0000877A17EE900A17F019FBCDE9000118217A
:10CB10002F4814F0EBFD2C4815F078FA0D212D4824
:10CB200014F0E4FDD9F89C0017F008FB41EC100B61
:10CB30000221254815F0C4FA234815F067FA0A21A6
:10CB4000254814F0D3FD00230A22D9F898101E4876
:10CB500015F06CFA1C4815F059FA0B211F4814F017
:10CB6000C5FD00230A22D9F89410174815F05EFA83
:10CB7000154815F04BFA0921194814F0B7FDE86A79
:10CB800017F0DCFA41EC100B02210F4815F098FA6F
:10CB90000D4815F03BFAFFF719BBF4F789F910EED1
:10CBA000100A17F0CBFACDE90001E4E4E89E020098
:10CBB000B412FF1FBC13FF1F141CFF1F2419FF1FFB
:10CBC000448B0200FC9E02002408FF1F849B02008D
:10CBD0007C9E0200289E0200389E0200449E0200B5
:10CBE000509E02002DE9F04FC9B041F28832052174
:10CBF00006460DF128081AA8DFF83890DFF838A0AB
:10CC0000FCF73EFA0024404602220321CDF868A03A
:10CC1000359411F0DDFBD9F800300B94013B042B67
:10CC200000F24382DFE813F01D02210225022902EF
:10CC30000A0000BF7415FF1F44850200C348C44C9E
:10CC4000082114F053FD0521C24814F04FFDA168DE
:10CC5000C14815F02BFAC04815F0D8F9A06817F0B4
:10CC60005BFA41EC100B15F0ABFF51EC100B17F019
:10CC700069FD019006FB00FB0A21B848B84DB94C8C
:10CC8000B94F14F033FD3146B348B84E15F00EFAE3
:10CC9000B14815F0BBF90C21B54814F027FD00236D
:10CCA0000A222968AC4815F0C1F9AB4815F0AEF975
:10CCB0000B21B04814F01AFDA86817F03FFA41ECB8
:10CCC000100B0221A44815F0FBF9A34815F09EF9BA
:10CCD0000B21A94814F00AFD00230A2269689E4826
:10CCE00015F0A4F99C4815F091F90C21A34814F013
:10CCF000FDFC00230A22D5F88410974815F096F918
:10CD0000954815F083F913219D4814F0EFFC00239A
:10CD10000A22D5F88810904815F088F98E4815F049
:10CD200075F90E21974814F0E1FC01998A4815F035
:10CD3000BDF9894815F06AF9D9F80410404611F098
:10CD400089FBD9F80C10404611F078FB4046594653
:10CD500011F0BEFB10218C4814F0C8FC59467E48E7
:10CD600015F0A4F97C4815F051F901221146032071
:10CD7000F3F794FE349B48A903F10B0201EB820206
:10CD800001EB83034FF0000E43F88C8CB7EE000AE2
:10CD900001211AA842F8B4ECCDF8D0E0FEF76EFC01
:10CDA000DDF87080B8F1000F22D023680393039A56
:10CDB00023680293029B9B1A042BF9D9F5F762F9B9
:10CDC000002807DB3868F5F74DF9C0B253283070FA
:10CDD00000F0578123680593059A23680493049B08
:10CDE0009B1A092BF9D9DDF87080B8F1000FDCD15E
:10CDF0006649674E674C06A815F0D6FA414606A864
:10CE0000F4F712FC06A815F08FFA634906A815F08E
:10CE1000CBFA414606A8F4F707FC06A815F084FAF9
:10CE20005E4906A815F0C0FA414606A8F4F7FCFBD7
:10CE300006A815F079FA584906A815F0B5FA414642
:10CE400006A8F4F7F1FB06A815F06EFA544906A8F7
:10CE500015F0AAFA414606A8F4F7E6FB06A815F075
:10CE600063FA4D4906A815F09FFA414606A8F4F763
:10CE7000DBFB06A815F058FA4A4906A815F094FA03
:10CE8000414606A8F4F7D0FB06A815F04DFA424932
:10CE900006A815F089FA414606A8F4F7C5FB06A8CE
:10CEA00015F042FA69682B680B9A95ED027ADFED6E
:10CEB0003E6A03FB01F307EE903A06EE102AF8EE05
:10CEC000677AB8EEC66A67EE877A3368374986EEC6
:10CED000277A0A6006A81A443549326067EE267A36
:10CEE000C4ED007A15F060FA414606A8F4F79CFB01
:10CEF00006A815F019FA2220F4F714FD94ED000AA3
:10CF00004046F4F7B3FC2B4906A815F04DFA41460C
:10CF100006A8F4F789FB06A815F006FA0122414697
:10CF20000320F3F7BBFDD5F8A430012B00F0B0804F
:10CF3000214906A815F038FA414606A8F4F774FB13
:10CF400006A815F0F1F9144906A837E0DC9F0200A5
:10CF50005017FF1FB09F02002408FF1F0CBA0200E9
:10CF6000EC15FF1F141CFF1F4807FF1FF413FF1FC2
:10CF7000E89F0200F89F020004A0020010A0020037
:10CF800020A0020034A0020044A0020058A0020029
:10CF90006418FF1F9416FF1F308902006CA0020066
:10CFA00080A0020094A002000000B4436C15FF1F93
:10CFB000749B0200448B0200C0A0020015F0F4F93B
:10CFC000414606A8F4F730FB06A815F0ADF939493B
:10CFD00006A815F0E9F9414606A8F4F725FB06A8CE
:10CFE00015F0A2F9344906A815F0DEF9414606A865
:10CFF000F4F71AFB06A815F097F9304906A815F0C2
:10D00000D3F9414606A8F4F70FFB06A815F08CF9F2
:10D010002B4906A815F0C8F9414606A8F4F704FB09
:10D0200006A815F081F9274906A815F0BDF90021D9
:10D0300006A8F4F7F9FA06A815F076F9224906A829
:10D0400015F0B2F9002106A8F4F7EEFA06A815F0DB
:10D050006BF91AA8CDF868A0FCF75CF849B0BDE8F8
:10D06000F08F082119481A4CEBE5082119481A4C91
:10D07000E7E5082119481A4CE3E5082119481A4C3C
:10D08000DFE51AA8FBF7EEFF184B01221A70A1E6A4
:10D09000174906A815F088F9414606A8F4F7C4FA1E
:10D0A00006A815F041F90849B3E74FF0000BCDF899
:10D0B00004B0E1E5D8A00200688B0200D09B02001A
:10D0C000448B0200ECA0020030890200A49F020001
:10D0D000F016FF1FB89F02000817FF1FC49F020031
:10D0E0002017FF1FD09F02003817FF1FEC16FF1FED
:10D0F000A8A002002DE9F04FCC4FDFF88C93BB6C59
:10D10000CB4AD9F81C40D9F818602DED028BE5B058
:10D110000025012B0590156000F0A485C0F0648502
:10D12000022B00F00584A8460395AB4604950195B3
:10D13000AA46E4B220460121F6B211F0DDFF3046E6
:10D14000012111F0D9FF41F28832052136A8FBF701
:10D1500097FF0025B74B36930222032116A851955D
:10D1600011F036F95146019ADFF8C0A226A811F055
:10D170002FF93A683B699FEDB07A03FB02F307EEA3
:10D18000903AF8EEE77A16A867EE877AFDEEE77A2E
:10D1900017EE901A11F05EF9396A11F04FF9FB6C35
:10D1A0001795002B00F0AC84012B40F0EA849AED37
:10D1B0000F6A9FEDA27AD9ED027ADAF848009AED6B
:10D1C0000E0ADAF83050C6EE076A99E80C0003FB45
:10D1D00002F3043507EE103AB8EE477A9DED056A82
:10D1E00067EE277AB8EEC68A67EEA67A67EE887A87
:10D1F000FDEEE77ACDED017AF3F78AFEDAF830300A
:10D200005B0007EE903AF8EEE77A6B0080EE270AB3
:10D21000029320EE088AFDEEC87A17EE905A3B2161
:10D220008748DFF808A214F061FA864814F0EEFE91
:10D230000D21854814F05AFA0199824814F036FFFE
:10D24000804814F0E3FE1121804814F04FFA804B1F
:10D250007C48196814F02AFF7A4814F0D7FE0A2196
:10D260007C4814F043FA2946764814F01FFF7548AD
:10D2700014F0CCFE3B21724814F038FA714814F0D7
:10D28000C5FE039926A811F0E5F8414611F0D6F83D
:10D290004FF000080E217048CDF89C8014F026FA5B
:10D2A0003968684814F002FF664814F0AFFE142194
:10D2B0006A4814F01BFA3969624814F0F7FE6148B5
:10D2C00014F0A4FE0D21664814F010FA43460A2219
:10D2D000396A5C4814F0AAFE5A4814F097FE1321EC
:10D2E000604814F003FA43460A22D9F80010554862
:10D2F00014F09CFE534814F089FE11215A4814F092
:10D30000F5F943460A22D9F804104E4814F08EFE6F
:10D310004C4814F07BFE1221544814F0E7F9D9F878
:10D32000080016F00BFF41EC100B0221454814F0E9
:10D33000C7FE444814F06AFEFB6C002B00F0B1837A
:10D34000012B2DD110214A4814F0D0F9DAF83C0015
:10D3500016F0F4FE41EC100B02213A4814F0B0FE36
:10D36000384814F053FE0F21424814F0BFF9DAF8A0
:10D37000380016F0E3FE41EC100B0221314814F0A6
:10D380009FFE304814F042FE0C213B4814F0AEF9E9
:10D39000DAF830102B4814F089FE2A4814F036FED3
:10D3A0000D21294814F0A2F90199264814F07EFEB7
:10D3B000244814F02BFE0A21264814F097F9294638
:10D3C000204814F073FE1F4814F020FE0B212B4858
:10D3D00014F08CF903991B4814F068FE194814F0F6
:10D3E00015FE1121264814F081F95946154814F00C
:10D3F0005DFE144814F00AFE0A21224814F076F962
:10D400000499104814F052FE0E4814F0FFFD01225A
:10D4100003201146F3F742FBB86C012800F0BC83EF
:10D42000C0F0B48302283CD130E000BF8014FF1F5D
:10D43000F812FF1F448502000AD7233C0000B443C2
:10D44000A8A102002408FF1FE4A10200F4A1020029
:10D45000B412FF1F08A2020014A2020024A20200BC
:10D460003CA20200FCA802001CA902003CA9020088
:10D470008CA20200A0A20200B0A2020074A10200CD
:10D4800084A102009CA10200EC15FF1F012211469D
:10D49000F3F704FB23212E4814F028F92D4814F04B
:10D4A000B5FD029B042B40F38F80DFF8B0804FF076
:10D4B000040A0AF0030B0521274814F017F959460E
:10D4C000244814F0F3FD234814F0A0FDBBF1020F33
:10D4D00000F08882BBF1030F00F0B482BBF1010FB2
:10D4E00000F0B082D7F84CB0BBF1000F00F04184DF
:10D4F000BBF1010F41D1019916A810F0E9FF509A34
:10D5000064AB02F10B0E03EB8E0E03EB820216A846
:10D51000002342F88C0C59464EF8B43CB7EE000A92
:10D5200036A85093FEF7AAF8D8F800300993099A64
:10D53000D8F800300893089B9B1A042BF8D9389B25
:10D540002046F3B9029B0AF1010A9A45B1D13BE0AA
:10D55000C0A202002408FF1FE4A20200141CFF1F47
:10D56000C14814F0C3F8C14814F050FD002D1DDC73
:10D57000F4F788FD002800F31D82389B2046002B1D
:10D58000E0D011F0BFFD2E2183460028E8D03046C0
:10D5900011F0B8FD83460028EAD12E21B44814F0DA
:10D5A000A5F8B24814F032FD002DE1DA39A814F0E4
:10D5B0009BFC3E98CDF8E0B011F08AF83F9811F04E
:10D5C00087F8AC4B01221A70D9F80410D9F8003052
:10D5D0002798179A99ED027ADFEDA76AA74CA84E13
:10D5E000A84D226003FB01F307EE903A06EE102AE5
:10D5F000F8EE677AB8EEC66A67EE877A07EE100A29
:10D60000B8EEC70A86EE277A28609F4D67EE267A25
:10D61000C6ED007AF2F79CFF9C4985ED000A12A83E
:10D6200014F0C2FE002112A8F3F7FEFF12A814F0B6
:10D630007BFE2220F4F776F996ED000A0020F4F73D
:10D6400015F9934912A814F0AFFE002112A8F3F7C0
:10D65000EBFF12A814F068FE8E4912A814F0A4FE85
:10D66000002112A8F3F7E0FF12A814F05DFE2220BB
:10D67000F4F758F995ED000A0020F4F7F7F884491B
:10D6800012A814F091FE002112A8F3F7CDFF12A802
:10D6900014F04AFE804912A814F086FE002112A858
:10D6A000F3F7C2FF12A814F03FFE7C4912A814F051
:10D6B0007BFE002112A8F3F7B7FF12A814F034FE86
:10D6C000774912A814F070FE002112A8F3F7ACFFFE
:10D6D00012A814F029FE714912A814F065FE002169
:10D6E00012A8F3F7A1FF12A814F01EFE6D4912A8AC
:10D6F00014F05AFE002112A8F3F796FF12A814F0B6
:10D7000013FE664912A814F04FFE002112A8F3F789
:10D710008BFF12A814F008FE634912A814F044FE0F
:10D72000002112A8F3F780FF12A814F0FDFD5B4959
:10D7300012A814F039FE002112A8F3F775FF12A801
:10D7400014F0F2FD0821594813F0D0FF2168474832
:10D7500014F0ACFC454814F059FC0521544813F072
:10D76000C5FF484B4148196814F0A0FC3F4814F02D
:10D770004DFC504B22681A60002101220320F3F770
:10D780008DF9002108460122F3F788F9012210469D
:10D790000021F3F783F9012200210220F3F77EF93B
:10D7A000D9F8A430012B00F09F82434912A814F04D
:10D7B000FBFD002112A8F3F737FF12A814F0B4FD07
:10D7C000364912A814F0F0FD002112A8F3F72CFF3F
:10D7D00012A814F0A9FD394912A814F0E5FD0021A2
:10D7E00012A8F3F721FF12A814F09EFD344912A8E5
:10D7F00014F0DAFD002112A8F3F716FF12A814F0B6
:10D8000093FD304912A814F0CFFD002112A8F3F7C0
:10D810000BFF12A814F088FD1D4912A814F0C4FDD6
:10D82000002112A8F3F700FF12A814F07DFD26498D
:10D8300012A814F0B9FD002112A8F3F7F5FE12A802
:10D8400014F072FD154912A814F0AEFD002112A8C3
:10D85000F3F7EAFE12A814F067FD1C4912A814F0B1
:10D86000A3FD002112A833E0449F02002408FF1FFB
:10D87000749F0200EC16FF1F0000B4436418FF1FE2
:10D880009416FF1FB412FF1FBC13FF1F749B0200EE
:10D89000448B0200849B020008A30200308902002E
:10D8A0001CA3020030A3020044A3020010A6020041
:10D8B00000A202006C15FF1F80A3020094A30200C7
:10D8C000688B0200D09B0200A8A30200BCA3020048
:10D8D000F3F7AAFE12A814F027FDB24912A814F01B
:10D8E00063FD002112A8F3F79FFE12A814F01CFD9F
:10D8F000AD4912A814F058FD002112A8F3F794FEC8
:10D9000012A814F011FDA94912A814F04DFD002130
:10D9100012A8F3F789FE12A814F006FDA44B369363
:10D9200036A8FBF7F7FB65B0BDEC028BBDE8F08FC6
:10D93000D7F81CB0FB689FEDAB7AD7F82C809D48D8
:10D94000D9F85040D9F84C60CDF8108003FB0BF3A8
:10D9500007EE903AF8EEE77A0F2167EE877A4FF0FC
:10D96000100AFDEEE77ACDED037A13F0BFFEF968F9
:10D97000914814F09BFB904814F048FB15218F4808
:10D9800013F0B4FEF9698C4814F090FB8A4814F047
:10D990003DFB0E218A4813F0A9FE2B460A22F96AA4
:10D9A000854814F043FB844814F030FB172301939F
:10D9B000FFF7BFBB834B1868F4F754FB824BC0B230
:10D9C000532818707FF4D9AD1A21804813F08EFEC9
:10D9D000794814F01BFB36A8FBF744FB7C4B012273
:10D9E0001A70F1E5D7F84CB0BBF1000F00F0E481FC
:10D9F000BBF1010F7FF4C1AD019B16A8594210F095
:10DA000067FD509A64AB02F10B0E03EB8E0E03EB35
:10DA1000820216A8002342F88C0C59464EF8B43CFA
:10DA2000B7EE000A36A85093FDF728FED8F800306C
:10DA30001193119AD8F800301093109B9B1A042B65
:10DA4000F8D99AE5D7F84CB0BBF1000F00F06F8120
:10DA5000BBF1010F7FF491AD294626A810F038FDE7
:10DA6000509A64AB02F10B0E03EB8E0E03EB8202B5
:10DA700026A8002342F88C0C59464EF8B43CB7EE69
:10DA8000000A36A85093FDF7F9FDD8F800300D9341
:10DA90000D9AD8F800300C930C9B9B1A042BF8D9E4
:10DAA0006BE50F214B4813F021FEDAF8440016F025
:10DAB00045FB41EC100B02213F4814F001FB3E48AE
:10DAC00014F0A4FA1C21444813F010FEDAF84000C8
:10DAD00016F034FB41EC100B0221374814F0F0FA39
:10DAE000354814F093FA0D213C4813F0FFFDDAF8A5
:10DAF0003410314814F0DAFA2F4814F087FA4FE462
:10DB0000DAF83420DAED116ADFED355A99ED026A60
:10DB1000520007EE902AB8EEE77A99E80A0086EEFE
:10DB2000875A03FB01F307EE903AC5EE256A02F12E
:10DB300008030293B8EE677A67EE067A9DED057AE0
:10DB400067EEA67AB8EEC78A67EE887A17EE900A73
:10DB500016F0F4FA41EC100B15F032F851EC100B02
:10DB600016F0F0FD9AED100A0190DAF84800F3F78C
:10DB7000CFF928EE000AFDEEC07A17EE905AFFF7B3
:10DB80004EBB082301950293FFF749BB01221146C2
:10DB90000020F2F783FF84E402460146F2F77EFF9D
:10DBA0007FE400BF688B0200D09B0200448B020020
:10DBB0004485020070A102002408FF1F80A102001A
:10DBC00098A102004807FF1FF413FF1FECA20200F8
:10DBD000EC16FF1F4CA202005CA202007CA2020015
:10DBE0000000B4430AD7233CD7F814B07B681FED7C
:10DBF000037AD7F824808248CDF8108003FB0BF31A
:10DC000007EE903AF8EEE77A0F2167EE877A4FF049
:10DC1000060AFDEEE77ACDED037A13F067FD796829
:10DC2000784814F043FA774814F0F0F91521764853
:10DC300013F05CFD7969734814F038FA714814F0F8
:10DC4000E5F90E21714813F051FD2B460A22796A3D
:10DC50006C4814F0EBF96B4814F0D8F905230193E4
:10DC6000FFF767BAD7F818B0BB689FED697AD7F8A5
:10DC700028806848D9F83040D9F82C60CDF8108059
:10DC800003FB0BF307EE903AF8EEE77A0F2167EE0D
:10DC9000877A4FF0150AFDEEE77ACDED037A13F09F
:10DCA00025FDB968574814F001FA564814F0AEF94A
:10DCB0001521594813F01AFDB969524814F0F6F9C4
:10DCC000504814F0A3F90E21544813F00FFD2B46D1
:10DCD0000A22B96A4B4814F0A9F94A4814F096F997
:10DCE00014230193FFF725BA4D4912A814F05CFBE9
:10DCF000002112A8F3F798FC12A814F015FB49496B
:10DD000012A814F051FB002112A8F3F78DFC12A801
:10DD100014F00AFB444912A814F046FB002112A893
:10DD2000F3F782FC12A814F0FFFA3E49ECE50199E2
:10DD300016A810F0CDFB509ACDF840B164AB03EBC0
:10DD40008200024616AB40F88C3CB7EE000A42F85F
:10DD500088BC012136A8FDF791FCD8F800300B9360
:10DD60000B9AD8F800300A930A9B9B1A042BF8D917
:10DD700003E4294626A810F0ABFB509ACDF840B139
:10DD800064AB03EB8200024626AB40F88C3CB7EE56
:10DD9000000A42F888BC012136A8FDF76FFCD8F8CC
:10DDA00000300793079AD8F800300693069B9B1A19
:10DDB000042BF8D9FFF7E1BB694226A810F088FBD5
:10DDC000509ACDF840B164AB03EB8200024626AB1B
:10DDD00040F88C3CB7EE000A42F888BC012136A816
:10DDE000FDF74CFCD8F800300F930F9AD8F80030AC
:10DDF0000E930E9B9B1A042BF8D9FFF7BEBB00BFF6
:10DE000000A102002408FF1F10A1020028A10200A7
:10DE10000AD7233C38A1020048A1020060A10200F9
:10DE200058A30200308902006CA302002DE9F04FD4
:10DE30002DED088BCBB0D14CDFF8A0930090884635
:10DE400008A8CF49F0EE408AB0EE60BA14F0ACFA00
:10DE5000E569A669D9F80070B8F1000F07D1012F64
:10DE600000F0A082C0F01D82022F00F01A82302143
:10DE7000C44813F03BFC3946C34814F017F9C248B4
:10DE800014F0C4F81721C14813F030FC18EE900AC2
:10DE900016F054F941EC1A0B0221B0EE4A0AF0EEEA
:10DEA0006A0AB94814F00CF9B74814F0AFF8152114
:10DEB000B74813F01BFC1BEE100A16F03FF941ECBB
:10DEC000190B0221B0EE490AF0EE690AAE4814F0CF
:10DED000F7F8AD4814F09AF81421AE4813F006FC98
:10DEE0000099A94814F0E2F8A74814F08FF8192116
:10DEF000A94813F0FBFB4146A34814F0D7F8A24809
:10DF000014F084F8012F00F02F82022F00F00E820F
:10DF1000002F00F0A8814FF0000908EE109A4B4640
:10DF2000CDF81090CDF80C90CDF80890CB46EDB21E
:10DF300028460121F6B2059311F0DEF830460121A2
:10DF400011F0DAF8B8EEC88ADFED947A944C68EEF6
:10DF5000277A0DF1300AFDEEE77A41F28832052189
:10DF60001CA8CDED017AFBF78BF88E4B029A1C931F
:10DF7000594650464FF0000BCDF8DCB010F028FAAF
:10DF8000DDED007A68EE8B8AF8EEE77A68EEA77A24
:10DF900017EE900A16F0D2F841EC100B14F010FEB8
:10DFA00051EC100B16F016FC019908EE100A5046C1
:10DFB00010F050FA494610F041FAFDEEC87A17EE1B
:10DFC000901A10F085FA03217748CDF834B013F099
:10DFD0008DFB08A96C4813F0F3FF1921734813F067
:10DFE00085FB08A9684813F0EBFF03216E4813F086
:10DFF0007DFB654814F00AF80E216D4813F076FB9E
:10E00000B0EE4A0AF0EE6A0A02215F4814F058F8AE
:10E010005D4813F0FBFF0C21664813F067FBB0EE80
:10E02000490AF0EE690A0221574814F049F85648A7
:10E0300013F0ECFF0B21604813F058FB0099524895
:10E0400014F034F8504813F0E1FF0D215B4813F051
:10E050004DFB18EE100A16F071F841EC100B02217E
:10E06000494814F02DF8484813F0D0FF0D215448CA
:10E0700013F03CFB0199444814F018F8424813F09F
:10E08000C5FF0A214F4813F031FB03993E4814F0B5
:10E090000DF83D4813F0BAFF0E214B4813F026FB54
:10E0A0000499394814F002F8374813F0AFFF1121F2
:10E0B000464813F01BFB059B3348194613F0F6FF47
:10E0C000314813F0A3FF0321414813F00FFB08A9C7
:10E0D0002D4813F075FF1921344813F007FB08A9E8
:10E0E000294813F06DFF0321394813F0FFFA264841
:10E0F00013F08CFF369BCDF8D8B04AA903F10B0280
:10E1000001EB820201EB83031CA8012143F88CACD4
:10E11000B7EE000A42F8B4BCFDF7B0FA1E99002928
:10E1200000F0E280284610F0EDFF002840F0C680A5
:10E130002921284813F0DAFA134813F067FF1FA8C3
:10E1400013F0D2FE002424981E9410F0C1FA2598F2
:10E1500010F0BEFA0125204B21462A4603201D70EF
:10E16000F2F79CFC2A4621462046F2F797FC2A4605
:10E1700021462846F2F792FC32E000BFEC15FF1F63
:10E1800054A00200F8A302002408FF1F2CA40200E0
:10E1900044A402005CA4020074A402000AD7233C39
:10E1A000141CFF1F44850200E0A1020090A402009D
:10E1B000ACA40200BCA40200CCA402000CAA020081
:10E1C000D8A40200B09C0200E8A40200F8A4020057
:10E1D000CCAC020058A50200EC16FF1F0814FF1F6C
:10E1E0002A4621460220F2F759FC754D7548112147
:10E1F00013F07CFA2968744813F058FF724813F042
:10E2000005FFB8F1000F03D02A680D9B13442B6063
:10E2100011216C4813F06AFA29686B4813F046FF25
:10E22000694813F0F3FE1A21684813F05FFA394683
:10E23000654813F03BFF644813F0E8FE172164487B
:10E2400013F054FA604813F0E1FE624B1C931CA8D3
:10E25000FAF760FF08A814F067F820464BB0BDEC51
:10E26000088BBDE8F08F5C4908A814F025F901225D
:10E2700011463846E569A669F2F710FCD9F8343042
:10E2800003931A46D9F84430D9F85490CDF8109039
:10E2900003FB02F208EE102A052202924FF0060B51
:10E2A00045E610214D4813F021FA0121464813F0AC
:10E2B000FDFE454813F0AAFE0127D8E5304610F0D0
:10E2C00021FF00283FF434AFF3F712FF70B9236841
:10E2D0000793079A23680693069B9B1A042BF9D988
:10E2E0001E9900297FF41EAF0C467EE717213C489B
:10E2F00013F0FCF9344813F089FE1CA8FAF7B2FEBB
:10E30000012200210320F2F7C9FB00210846012267
:10E31000F2F7C4FB012210460021F2F7BFFB0122F5
:10E3200000210220F2F7BAFB01245EE72D4908A87C
:10E3300014F0C2F8012211463846256DE66CF2F75A
:10E34000ADFBD9F83C3003931A46D9F84C30D9F8D4
:10E350005C90CDF8109003FB02F208EE102A172211
:10E3600002924FF0100BE2E51F4908A814F0A4F840
:10E370003A4639463846256BE66AF2F78FFBD9F8FC
:10E38000383003931A46D9F84830D9F85890CDF868
:10E39000109003FB02F208EE102A142202924FF0B2
:10E3A000150BC4E51021114813F0A0F941460648A9
:10E3B00013F07CFE044813F029FE474657E500BFE2
:10E3C000B412FF1FF4A102002408FF1F24A50200BD
:10E3D00040A5020044850200AC980200D0A30200D0
:10E3E0000CA50200749902007CC30200E4A30200A1
:10E3F0002DE9F0412DED068BC2B0322101909448F9
:10E40000944EDFF888829FED948A944FB0EE409A44
:10E41000F0EE608A13F06AF9914813F0F7FD0122DB
:10E4200011460320F2F73AFB04AC41F28832052191
:10E4300014A8FAF725FE0025204602220321CDF874
:10E4400050802F950FF0C4FF326B336C03FB02F347
:10E4500007EE903AF8EEE77A204667EE887AFDEE0E
:10E46000E77A17EE901A0FF0F5FF316D0FF0E6FF27
:10E47000326B336C7B4E03FB02F307EE903AF8EEFF
:10E48000E77A204667EE887AFDEEE77A17EE901A73
:10E490000FF0E0FFDDED017A059529EE287AF8EE20
:10E4A000E77A67EE277A17EE900A15F047FE41ECFF
:10E4B000100B14F085FB51EC100B16F08BF908EEE5
:10E4C000100A1321684813F011F918EE100A15F01C
:10E4D00035FE41EC1A0B0221B0EE4A0AF0EE6A0A50
:10E4E0005F4813F0EDFD5E4813F090FD0C215F488E
:10E4F00013F0FCF8B0EE4A0AF0EE6A0A022158481E
:10E5000013F0DEFD564813F081FD0F21584813F03B
:10E51000EDF819EE100A15F011FE41EC100B022176
:10E520004F4813F0CDFD4E4813F070FD0B215148BC
:10E5300013F0DCF818EE900A15F000FE41EC100B19
:10E540000221474813F0BCFD454813F05FFD0A2146
:10E55000494813F0CBF80199414813F0A7FD404812
:10E5600013F054FDFDEEC87A204617EE901A0FF016
:10E57000AFFF2E9B2E9542AA02EB830242A90B33DA
:10E5800001EB830342F88C4CB7EE000A43F8B45C0D
:10E5900014A80121FDF772F8169B384CB3B1F3F7BC
:10E5A00071FD002806DB3868F3F75CFDC0B2532824
:10E5B000307038D023680393039A23680293029B38
:10E5C0009B1A042BF9D9169B002BE8D12C4C2D4813
:10E5D000142113F08BF82168214813F067FD2048BF
:10E5E00013F014FD2268059B264813441421236070
:10E5F00013F07CF821681A4813F058FD184813F0FE
:10E6000005FD3121204813F071F8154813F0FEFC88
:10E6100014A8CDF85080FAF77DFD284642B0BDEC35
:10E62000068BBDE8F08114A8FAF71CFD0122002139
:10E630000320F2F733FA002108460122F2F72EFAFE
:10E64000012210460021F2F729FA0125B2E700BFA6
:10E6500084A502000814FF1F0AD7233C4807FF1FA8
:10E660002408FF1FF413FF1FB8A50200CCA5020069
:10E67000DCA50200ECA50200F8A50200141CFF1F97
:10E680006418FF1F04A602001CA6020044850200B5
:10E690002DE9F04FDFF86083D8F81430012B14BF58
:10E6A0000820042087B0F2F775FED8F81030002B50
:10E6B00040F39281CB4CCC4DA146AA460126CB49D2
:10E6C00002A813F071FE002102A8F2F7ADFF02A824
:10E6D00013F02AFE2220F3F725F907EE906A0020B6
:10E6E000B8EEE70AF3F7C2F8C14902A813F05CFEDE
:10E6F000002102A8F2F798FF02A813F015FED8F83F
:10E700001430002B00F07A81012B40F05F81B94F6B
:10E710002068D7ED007A0193F0EE080AB8EEE70A18
:10E72000FFF766FE8346F3F7E3FC002840F05481D0
:10E73000019BBBF1000F40F04F81D5ED007AD9F875
:10E74000000001931946B8EEE70AF0EE000A4042D5
:10E75000FFF76CFB8346F3F7CBFC019B002840F0EE
:10E760003B81BBF1000F40F03781D7ED007AD9F83B
:10E7700000000193B8EEE70AF7EE000A4042FFF707
:10E7800037FE8346F3F7B4FC019B002840F0248158
:10E79000BBF1000F40F02081DAED007AD9F80000DB
:10E7A0001946B8EEE70AF7EE000AFFF73FFB83468B
:10E7B000F3F79EFC002840F00F81BBF1000F40F002
:10E7C0000B812068D7ED007A4042B8EEE70AF7EEF9
:10E7D000000AFFF70DFE8346F3F78AFC002840F09D
:10E7E000FB80BBF1000F40F0F7802068D5ED007A88
:10E7F0004042B8EEE70A0121F0EE000AFFF716FBEF
:10E800008346F3F775FC002840F0E680BBF1000F6B
:10E8100040F0E280774B206893ED000AF0EE080AA2
:10E82000B8EEC00AFFF7E4FD8346F3F761FC002869
:10E8300040F0D280BBF1000F40F0CE80D5ED007AE1
:10E840002068B8EEE70A0121F1EE000AFFF7EEFAC0
:10E850008346F3F74DFC002840F0BE80BBF1000F6B
:10E8600040F0BA802068D5ED007A4042B8EEE70A61
:10E870000121F2EE000AFFF7D9FA8346F3F738FCDC
:10E88000002840F0A980BBF1000F40F0A58020686F
:10E89000D7ED007A4042B8EEE70AF0EE080AFFF73B
:10E8A000A7FD8346F3F724FC002840F09580BBF1D8
:10E8B000000F40F09180D5ED007A2068B8EEE70AAD
:10E8C0000121F0EE000AFFF7B1FA8346F3F710FCDE
:10E8D000002840F08180BBF1000F7DD1454B2068BE
:10E8E0001B68019307EE903AF7EE000AB8EEE70ACC
:10E8F000FFF77EFD8346F3F7FBFB00286CD1BBF1ED
:10E90000000F69D12068D5ED007A4042B8EEE70AE1
:10E910000121F7EE000AFFF789FA8346F3F7E8FBD7
:10E92000002859D1BBF1000F56D1324B206893ED2E
:10E93000000AF7EE000AB8EEC00AFFF759FD834659
:10E94000F3F7D6FB002847D1BBF1000F44D1D5ED3A
:10E95000007A2068B8EEE70A0121F0EE000AFFF71E
:10E9600065FA8346F3F7C4FBB0BBBBF1000F33D1AC
:10E9700097ED000A2068B8EEC00A4042F0EE080A9F
:10E98000FFF736FD0746F3F7B3FB28BB27BBD5EDF2
:10E99000007A2068B8EEE70A0121F1EE000AFFF7DD
:10E9A00045FA0746F3F7A4FBB0B9AFB92068D5ED37
:10E9B000007A4042B8EEE70A0121F2EE000AFFF7C2
:10E9C00035FA0746F3F794FB30B92FB9D8F8103071
:10E9D0000136B342BFF673AEF2F74AFE07B0BDE8A8
:10E9E000F08F00BF4007FF1F1C13FF1F7491020030
:10E9F000448B02008415FF1F0814FF1FD5ED007A19
:10EA00002068B8EEE70A0121F0EE080AFFF70EFAD7
:10EA10000746F3F76DFB0028DED1002FDCD1AB4FAA
:10EA2000D9F80000D7ED007A4042B8EEE70AF0EEE0
:10EA3000000AFFF7DDFC8346F3F75AFB0028CBD131
:10EA4000BBF1000FC8D1D9F80000DAED007A4042DE
:10EA5000B8EEE70A0121F7EE000AFFF7E7F983466F
:10EA6000F3F746FB0028B7D1BBF1000FB4D1D7EDC7
:10EA7000007AD9F80000B8EEE70AF7EE000AFFF7CF
:10EA8000B7FC8346F3F734FB0028A5D1BBF1000F98
:10EA9000A2D1D9F80000DAED007A4042B8EEE70AD8
:10EAA0000121F7EE000AFFF7C1F98346F3F720FBD7
:10EAB000002891D1BBF1000F8ED12068D7ED007AEC
:10EAC0004042B8EEE70AF0EE000AFFF791FC8346F9
:10EAD000F3F70EFB00287FF47FAFBBF1000F7FF44C
:10EAE0007BAFD5ED007A2068B8EEE70A0121F0EEA1
:10EAF000080AFFF79BF98346F3F7FAFA00287FF438
:10EB00006BAFBBF1000F7FF467AF704B20681B68E1
:10EB1000019307EE903AF1EE000AB8EEE70AFFF72C
:10EB200067FC8346F3F7E4FA00287FF455AFBBF1A6
:10EB3000000F7FF451AF654B206893ED000A40420F
:10EB4000B8EEC00AF2EE000AFFF752FC8346F3F774
:10EB5000CFFA00287FF440AFBBF1000F7FF43CAF49
:10EB60002068D5ED007A4042B8EEE70A0121F0EEC8
:10EB7000080AFFF75BF98346F3F7BAFA00287FF437
:10EB80002BAFBBF1000F7FF427AFD7ED007A2068E1
:10EB9000B8EEE70AF0EE000AFFF72AFC8346F3F727
:10EBA000A7FA00287FF418AFBBF1000F7FF414AF71
:10EBB000D5ED007A2068B8EEE70A0121F7EE000AE9
:10EBC000FFF734F98346F3F793FA00287FF404AF94
:10EBD000BBF1000F7FF400AF3C4B20681B68019332
:10EBE00007EE903A4042B8EEE70AF7EE000AFFF768
:10EBF000FFFB8346F3F77CFA00287FF4EDAEBBF110
:10EC0000000F7FF4E9AED5ED007A2068B8EEE70A90
:10EC10000121F7EE000AFFF709F98346F3F768FAD6
:10EC200000287FF4D9AEBBF1000F7FF4D5AE274B9F
:10EC3000206893ED000AF0EE000AB8EEC00AFFF774
:10EC4000D7FB8346F3F754FA00287FF4C5AEBBF137
:10EC5000000F7FF4C1AE2068D5ED007A4042B8EED7
:10EC6000E70A0121F0EE080AFFF7E0F88346F3F720
:10EC70003FFA00287FF4B0AEBBF1000F7FF4ACAEDA
:10EC800097ED000A2068114FB8EEC00AF1EE000AB5
:10EC9000FFF7AEFB8346F3F72BFA00287FF49CAE18
:10ECA000BBF1000F7FF498AE97ED000A2068B8EE34
:10ECB000C00A4042F2EE000AFFF79AFB0746F3F75C
:10ECC00017FA00283FF481AE86E600BF8415FF1FC7
:10ECD0002DE9F04FDFF8A883D8F81430012B14BFCA
:10ECE0000D20042087B0F2F755FBD8F81030002B28
:10ECF00040F3B382DD4CDE4DA146AA460127DD4933
:10ED000002A813F051FB002102A8F2F78DFC02A823
:10ED100013F00AFB2220F2F705FE07EE907A00209E
:10ED2000B8EEE70AF2F7A2FDD34902A813F03CFBC4
:10ED3000002102A8F2F778FC02A813F0F5FAD8F83F
:10ED40001430002B00F09082012B40F08082CB4EDB
:10ED50002068D6ED007A01934042B8EEE70A1946E2
:10ED6000F7EE000AFFF762F88346F3F7C1F90028CF
:10ED700040F07382019BBBF1000F40F06E82D5ED35
:10ED8000007AD9F800000193B8EEE70AF0EE080A1D
:10ED9000FFF72EFB8346F3F7ABF9019B002840F009
:10EDA0005C82BBF1000F40F05882D9F80000D6ED2C
:10EDB000007A19464042B8EEE70AF0EE000AFFF783
:10EDC00035F88346F3F794F9002840F04682BBF10A
:10EDD000000F40F04282D9F80000DAED007A40429C
:10EDE000B8EEE70AF7EE000AFFF702FB8346F3F7F7
:10EDF0007FF9002840F03182BBF1000F40F02D82F6
:10EE0000D6ED007A2068B8EEE70A0121F7EE000A95
:10EE1000FFF70CF88346F3F76BF9002840F01D82EA
:10EE2000BBF1000F40F019822068D5ED007A404216
:10EE3000B8EEE70AF7EE000AFFF7DAFA8346F3F7CF
:10EE400057F9002840F00982BBF1000F40F005821D
:10EE50008A4B20681B68019307EE903A4042B8EE57
:10EE6000E70A0121F0EE080AFEF7E0FF8346F3F718
:10EE70003FF9002840F0F181BBF1000F40F0ED8137
:10EE8000D5ED007A2068B8EEE70AF7EE000AFFF742
:10EE9000AFFA8346F3F72CF9002840F0DE81BBF18E
:10EEA000000F40F0DA81754B206893ED000A0121D4
:10EEB000B8EEC00AF7EE000AFEF7B8FF8346F3F794
:10EEC00017F9002840F0C981BBF1000F40F0C5815F
:10EED000D5ED007A2068B8EEE70AF7EE000AFFF7F2
:10EEE00087FA8346F3F704F9002840F0B681BBF1B6
:10EEF000000F40F0B2812068D6ED007A4042B8EEB3
:10EF0000E70A0121F0EE000AFEF790FF8346F3F7CF
:10EF1000EFF8002840F0A181BBF1000F40F09D8187
:10EF20002068D5ED007A4042B8EEE70AF0EE080A14
:10EF3000FFF75EFA8346F3F7DBF8002840F08D8197
:10EF4000BBF1000F40F089814C4B206893ED000A23
:10EF50000121B8EEC00AF1EE080AFEF767FF83460A
:10EF6000F3F7C6F8002840F07881BBF1000F40F0BD
:10EF70007481D5ED007A2068B8EEE70AF1EE000A58
:10EF8000FFF736FA8346F3F7B3F8002840F06581BF
:10EF9000BBF1000F40F061812068D6ED007A40425D
:10EFA000B8EEE70A0121F1EE0C0AFEF73FFF8346B7
:10EFB000F3F79EF8002840F05081BBF1000F40F0BD
:10EFC0004C812068D5ED007A4042B8EEE70AF0EEB9
:10EFD000080AFFF70DFA8346F3F78AF8002840F095
:10EFE0003C81BBF1000F40F03881244B20681B6846
:10EFF000019307EE903A4042B8EEE70A0121F0EEA5
:10F00000000AFEF713FF8346F3F772F8002840F07A
:10F010002481BBF1000F40F02081D5ED007A2068FB
:10F02000B8EEE70AF7EE000AFFF7E2F98346F3F7D6
:10F030005FF8002840F01181BBF1000F40F00D8116
:10F040000E4B206893ED000A0121B8EEC00AF7EEDE
:10F05000000AFEF7EBFE8346F3F74AF8002840F07B
:10F06000FC80BBF1000F40F0F8800BE04007FF1F71
:10F070008415FF1F74910200448B02001C13FF1FB4
:10F080000814FF1FD5ED007A2068B8EEE70AF7EE06
:10F09000000AFFF7ADF98346F3F72AF8002840F09D
:10F0A000DC80BBF1000F40F0D8802068D6ED007AFC
:10F0B0004042B8EEE70A0121F0EE080AFEF7B6FE7C
:10F0C0008346F3F715F8002840F0C780BBF1000F26
:10F0D00040F0C3802068D5ED007A4042B8EEE70AE0
:10F0E000F7EE000AFFF784F98346F3F701F80028EA
:10F0F00040F0B380BBF1000F40F0AF80594B206867
:10F1000093ED000A0121B8EEC00AF7EE000AFEF7FF
:10F110008DFE8346F2F7ECFF002840F09E80BBF1A5
:10F12000000F40F09A802068D5ED007A4042B8EE9A
:10F13000E70AF7EE000AFFF75BF98346F2F7D8FF1C
:10F14000002840F08A80BBF1000F40F086802068E4
:10F15000D6ED007A4042B8EEE70A0121F0EE000A4F
:10F16000FEF764FE8346F2F7C3FF002875D1BBF1BA
:10F17000000F72D1D5ED007A2068B8EEE70AF0EE04
:10F18000080AFFF735F98346F2F7B2FF002864D189
:10F19000BBF1000F61D1334B20681B68019307EE70
:10F1A000903A0121B8EEE70AF1EE040AFEF73EFEBE
:10F1B0008346F2F79DFF00284FD1BBF1000F4CD1E1
:10F1C000284B206893ED000A4042B8EEC00A0121A6
:10F1D000F1EE080AFEF72AFE8346F2F789FF0028BF
:10F1E0003BD1BBF1000F38D12068D5ED007A404209
:10F1F000B8EEE70AF1EE000AFFF7FAF88346F2F7F5
:10F2000077FF50BBBBF1000F27D196ED000A2068B5
:10F21000144EB8EEC00A0121F1EE0C0AFEF706FE0C
:10F220008346F2F765FFC0B9BBF1000F15D196ED2B
:10F23000000A2068B8EEC00A40420121F1EE0C0A33
:10F24000FEF7F4FD0646F2F753FF30B92EB9D8F8B1
:10F2500010300137BB42BFF652ADF2F709FA07B0E2
:10F26000BDE8F08F1C13FF1F2068D5ED007A4042E7
:10F27000B8EEE70AF7EE000AFFF7BAF80646F2F72B
:10F2800037FF0028E9D1002EE7D1DF4ED9F8000082
:10F29000D6ED007AF0EE080AB8EEE70A0121FEF793
:10F2A000C5FD8346F2F724FF0028D6D1BBF1000F3D
:10F2B000D3D1D9F80000DAED007A4042B8EEE70A7F
:10F2C000F0EE000AFFF794F88346F2F711FF0028EA
:10F2D000C3D1BBF1000FC0D1D9F80000D6ED007A40
:10F2E0004042B8EEE70A0121F7EE000AFEF79EFD64
:10F2F0008346F2F7FDFE0028AFD1BBF1000FACD181
:10F30000DAED007AD9F80000B8EEE70AF7EE000A65
:10F31000FFF76EF88346F2F7EBFE00289DD1BBF1B4
:10F32000000F9AD12068D6ED007A4042B8EEE70A85
:10F330000121F7EE000AFEF779FD8346F2F7D8FEC9
:10F3400000288AD1BBF1000F87D12068D5ED007A63
:10F350004042B8EEE70AF0EE080AFFF749F88346A4
:10F36000F2F7C6FE00287FF478AFBBF1000F7FF400
:10F3700074AFA54B20681B68019307EE903A0121FA
:10F38000B8EEE70AF7EE000AFEF750FD8346F2F703
:10F39000AFFE00287FF461AFBBF1000F7FF45DAFDB
:10F3A000D5ED007A2068B8EEE70AF7EE000AFFF71D
:10F3B0001FF88346F2F79CFE00287FF44EAFBBF1A6
:10F3C000000F7FF44AAF904B206893ED000A0121B3
:10F3D000B8EEC00AF7EE000AFEF728FD8346F2F702
:10F3E00087FE00287FF439AFBBF1000F7FF435AF03
:10F3F0002068D5ED007A4042B8EEE70AF0EE000A48
:10F40000FEF7F6FF8346F2F773FE00287FF425AF80
:10F41000BBF1000F7FF421AF2068D6ED007A4042A7
:10F42000B8EEE70A0121F0EE080AFEF7FFFC83467A
:10F43000F2F75EFE00287FF410AFBBF1000F7FF4FF
:10F440000CAFD5ED007A2068B8EEE70AF1EE080AB5
:10F45000FEF7CEFF8346F2F74BFE00287FF4FDAEA9
:10F46000BBF1000F7FF4F9AE674B206893ED000A03
:10F470000121B8EEC00AF1EE000AFEF7D7FC834680
:10F48000F2F736FE00287FF4E8AEBBF1000F7FF400
:10F49000E4AE2068D5ED007A4042B8EEE70AF1EE1E
:10F4A0000C0AFEF7A5FF8346F2F722FE00287FF440
:10F4B000D4AEBBF1000F7FF4D0AE2068D6ED007A59
:10F4C0004042B8EEE70A0121F0EE080AFEF7AEFC72
:10F4D0008346F2F70DFE00287FF4BFAEBBF1000FAC
:10F4E0007FF4BBAE2068D5ED007A4042B8EEE70A63
:10F4F000F0EE000AFEF77CFF8346F2F7F9FD0028E4
:10F500007FF4ABAEBBF1000F7FF4A7AE3E4B20689B
:10F510001B68019307EE903A0121B8EEE70AF7EE77
:10F52000000AFEF783FC8346F2F7E2FD00287FF431
:10F5300094AEBBF1000F7FF490AED5ED007A206859
:10F54000B8EEE70AF7EE000AFEF752FF8346F2F73D
:10F55000CFFD00287FF481AEBBF1000F7FF47DAEBC
:10F56000294B206893ED000A0121B8EEC00AF7EE9E
:10F57000000AFEF75BFC8346F2F7BAFD00287FF431
:10F580006CAEBBF1000F7FF468AE2068D5ED007A59
:10F590004042B8EEE70AF0EE080AFEF729FF83467C
:10F5A000F2F7A6FD00287FF458AEBBF1000F7FF400
:10F5B00054AE2068D6ED007A4042B8EEE70A012149
:10F5C000F7EE000AFEF732FC8346F2F791FD0028C1
:10F5D0007FF443AEBBF1000F7FF43FAED5ED007A70
:10F5E0002068B8EEE70AF7EE000AFEF701FF83464F
:10F5F000F2F77EFD00287FF430AEBBF1000F7FF400
:10F600002CAE014B206801E01C13FF1F93ED000A94
:10F610004042B8EEC00A0121F7EE000AFEF706FCF0
:10F620008346F2F765FD00287FF417AEBBF1000FAB
:10F630007FF413AE2068D5ED007A4042B8EEE70AB9
:10F64000F0EE000AFEF7D4FE8346F2F751FD0028E3
:10F650007FF403AEBBF1000F7FF4FFAD96ED000A1F
:10F660002068384EB8EEC00A0121F0EE080AFEF715
:10F67000DDFB8346F2F73CFD00287FF4EEADBBF1E5
:10F68000000F7FF4EAADD5ED007A2068B8EEE70A06
:10F69000F1EE040AFEF7ACFE8346F2F729FD0028DE
:10F6A0007FF4DBADBBF1000F7FF4D7AD2068D5ED63
:10F6B000007A4042B8EEE70AF1EE080AFEF798FE3B
:10F6C0008346F2F715FD00287FF4C7ADBBF1000FAC
:10F6D0007FF4C3AD96ED000A2068B8EEC00A404240
:10F6E0000121F1EE000AFEF7A1FB0646F2F700FD4C
:10F6F00000287FF4B2AD002E7FF4AFADD5ED007AD7
:10F700002068B8EEE70AF1EE0C0AFEF771FE064635
:10F71000F2F7EEFC00287FF4A0AD002E7FF49DAD43
:10F720002068D5ED007A4042B8EEE70AF1EE0C0A07
:10F73000FEF75EFE0646F2F7DBFC00283FF486ADDE
:10F740008BE500BF1C13FF1F2DE9F04FDFF8F0829F
:10F75000D8F81430012B14BF0420032087B0F1F730
:10F7600019FED8F81030002B40F3C680B04DDFF8FA
:10F77000D4922F46CA460124AE4902A812F014FEC4
:10F78000002102A8F1F750FF02A812F0CDFD2220BF
:10F79000F2F7C8F807EE904A0020B8EEE70AF2F751
:10F7A00065F8A54902A812F0FFFD002102A8F1F7B3
:10F7B0003BFF02A812F0B8FDD8F81430002B00F07F
:10F7C000A080012B40F092809C4E2868D6ED007AF4
:10F7D0000193F0EE080AB8EEE70AFEF709FE834649
:10F7E000F2F786FC002840F08780019BBBF1000FF8
:10F7F00040F08280D9ED007A386801931946B8EE5E
:10F80000E70AF0EE080A4042FEF710FB8346F2F7E3
:10F810006FFC019B00286FD1BBF1000F6CD1D6EDBE
:10F82000007A38680193B8EEE70AF0EE000A404229
:10F83000FEF7DEFD8346F2F75BFC019B00285BD1FF
:10F84000BBF1000F58D1DAED007A38681946B8EEEE
:10F85000E70AF7EE000AFEF7E9FA8346F2F748FCFA
:10F86000002849D1BBF1000F46D196ED000A286867
:10F87000724EB8EEC00AF7EE000AFEF7B9FD8346F5
:10F88000F2F736FCC0BBBBF1000F35D1D9ED007AE1
:10F890002868B8EEE70A0121F7EE000AFEF7C6FA7B
:10F8A0008346F2F725FC38BBBBF1000F24D196ED5F
:10F8B000000A2868B8EEC00A4042F0EE000AFEF7DF
:10F8C00097FD0646F2F714FCB0B9AEB92868D9ED39
:10F8D000007A4042B8EEE70A0121F0EE080AFEF78E
:10F8E000A5FA0646F2F704FC30B92EB9D8F8103064
:10F8F0000134A342BFF640AFF1F7BAFE07B0BDE84E
:10F90000F08FD9ED007A2868B8EEE70A0121F0EE11
:10F91000080AFEF78BFA0646F2F7EAFB0028EBD15D
:10F92000002EE9D1454E3868D6ED007A4042B8EE57
:10F93000E70AF0EE080AFEF75BFD8346F2F7D8FB14
:10F940000028D9D1BBF1000FD6D13868DAED007AA2
:10F950004042B8EEE70A0121F0EE000AFEF766FA2F
:10F960008346F2F7C5FB0028C6D1BBF1000FC3D117
:10F97000D6ED007A3868B8EEE70AF7EE000AFEF72F
:10F9800037FD8346F2F7B4FB0028B5D1BBF1000F79
:10F99000B2D1DAED007A3868B8EEE70A0121F7EE65
:10F9A000000AFEF743FA8346F2F7A2FB0028A3D130
:10F9B000BBF1000FA0D196ED000A28681F4EB8EEEB
:10F9C000C00AF7EE000AFEF713FD8346F2F790FB3C
:10F9D000002891D1BBF1000F8ED12868D9ED007AB3
:10F9E0004042B8EEE70A0121F0EE000AFEF71EFAE7
:10F9F0008346F2F77DFB00287FF47EAFBBF1000F5A
:10FA00007FF47AAF96ED000A2868B8EEC00A40424B
:10FA1000F0EE080AFEF7ECFC0646F2F769FB002858
:10FA20003FF463AFF1F724FE07B0BDE8F08F00BFED
:10FA30004007FF1F74910200448B02008415FF1FD2
:10FA40000814FF1F1C13FF1F2DE9F04FDFF8108370
:10FA5000D8F81430012B14BF0820032087B0F1F729
:10FA600099FCD8F81030002B40F36B81B74CB84D9F
:10FA7000A146AA460126B74902A812F095FC00212A
:10FA800002A8F1F7D1FD02A812F04EFC2220F1F7F6
:10FA900049FF07EE906A0020B8EEE70AF1F7E6FEAC
:10FAA000AD4902A812F080FC002102A8F1F7BCFDCC
:10FAB00002A812F039FCD8F81430002B00F0528163
:10FAC000012B40F03881A54F2068D7ED007A0193D3
:10FAD000F0EE080AB8EEE70AFEF78AFC8346F2F772
:10FAE00007FB002840F02D81019BBBF1000F40F087
:10FAF0002881D5ED007AD9F8000001931946B8EEB7
:10FB0000E70AF0EE080A4042FEF790F98346F2F762
:10FB1000EFFA019B002840F01481BBF1000F40F088
:10FB20001081D7ED007AD9F800000193B8EEE70A0A
:10FB3000F0EE000A4042FEF75BFC8346F2F7D8FA8B
:10FB4000019B002840F0FD80BBF1000F40F0F980E0
:10FB5000DAED007AD9F800001946B8EEE70AF7EEB8
:10FB6000000AFEF763F98346F2F7C2FA002840F074
:10FB7000E880BBF1000F40F0E480D7ED007A206808
:10FB8000B8EEE70AF7EE000AFEF732FC8346F2F71A
:10FB9000AFFA002840F0D580BBF1000F40F0D180D3
:10FBA000D5ED007A2068B8EEE70A0121F7EE000AE9
:10FBB000FEF73CF98346F2F79BFA002840F0C1803B
:10FBC000BBF1000F40F0BD80644B20681B680193BF
:10FBD00007EE903A4042B8EEE70AF0EE000AFEF770
:10FBE00007FC8346F2F784FA002840F0AA80BBF1B4
:10FBF000000F40F0A6802068D5ED007A4042B8EEB4
:10FC0000E70A0121F1EE040AFEF710F98346F2F744
:10FC10006FFA002840F09580BBF1000F40F0918012
:10FC20004E4B206893ED000AF0EE000AB8EEC00AD1
:10FC3000FEF7DEFB8346F2F75BFA002840F0818096
:10FC4000BBF1000F7DD1D5ED007A2068B8EEE70A50
:10FC50000121F7EE000AFEF7E9F88346F2F748FAC9
:10FC600000286ED1BBF1000F6BD12068D7ED007A70
:10FC70004042B8EEE70AF7EE000AFEF7B9FB83460A
:10FC8000F2F736FA00285CD1BBF1000F59D1D5ED5F
:10FC9000007A2068B8EEE70A0121F7EE000AFEF7C5
:10FCA000C5F88346F2F724FA00284AD1BBF1000FC9
:10FCB00047D12A4B206893ED000AF0EE000AB8EE17
:10FCC000C00AFEF795FB8346F2F712FAC8BBBBF1F8
:10FCD000000F36D12068D5ED007A4042B8EEE70A31
:10FCE0000121F0EE080AFEF7A1F88346F2F700FAC8
:10FCF00038BBBBF1000F24D197ED000A2068B8EEA5
:10FD0000C00A4042F0EE080AFEF772FB0746F2F71F
:10FD1000EFF9B0B9AFB92068D5ED007A4042B8EE3E
:10FD2000E70A0121F7EE000AFEF780F80746F2F72E
:10FD3000DFF930B92FB9D8F810300136B342BFF629
:10FD40009AAEF1F795FC07B0BDE8F08F4007FF1FB2
:10FD50001C13FF1F74910200448B02008415FF1FC7
:10FD60000814FF1FD5ED007A2068B8EEE70A0121DC
:10FD7000F0EE080AFEF75AF80746F2F7B9F900283C
:10FD8000DFD1002FDDD1974FD9F80000D7ED007AF1
:10FD90004042B8EEE70AF0EE080AFEF729FB834678
:10FDA000F2F7A6F90028CCD1BBF1000FC9D1D9F8E0
:10FDB0000000DAED007A4042B8EEE70A0121F0EEE9
:10FDC000000AFEF733F88346F2F792F90028B8D11B
:10FDD000BBF1000FB5D1D7ED007AD9F80000B8EE2D
:10FDE000E70AF7EE000AFEF703FB8346F2F780F915
:10FDF0000028A6D1BBF1000FA3D1DAED007AD9F823
:10FE00000000B8EEE70A0121F7EE000AFEF70EF84F
:10FE10008346F2F76DF9002893D1BBF1000F90D122
:10FE2000D7ED007A2068B8EEE70AF7EE000AFEF791
:10FE3000DFFA8346F2F75CF9002882D1BBF1000FAC
:10FE40007FF47FAF2068D5ED007A4042B8EEE70A34
:10FE50000121F0EE000AFDF7E9FF8346F2F748F9C9
:10FE600000287FF46EAFBBF1000F7FF46AAF5D4BEB
:10FE700020681B68019307EE903A4042B8EEE70A0B
:10FE8000F1EE040AFEF7B4FA8346F2F731F90028DE
:10FE90007FF457AFBBF1000F7FF453AFD5ED007A7D
:10FEA0002068B8EEE70A0121F0EE000AFDF7BEFF78
:10FEB0008346F2F71DF900287FF443AFBBF1000F32
:10FEC0007FF43FAF474B206893ED000AF7EE000A3E
:10FED000B8EEC00AFEF78CFA8346F2F709F900285B
:10FEE0007FF42FAFBBF1000F7FF42BAF2068D5ED6F
:10FEF000007A4042B8EEE70A0121F7EE000AFDF76A
:10FF000095FF8346F2F7F4F800287FF41AAFBBF1AF
:10FF1000000F7FF416AFD7ED007A2068B8EEE70A3D
:10FF2000F7EE000AFEF764FA8346F2F7E1F80028DC
:10FF30007FF407AFBBF1000F7FF403AFD5ED007A7C
:10FF40002068B8EEE70A0121F0EE000AFDF76EFF27
:10FF50008346F2F7CDF800287FF4F3AEBBF1000F33
:10FF60007FF4EFAE1F4B206893ED000A4042B8EEDD
:10FF7000C00AF0EE080AFEF73BFA8346F2F7B8F83B
:10FF800000287FF4DEAEBBF1000F7FF4DAAE20680C
:10FF9000D5ED007A4042B8EEE70A0121F0EE080AFA
:10FFA000FDF744FF8346F2F7A3F800287FF4C9AEBB
:10FFB000BBF1000F7FF4C5AE97ED000A2068B8EEE4
:10FFC000C00A4042F7EE000AFEF712FA0746F2F7BF
:10FFD0008FF800283FF4AEAEF1F74AFB07B0BDE85A
:10FFE000F08F00BF8415FF1F2DE9F04FA54FDFF8FC
:10FFF000B4927B69012B14BF0320022087B0F1F774
:020000021000EC
:10000000C9F91421A04811F071FBD9F800109F48DC
:1000100012F04CF89D4811F0F9FF3B69002B40F3BA
:10002000B880DFF88482012446461221984811F0F6
:100030005DFB2146954812F039F8944811F0E6FF2F
:10004000944902A812F0B0F9002102A8F1F7ECFAE5
:1000500002A812F069F92220F1F764FC07EE904A39
:100060000020B8EEE70AF1F701FC8B4902A812F074
:100070009BF9002102A8F1F7D7FA02A812F054F96F
:10008000D7F814A0BAF1000F00F08880BAF1010F80
:100090007AD114218148824D11F028FBD9F8001043
:1000A0007A4812F003F8794811F0B0FFD5ED007AE4
:1000B000D8F80000B8EEE70AF0EE000AFEF798F96B
:1000C0008346F2F715F8002863D1BBF1000F60D129
:1000D000744B30681B68019307EE903A4042B8EECB
:1000E000E70A5146F0EE000AFDF7A0FE8346F1F75D
:1000F000FFFF00284DD1BBF1000F4AD13068D5ED8C
:10010000007A4042B8EEE70AF7EE000AFEF770F90F
:100110008346F1F7EDFF00283BD1BBF1000F38D14A
:10012000604B306893ED000A5146B8EEC00A404279
:10013000F7EE000AFDF77AFE8246F1F7D9FF40BBE1
:10014000BAF1000F25D195ED000AD8F80000B8EEFD
:10015000C00A4042F7EE000AFEF74AF90546F1F7F9
:10016000C7FFB0B9ADB9D8F80000D9ED007A404268
:10017000B8EEE70A0121F0EE000AFDF757FE05464A
:10018000F1F7B6FF28B925B93B690134A342BFF6A0
:100190004CAFF1F76DFA07B0BDE8F08FD9ED007AFA
:1001A000D8F80000DFF8FCA0B8EEE70A0121F0EE75
:1001B000000AFDF73BFE0546F1F79AFF0028E8D15B
:1001C000002DE6D1364D3068D5ED007A4042B8EECC
:1001D000E70AF0EE000AFEF70BF98346F1F788FF15
:1001E0000028D6D1BBF1000FD3D13068DAED007A08
:1001F0004042B8EEE70A0121F7EE000AFDF716FECD
:100200008346F1F775FF0028C3D1BBF1000FC0D1C1
:10021000D5ED007A3068B8EEE70AF7EE000AFEF78F
:10022000E7F88346F1F764FF0028B2D1BBF1000F75
:10023000AFD19AED000A3068B8EEC00A4042012101
:10024000F7EE000AFDF7F2FD8246F1F751FF0028B4
:100250009FD1BAF1000F9CD195ED000AD8F80000AB
:10026000B8EEC00A4042F0EE000AFEF7C1F80546BB
:10027000F1F73EFF002886D0F1F7FAF907B0BDE8A4
:10028000F08F00BF0814FF1F50A602002408FF1FB4
:1002900068A6020074910200448B02007CA6020052
:1002A0008415FF1F1C13FF1F4007FF1F2DE9F04F90
:1002B000DFF8C092D9F81430012B14BF06200220B9
:1002C00087B0F1F767F8D9F81030002B40F342817E
:1002D000A34CA44DA0460126A34902A812F064F83D
:1002E000002102A8F1F7A0F902A812F01DF82220BF
:1002F000F1F718FB07EE906A0020B8EEE70AF1F775
:10030000B5FA9A4902A812F04FF8002102A8F1F7B5
:100310008BF902A812F008F8D9F814A0BAF1000F6E
:1003200000F02A81BAF1010F40F00E81904F206851
:10033000D7ED007AF7EE000AB8EEE70A5146FDF76E
:1003400075FD8346F1F7D4FE002840F00381BBF130
:10035000000F40F0FF80D8F80000D7ED007A40424F
:10036000B8EEE70A5146F7EE000AFDF75FFD834657
:10037000F1F7BEFE002840F0ED80BBF1000F40F029
:10038000E980D8F80000D5ED007A4042B8EEE70ADF
:10039000F0EE000AFEF72CF88346F1F7A9FE0028DC
:1003A00040F0D880BBF1000F40F0D480D8F80000B6
:1003B000D7ED007A51464042B8EEE70AF0EE000A67
:1003C000FDF734FD8346F1F793FE002840F0C2802C
:1003D000BBF1000F40F0BE802068D5ED007A4042AE
:1003E000B8EEE70AF0EE000AFEF702F88346F1F7EE
:1003F0007FFE002840F0AE80BBF1000F40F0AA80E5
:10040000D7ED007A2068B8EEE70A0121F7EE000A7E
:10041000FDF70CFD8346F1F76BFE002840F09A8053
:10042000BBF1000F40F096802068D5ED007A404285
:10043000B8EEE70AF7EE000AFDF7DAFF8346F1F7B8
:1004400057FE002840F08680BBF1000F40F082800C
:10045000474B206893ED000A4042B8EEC00A0121E4
:10046000F0EE080AFDF7E2FC8346F1F741FE0028B2
:1004700070D1BBF1000F6DD1D5ED007A2068B8EED8
:10048000E70AF7EE000AFDF7B3FF8346F1F730FE07
:1004900000285FD1BBF1000F5CD197ED000A206806
:1004A000334FB8EEC00A0121F7EE000AFDF7BEFC9B
:1004B0008346F1F71DFE00284CD1BBF1000F49D156
:1004C000D5ED007A2068B8EEE70AF7EE000AFDF7EE
:1004D0008FFF8346F1F70CFE00283BD1BBF1000FE4
:1004E00038D12068D7ED007A4042B8EEE70A012102
:1004F000F0EE000AFDF79AFC8346F1F7F9FD48BBE0
:10050000BBF1000F26D12068D5ED007A4042B8EE4D
:10051000E70AF0EE000AFDF76BFF8346F1F7E8FD0E
:10052000C0B9BBF1000F15D197ED000A2068B8EEF5
:10053000C00A40420121F7EE000AFDF777FC0746AA
:10054000F1F7D6FD30B92FB9D9F810300136B342E2
:10055000BFF6C2AEF1F78CF807B0BDE8F08F00BF70
:100560004007FF1F8415FF1F74910200448B020097
:100570001C13FF1F0814FF1FD5ED007A2068B8EE8A
:10058000E70AF7EE000AFDF733FF0746F1F7B0FD83
:100590000028DFD1002FDDD1844BD8F800001B6884
:1005A000019307EE903A4042B8EEE70AF7EE000AF0
:1005B000FDF71EFF0746F1F79BFD0028CAD1002F6B
:1005C000C8D17B4FD8F80000D7ED007AF0EE000AD2
:1005D000B8EEE70A0121FDF729FC8346F1F788FD13
:1005E0000028B7D1BBF1000FB4D1704BD8F8000090
:1005F0001B68019307EE903A4042B8EEE70AF0EE2E
:10060000000AFDF7F5FE8346F1F772FD0028A1D13F
:10061000BBF1000F9ED1D8F80000D7ED007A404220
:10062000B8EEE70A0121F7EE000AFDF7FFFB83466B
:10063000F1F75EFD00288DD1BBF1000F8AD1D5ED19
:10064000007A2068B8EEE70AF7EE000AFDF7D0FE60
:100650008346F1F74DFD00287FF47CAFBBF1000F1E
:100660007FF478AF2068D7ED007ADFF844A14042EC
:10067000B8EEE70A0121F7EE000AFDF7D7FB834643
:10068000F1F736FD00287FF465AFBBF1000F7FF472
:1006900061AF2068D5ED007A4042B8EEE70AF0EE8F
:1006A000080AFDF7A5FE8346F1F722FD00287FF436
:1006B00051AFBBF1000F7FF44DAF9AED000A2068F7
:1006C000B8EEC00A0121F7EE000AFDF7AFFB834642
:1006D000F1F70EFD00287FF43DAFBBF1000F7FF472
:1006E00039AFD5ED007A2068B8EEE70AF7EE000AD8
:1006F000FDF77EFE8346F1F7FBFC00287FF42AAF6E
:10070000BBF1000F7FF426AF97ED000A2068284F59
:10071000B8EEC00A0121F7EE000AFDF787FB834619
:10072000F1F7E6FC00287FF415AFBBF1000F7FF472
:1007300011AF2068D5ED007A4042B8EEE70AF0EE3E
:10074000000AFDF755FE8346F1F7D2FC00287FF43E
:1007500001AFBBF1000F7FF4FDAE97ED000A2068FA
:10076000B8EEC00A40420121F0EE000AFDF75EFB40
:100770000746F1F7BDFC00287FF4ECAE002F7FF4B4
:10078000E9AE2068D5ED007A4042B8EEE70AF7EE10
:10079000000AFDF72DFE0746F1F7AAFC00283FF4FA
:1007A000D2AEF0F765FF07B0BDE8F08F8415FF1FEC
:1007B0001C13FF1F2DE9F041EAB0044641F28832D4
:1007C00005213CA8F8F75CFCDFF8C882CDF8F08082
:1007D000052206210CA8002657960DF0F9FD1422DB
:1007E00015211CA80DF0F4FD172210212CA80DF0E6
:1007F000EFFD1D219548964D964F10F077FF9648D6
:1008000011F004FC1821954810F070FF29689248F7
:1008100011F04CFC904811F0F9FB1221904810F0B7
:1008200065FF39688C4811F041FC8B4811F0EEFBF4
:10083000052C4DD80123A34013F0240100F02C8196
:10084000884A2D9613680593059913680493049BB1
:100850005B1A132BF9D90C218348844E10F046FF04
:100860002D997D4811F022FC7B4811F0CFFBF16EF1
:100870002CA80DF0EFFD316F0DF0E0FD29680DF0B3
:100880000DFE16217A4810F031FF316F72480023B7
:100890000A2211F0CBFB704811F0B8FB012211467F
:1008A0000220F0F7FBF8569B6AA903F10B0201EB5B
:1008B000820201EB830300252CAE43F88C6CB7EE6B
:1008C000000A01213CA842F8B45C5695FAF7D6FE1E
:1008D0003E9B684E684DFBB10D995F4811F0E6FBF9
:1008E0005D4811F093FBF1F7CDFB002807DB306882
:1008F000F1F7B8FBC0B25328287000F0A380594A22
:1009000013680793079913680693069B5B1A092BD4
:10091000F9D93E9B002BDFD1052C0ED8012202FA1B
:1009200004F414F0240140F0078114F0120340F0A5
:100930005A8114F0090F40F04F8108A84F4911F077
:1009400033FD08A80021F0F76FFE08A811F0ECFCB9
:1009500008A84B4911F028FD08A80021F0F764FE13
:1009600008A811F0E1FC08A8444911F01DFD08A8F1
:100970000021F0F759FE08A811F0D6FC08A840495C
:1009800011F012FD08A80021F0F74EFE08A811F0A2
:10099000CBFC08A83B4911F007FD08A80021F0F79F
:1009A00043FE08A811F0C0FC08A8354911F0FCFC72
:1009B00008A80021F0F738FE08A811F0B5FC08A837
:1009C000314911F0F1FC08A80021F0F72DFE08A82C
:1009D00011F0AAFC08A82A4911F0E6FC08A8002199
:1009E000F0F722FE08A811F09FFC08A8274911F093
:1009F000DBFC002108A8F0F717FE08A811F094FC12
:100A00002220F0F78FFFD7ED007A0020B8EEE70A3A
:100A1000F0F72CFF08A81E4911F0C6FC002108A819
:100A2000F0F702FE08A811F07FFC00233CA81D93FC
:100A3000CDF8F0800D933B602D93F8F76BFB6AB017
:100A4000BDE8F0813CA8F8F70DFB58E794A602003A
:100A5000F812FF1FB412FF1F2408FF1FB4A60200E4
:100A6000D0A60200141CFF1F34A70200EC15FF1FC4
:100A700044A702004807FF1FF413FF1FAC9E0200AB
:100A800030890200989E02005CA70200849B02004D
:100A9000448B02004485020013F0120053D113F07E
:100AA000090F3FF415AF534A0D9013680193019954
:100AB00013680093009B5B1A132BF9D90C214E4845
:100AC0004E4E10F013FE0D994D4811F0EFFA4C48C0
:100AD00011F09CFAF16D0CA80DF0BCFC316E0DF01C
:100AE000ADFC29680DF0DAFC1621464810F0FEFD39
:100AF000316E434800230A2211F098FA404811F061
:100B000085FA012211460020EFF7C8FF569B6AA91B
:100B100003F10B0201EB820201EB830300250CAE13
:100B200043F88C6CB7EE000A01213CA842F8B45C93
:100B30005695FAF7A3FDCBE6194602202D9B3B60A4
:100B4000EFF7ACFFF9E62B4A1D9113680393039965
:100B500013680293029B5B1A132BF9D90C212A48C4
:100B6000264E10F0C3FD1D99254811F09FFA244828
:100B700011F04CFA716E1CA80DF06CFCB16E0DF00A
:100B80005DFC29680DF08AFC1621204810F0AEFDAE
:100B9000B16E1B4800230A2211F048FA184811F0E0
:100BA00035FA012211461046EFF778FF569B6AA9E5
:100BB00003F10B0201EB820201EB830300251CAE63
:100BC00043F88C6CB7EE000A01213CA842F8B45CF3
:100BD0005695FAF753FD7BE60D993960184619468C
:100BE000EFF75CFFA9E61D9B3B601046EFF756FF51
:100BF000A3E600BF141CFF1FE4A60200EC15FF1FB4
:100C00002408FF1FF4A602000CA702001CA7020084
:100C10002DE9F04FDFF8A8B3DFF8A883DBF8002058
:100C2000D14ED8F81C40D8F818502DED028B002377
:100C3000012AD9B0336008EE900A08EE101A00F0CD
:100C4000AE82C0F08782022A00F023821F46029300
:100C5000994601930393E4B2EBB21D46204601216D
:100C600000930EF049FA284601210EF045FA0AAD2C
:100C700041F2883205212AA8F8F702FA4FF0000A5B
:100C8000BA4B2A93022203212846CDF814A10DF075
:100C90009FFB039B019A1AAE194630460DF098FB54
:100CA00098ED027ADBED0F7ADBF80420DBF82430D4
:100CB0009FEDAF6A67EE877A98ED007AF8EE476AA3
:100CC00003FB02F307EE103A67EEA67AD8ED016A4D
:100CD000B8EEC77AB8EE668A27EE067A67EE887AAB
:100CE000F8EEE88A284627EEA88AFDEEC77A17EEC6
:100CF000901A0DF0AFFBDBF808100DF09FFBFDEE36
:100D0000C87A17EE901A0DF0E3FB029930460DF009
:100D1000A1FB39460DF092FB49460DF0D9FB0821A5
:100D2000944810F0E3FC53460A22DBF80010924886
:100D300011F07CF9904811F069F908218F4810F002
:100D4000D5FC0D218E4810F0D1FC18EE100A13F0DE
:100D5000F5F941EC100B0221874811F0B1F98648F2
:100D600011F054F90821854810F0C0FC0C21854889
:100D700010F0BCFCDBF83C0013F0E0F941EC100B88
:100D800002217D4811F09CF97B4811F03FF90821C0
:100D9000784810F0ABFC09217B4810F0A7FCDBF889
:100DA000380013F0CBF941EC100B0221724811F01E
:100DB00087F9714811F02AF908216E4810F096FC65
:100DC0000D216F4810F092FC49466B4811F06EF906
:100DD000694811F01BF9012203201146EFF75EFE6E
:100DE000DBF80000012800F0B081C0F0A8810228E3
:100DF00003D101221146EFF751FE37216348644FBA
:100E000010F074FC5C4811F001F9449B58AA02EB05
:100E1000830158A803F10C0200EB8202002341F881
:100E2000886C41F88C5CB7EE000A42F8B43C0221B1
:100E30002AA84493FAF722FC2C9B564E002B30D064
:100E400020460EF05FF98246002840F047812E21AF
:100E5000514810F04BFC484811F0D8F8B9F1000F98
:100E600000F35E816A681B9B3A603360F1F70AF910
:100E7000002809DB494B1868F1F7F4F8484BC0B279
:100E80005328187000F04581464A13680593059968
:100E900013680493049B5B1A092BF9D92C9B002B34
:100EA000CED1DBF80090404B6A681B991A60B9F10B
:100EB000010F316000F08A83C0F08A82B9F1020F1D
:100EC00000F0AE8106AC4FF0000901224946032034
:100ED000C5F80490CDF86C90EFF7E0FD08212748A5
:100EE00010F004FC3968244811F0E0F8224811F0B1
:100EF0008DF805212D4810F0F9FB31681E4811F0DE
:100F0000D5F81D4811F082F8D8F8A430012B00F074
:100F100035842749204611F047FA49462046F0F724
:100F200083FB204611F000FA2249204611F03CFADA
:100F300049462046F0F778FB204611F0F5F91E49A6
:100F4000204611F031FA49462046F0F76DFB204665
:100F500011F0EAF91949204611F026FA49462046CF
:100F6000F0F762FB30E000BFF812FF1F448502007B
:100F70000AD7233C70A702002408FF1FA49C02008C
:100F80007CA702008CA70200509E02009CA70200D2
:100F90006418FF1FB412FF1F449F02004807FF1F81
:100FA000F413FF1F141CFF1F6C15FF1FD09C0200C1
:100FB00060A802003089020074A80200688B020059
:100FC0001418FF1FEC15FF1F204611F0ADF98849DA
:100FD000204611F0E9F949462046F0F725FB204666
:100FE00011F0A2F98349204611F0DEF94946204666
:100FF000F0F71AFB204611F097F97F49204611F0CF
:10100000D3F949462046F0F70FFB204611F08CF942
:101010007A49204611F0C8F949462046F0F704FB0A
:10102000204611F081F97649204611F0BDF9494674
:101030002046F0F7F9FA204611F076F9714920467A
:1010400011F0B2F949462046F0F7EEFA204611F0C9
:101050006BF96749204611F0A7F949462046F0F799
:10106000E3FA204611F060F96249204611F09CF93C
:1010700049462046F0F7D8FA204611F055F9624B60
:101080002A932AA8F8F746F859B0BDEC028BBDE8C0
:10109000F08FDBF81C00DBF830209FED5C7AD8F88D
:1010A0003410D8F85040D8F84C50DBF8207002FBD0
:1010B00000F207EE902AF8EEE77A67EE877AFDEE07
:1010C000E77ACDED027A002900F07B83012900F058
:1010D00089839946172301931023BBE500980EF0EE
:1010E00011F800287FF4BEAE01902E21484810F080
:1010F000FDFA484810F08AFFB9F1000F019BBFF6D6
:10110000B1AE2DA8009310F0EFFE009B32982C9307
:101110000CE02AA8F7F77AFF3F4B01221A70B3E6DA
:101120002DA810F0E1FE3298CDF8B0A00DF0D0FA65
:1011300033980DF0CDFA384B01221A70B1E6012236
:1011400050461146EFF7AAFC57E602460146EFF774
:10115000A5FC52E6DBF80C10DBF828209FED2B7A7B
:101160009BED0E0ADBF8107002FB01F207EE902AED
:10117000F8EEE77A184667EE877A0523FDEEE77A00
:101180000193CDED027AEFF7C3FEB8EEC88A0623CD
:1011900028EE000AFDEEC07A17EE909A5AE5DBF8C9
:1011A0001410DBF82C309FED197A9BED0E0AD8F85D
:1011B0003040D8F82C50DBF8187003FB01F307EE31
:1011C000903AF8EEE77A142367EE877A1046FDEE40
:1011D000E77A0193CDED027AEFF79AFEB8EEC88A6E
:1011E000152328EE000AFDEEC07A17EE909A31E53D
:1011F000D09B0200448B020088A8020030890200C4
:101200009CA80200688B0200448502000AD7233C98
:10121000749F02002408FF1FEC16FF1F0000B44358
:10122000D8F80420D8F8003098ED027AD7ED006A9B
:101230001FED066ADFF888A3DFF888B303FB02F32B
:1012400007EE903AF8EE677AF8EEE66A67EE877A8C
:10125000484686EEA77A06AC07EE901AB8EEE70A83
:1012600067EE067ACAED007AEFF756FD2046CB49C5
:101270008BED000A11F098F800212046F0F7D4F920
:10128000204611F051F82220F0F74CFB9AED000AAD
:101290000020F0F7EBFA2046C14911F085F820460E
:1012A0000021F0F7C1F9204611F03EF82046BD4973
:1012B00011F07AF800212046F0F7B6F9204611F037
:1012C00033F82220F0F72EFB9BED000A0020F0F708
:1012D000CDFA2046B24911F067F820460021F0F718
:1012E000A3F9204611F020F82046AF4911F05CF830
:1012F00020460021F0F798F9204611F015F8204615
:10130000AA4911F051F820460021F0F78DF9204646
:1013100011F00AF82046A64911F046F820460021AF
:10132000F0F782F9204610F0FFFF20469F4911F0A8
:101330003BF820460021F0F777F9204610F0F4FF43
:1013400020469C4911F030F820460021F0F76CF956
:10135000204610F0E9FF2046944911F025F8204678
:101360000021F0F761F9204610F0DEFF2046924997
:1013700011F01AF820460021F0F756F9204610F037
:10138000D3FF2046894911F00FF820460021F0F7DD
:101390004BF9204610F0C8FF2046884911F004F8A8
:1013A00020460021F0F740F9204610F0BDFF20460E
:1013B0007E4910F0F9FF20460021F0F735F920466C
:1013C00010F0B2FF484601220021EFF767FB7AE5F3
:1013D000D8F80400D8F8003098ED027AD7ED006A0A
:1013E000D8F81040D8F80C2098ED055ADFED765A61
:1013F000DFF8CCA1DFF8CC9103FB00F307EE903AC5
:10140000F8EE677AB8EEE66A67EE877A07EE101AAA
:1014100002FB04F2F8EEC76A86EE277A06AC5F4953
:10142000204607EE902A66EE856AF8EE677A27EE88
:10143000257A86EEA76A8AED007A89ED006A10F0B7
:10144000B3FF00212046F0F7EFF8204610F06CFFC4
:101450002220F0F767FA9AED000A0020F0F706FA6A
:1014600020464F4910F0A0FF20460021F0F7DCF89D
:10147000204610F059FF20464A4910F095FF002100
:101480002046F0F7D1F8204610F04EFF2220F0F76A
:1014900049FA99ED000A0020F0F7E8F920464049A2
:1014A00010F082FF20460021F0F7BEF8204610F031
:1014B0003BFF20463C4910F077FF20460021F0F723
:1014C000B3F8204610F030FF2046384910F06CFF8A
:1014D00020460021F0F7A8F8204610F025FF20460E
:1014E000334910F061FF20460021F0F79DF82046B7
:1014F00010F01AFF20462D4910F056FF204600211B
:10150000F0F792F8204610F00FFF2046294910F01E
:101510004BFF20460021F0F787F8204610F004FF2B
:101520002046224910F040FF20460021F0F77CF8C9
:10153000204610F0F9FE20461F4910F035FF2046E6
:101540000021F0F771F8204610F0EEFE2046174912
:1015500010F02AFF20460021F0F766F8204610F030
:10156000E3FE2046154910F01FFF20460021F0F74A
:101570005BF8204610F0D8FE20460C4910F014FF0E
:1015800020460021F0F750F8204610F0CDFE002153
:1015900008460122EFF782FA95E400BF749B02002F
:1015A000448B0200849B0200D4A702003089020011
:1015B000E8A70200FCA7020024A8020010A802006D
:1015C0009416FF1FBC13FF1F0000B443D8F804207B
:1015D000D8F8003098ED027AD7ED006A1FED066A60
:1015E000DFF838A2DFF838B203FB02F307EE903AD7
:1015F000F8EE677AF8EEE66A67EE877A07EE101A79
:10160000B8EEC70A86EEA77A06AC67EE067ACAED90
:10161000007AEEF79DFF204675498BED000A10F029
:10162000C3FE00212046EFF7FFFF204610F07CFEAE
:101630002220F0F777F99AED000A0020F0F716F96A
:1016400020466C4910F0B0FE20460021EFF7ECFF79
:10165000204610F069FE2046674910F0A5FE0021E3
:101660002046EFF7E1FF204610F05EFE2220F0F763
:1016700059F99BED000A0020F0F7F8F820465D4983
:1016800010F092FE20460021EFF7CEFF204610F02A
:101690004BFE2046594910F087FE20460021EFF707
:1016A000C3FF204610F040FE2046554910F07CFE56
:1016B00020460021EFF7B8FF204610F035FE204607
:1016C000504910F071FE20460021EFF7ADFF204693
:1016D00010F02AFE20464A4910F066FE20460021FE
:1016E000EFF7A2FF204610F01FFE2046464910F0FB
:1016F0005BFE20460021EFF797FF204610F014FE16
:1017000020463F4910F050FE20460021EFF78CFFA5
:10171000204610F009FE20463C4910F045FE2046C8
:101720000021EFF781FF204610F0FEFD20463449EE
:1017300010F03AFE20460021EFF776FF204610F029
:10174000F3FD2046324910F02FFE20460021EFF72E
:101750006BFF204610F0E8FD2046294910F024FEDA
:1017600020460021EFF760FF204610F0DDFD4A46DD
:1017700048460021EFF792F9FFF7A5BB254920461F
:1017800010F012FE49462046EFF74EFF204610F0BB
:10179000CBFD1B49204610F007FE49462046EFF7D7
:1017A00043FF204610F0C0FD1B49204610F0FCFD11
:1017B00049462046EFF738FF204610F0B5FD1049A6
:1017C00053E49BED0E0AEFF7D9FAB8EEC88A172357
:1017D00028EE000A0193FDEEC07A102317EE909ACE
:1017E000FFF738BA9BED0E0AEFF762FBEDE700BF9B
:1017F000749B0200448B0200849B0200D4A7020069
:1018000030890200E8A70200FCA7020010A802002D
:1018100024A8020038A802004CA802009416FF1F5A
:10182000BC13FF1F2DE9F04FDFF84C83DFF89C93CA
:10183000D8F84830CD4AD9F81C40D9F818602DEDB9
:10184000028BD9B00025012B0090156000F0C085F7
:10185000C0F04885022B00F01384AA460295AB46DF
:1018600003952F46E4B220460121F6B20DF044FC68
:10187000304601210DF040FC41F2883205212AA8B2
:10188000F7F7FEFBBA4B2A930222002303210AA892
:10189000459301930CF09CFD3A4629461AA80CF09A
:1018A00097FDD8F80010D8F810209FEDB27AB24D0D
:1018B00002FB01F307EE903AF8EEE77A0AA867EE2A
:1018C000877AFDEEE77A17EE901A0CF0C3FDD8F890
:1018D00020100CF0B3FDD8F84C70002F00F02E84CF
:1018E000012F40F0FA8495ED0F6A9FEDA47AD9EDAF
:1018F000027A2A6BA86C95ED0E0AC6EE076A99E883
:101900000A0003FB01F35200019207EE103AB8EE11
:10191000477A9DED006A67EE277AB8EEC68A67EED1
:10192000A67A67EE887AFDEEE77ACDED007AEFF7DA
:10193000EFFA2B6B5B0007EE903AF8EEE77A80EE59
:10194000270A20EE088AFDEEC87A17EE905A3B214E
:101950008B48894F0FF0CAFE8A4810F057FB0D21C3
:1019600089480FF0C3FE0099864810F09FFB854818
:1019700010F04CFB112185480FF0B8FE844B8148D4
:10198000196810F093FB7F4810F040FB0A21814852
:101990000FF0ACFE29467B4810F088FB794810F028
:1019A00035FB3B2176480FF0A1FE764810F02EFB68
:1019B00002991AA80CF04EFD51460CF03FFD0E2185
:1019C00075480FF093FED8F800106E4810F06EFBCB
:1019D0006C4810F01BFB142170480FF087FED8F8FC
:1019E0001010684810F062FB664810F00FFB0D21E4
:1019F0006B480FF07BFE00230A22D8F820106148C4
:101A000010F014FB5F4810F001FB132165480FF044
:101A10006DFE00230A22D9F800105A4810F006FB88
:101A2000584810F0F3FA11215F480FF05FFE0023D1
:101A30000A22D9F80410534810F0F8FA514810F06F
:101A4000E5FA122159480FF051FED9F8080012F0BA
:101A500075FB41EC100B02214A4810F031FB49485C
:101A600010F0D4FAD8F84C30002B00F00984012B88
:101A70002AD110214E480FF039FEF86B12F05EFBB0
:101A800041EC100B02213F4810F01AFB3D4810F0CA
:101A9000BDFA0F2147480FF029FEB86B12F04EFB3C
:101AA00041EC100B0221374810F00AFB354810F0CA
:101AB000ADFA0C2140480FF019FE396B314810F097
:101AC000F5FA304810F0A2FA0D212F480FF00EFE63
:101AD00000992C4810F0EAFA2A4810F097FA0A21E7
:101AE0002C480FF003FE2946264810F0DFFA25485F
:101AF00010F08CFA0B2131480FF0F8FD02992148C3
:101B000010F0D4FA1F4810F081FA11212C480FF080
:101B1000EDFD59461B4810F0C9FA1A4810F076FA44
:101B20000A2128480FF0E2FD0399164810F0BEFA8A
:101B3000144810F06BFA012203201146EEF7AEFFB5
:101B4000D8F84800012800F08E84C0F0858402286F
:101B50003ED101221146EEF7A1FF23211A480FF0D2
:101B6000C5FD084810F052FA32E000BFF812FF1F1E
:101B7000448502000AD7233C8014FF1F0000B443B1
:101B8000A8A102002408FF1FE4A10200F4A10200A2
:101B9000B412FF1F08A2020014A2020024A2020035
:101BA0003CA20200FCA802001CA902003CA9020001
:101BB0008CA20200A0A20200B0A2020074A1020046
:101BC00084A102009CA10200C0A20200EC15FF1F2C
:101BD000019B002B40F3A080304F4FF0000A002102
:101BE0002F480FF083FD2F4810F010FA0D212E48DA
:101BF0000FF07CFDDDF800B02A48594610F056FA87
:101C0000284810F003FA0A2128480FF06FFD2946F2
